:1000000000800020BD01000025DF0000DDDE0000D3
:10001000DDDE0000DDDE0000DDDE0000DDDE0000F4
:10002000DDDE0000DDDE0000DDDE000025DF00009B
:1000300025DF0000DDDE0000A5D50000A9D6000008
:1000400025DF000025DF000025DF000025DF0000A0
:1000500025DF000025DF000025DF000025DF000090
:1000600025DF000025DF000025DF000025DF000080
:1000700025DF000025DF000025DF000025DF000070
:1000800025DF000025DF000025DF000025DF000060
:1000900025DF000025DF000025DF000025DF000050
:1000A000E1BA0000EDBA000025DF000025DF000006
:1000B00025DF000025DF000025DF000025DF000030
:1000C00025DF000025DF000025DF000025DF000020
:1000D00025DF000025DF000025DF000025DF000010
:1000E00025DF000025DF000025DF000025DF000000
:1000F00025DF00004103010025DF000011EA0000B8
:1001000025DF0000ADEC000025DF000025DF00004A
:1001100025DF000025DF000025DF000025DF0000CF
:1001200025DF000025DF000025DF000025DF0000BF
:1001300025DF000025DF000025DF000025DF0000AF
:1001400025DF000025DF000025DF000025DF00009F
:1001500095D70000A9D70000BDD70000D1D7000077
:1001600025DF0000C9EF000025DF000025DF0000CB
:1001700025DF000025DF000025DF000025DF00006F
:1001800025DF000025DF000025DF000025DF00005F
:1001900025DF000025DF000025DF000025DF00004F
:1001A00025DF000025DF000025DF000025DF00003F
:1001B00025DF000025DF000025DF0000564B4CF254
:1001C000205210B51A804DF628121A8000BF00BFC9
:1001D0000DF0ACFE514B4FF010621A60504A9A601D
:1001E000504ADA60504A136813F4807304D14F49BF
:1001F0000B604FF4A85313604D4B1A78110703D5C9
:100200001A7842F008021A704A4B4B492A221A7097
:100210004A4A4B4B8B4204D252F8040F43F8040B6A
:10022000F8E7484B484900228B4202D243F8042B9E
:10023000FAE74649464A002352F8230041F82300D2
:1002400001336F2BF8D1434B434A802103F8011B44
:100250009342FBD1414B3D4A1A60414B8A221A70AE
:10026000A3F5805324225A70A0221A709A7992071B
:10027000FCD59A79D406FCD43A4A937903F00C035E
:10028000082B384BF9D103221A7140225A719A79FE
:100290009006FCD5334A9179324B4906FBD5324A58
:1002A000324911600221516020221A709A7902F0BD
:1002B0000C020C2AFAD12E4B2E4A1A602E4B2F4AD2
:1002C0001A6000225A60072243F8042C2C4AC3F813
:1002D0000C2D62B60EF0DAF9144B1B68DA0705D55F
:1002E00028480DF0A7FF284B284A1A60284B1B7896
:1002F0005B0609D5244C254B22689A4204D121483B
:100300000DF098FF0023236011F0D2FA0DF014FED7
:100310000DF042FDFEE700BF0E2005403080044096
:10032000823F04000100002B10D0034014D0034092
:1003300002D0074000E00740EC9CFF1F345501004D
:100340004088FF1FEC9CFF1F30A5FF1F0082FF1F8E
:100350000000000000E400E05FE400E008ED00E0E1
:100360000050064000400640448004400000030165
:1003700004800440C010050014E000E0FF76010096
:1003800000002020485EE8601CE00340A5C3945AAA
:1003900000F00740FFFFFFFFFFFFFFFFFFFFFFFF32
:1003A000FFFFFFFFFFFFFFFFFFFFFFFFFFFFFFFF5D
:1003B000FFFFFFFFFFFFFFFFFFFFFFFFFFFFFFFF4D
:1003C000FFFFFFFFFFFFFFFFFFFFFFFFFFFFFFFF3D
:1003D000FFFFFFFFFFFFFFFFFFFFFFFFFFFFFFFF2D
:1003E000FFFFFFFFFFFFFFFFFFFFFFFFFFFFFFFF1D
:1003F000FFFFFFFFFFFFFFFFFFFFFFFFFFFFFFFF0D
:10040000FFFFFFFFFFFFFFFFFFFFFFFFDEF9FFFF23
:1004100010B5054C237833B9044B13B10448AFF33E
:1004200000800123237010BDEC9CFF1F0000000022
:1004300038550100084B10B51BB108490848AFF307
:1004400000800848036803B910BD074B002BFBD0A0
:10045000BDE81040184700BF00000000F09CFF1FDF
:1004600038550100EC9CFF1F0000000038B5044621
:10047000104621700A491D4610F0FCFF01464FF05E
:100480007E5011F0ABF8074910F0F4FFE5606060B2
:10049000256165610EF08AF8E061204638BD00BF35
:1004A000DB0FC9400024744938B50446104621705A
:1004B00009491D4610F0DEFF01464FF07E5011F055
:1004C0008DF8064910F0D6FFE56060602561656132
:1004D0000EF06CF8E06138BDDB0FC94000247449B0
:1004E00038B503780446032B20D8DFE803F01A1848
:1004F0001002C168406910F0B3FE0D4905466068FE
:1005000011F06CF80146284611F068F838BD08492A
:10051000406811F063F8E16810F0ACFF38BDC068C6
:1005200038BDC168406910F09BFE38BD002038BD61
:100530000024744970B504460E460EF037F805469F
:10054000E069281A10F042FFE3682361E561666103
:10055000A0610146606811F041F80146A0601048B2
:1005600011F03CF810F012FB0FF0B2FF10F024FE77
:10057000054601464FF07E5010F072FE616910F0A2
:1005800079FF21690646284610F074FF014630467F
:1005900010F068FEE0602046BDE87040FFF7A0BFA5
:1005A000000080BF38B50E201C4C0DF0CFFA21881A
:1005B0001B4B884205461A881DDA0023511AB1F5F3
:1005C000805FAABF1B03C3EB03330131142093FBED
:1005D000F1F10DF041FE134B1988F1B923889D42CA
:1005E00010DAC3F57F630F33282091FBF3F1BDE8E8
:1005F00038400DF031BE9042D4BFC1EB0003C1EBD7
:100600000203DBE740F6FF718D42D4BFC3EB050167
:10061000C3EB0101C1EB0131E3E738BDF09DFF1FE2
:10062000BA9FFF1F589FFF1F10B504460DF090F8AA
:10063000204610BD70B44C88A04220D9012301335C
:10064000DBB21CB2660031F8144084421D46F6D37A
:10065000A04211D005F10045013D965B31F815101F
:1006600032F81530401AF21A00FB02F0641A90FBBF
:10067000F4F4E01870BC7047905B70BC70470226C1
:100680000125E5E700280CDA064A434282FB0320F5
:10069000DA17C2EB600000EB4000A3EB8000C0F172
:1006A0000C007047ABAAAA2A38B5234B1B78002B45
:1006B0002CD015200DF04AFA204B1860204B1B88D7
:1006C000984203DA1F4C237863BB38BD1E4A148856
:1006D000A042A4EB0302A8BF20467F2A1CDDC01A5B
:1006E000C001541C90FBF4F4002CEBD0154B1A788D
:1006F0000AB901221A70154D2B689C4204D0144B84
:10070000E1B2187809F0B0FA2C6038BD11200EF073
:1007100039FB0A4B1860D1E7C01AC0EBC01090FB40
:10072000F2F4E1E70A4B0021187809F09DFA002362
:10073000064A2370136038BD0C9FFF1F189DFF1FD2
:10074000929DFF1FEC9FFF1F849FFF1FE49FFF1FD1
:100750006C9DFF1F38B50F200EF014FB1B4A1C4B7D
:1007600012881860C0F53B600830904220DB194BBE
:100770001B889842A3EB0204A8BF1846801A7F2C5E
:10078000C6BFC0010134C0EBC01090FBF4F47CB1D3
:10079000114B1A780AB901221A70104D2B689C422D
:1007A00004D00F4BE1B2187809F05EFA2C6038BD26
:1007B000094C237803B938BD094B0021187809F09A
:1007C00053FA0023054A2370136038BDF49DFF1FC0
:1007D000309DFF1F709FFF1F949FFF1FA49DFF1F51
:1007E0008A9DFF1FF0B40E8886420DD203F10043AC
:1007F000013B31F81350854202D9F0BCFFF71ABF14
:1008000032F81300F0BC70471088F0BC704700BF8E
:10081000094B1B880C2B09D8084A80B252F82320B8
:1008200028B143F6FE73984203D9108C70471088A4
:1008300070470349FFF7FEBE469DFF1FE42E0100EF
:10084000803001004B4B4C4A2DE9F0471E8814685C
:100850004A4BB442B3F80080494B33DB4445A8BF50
:100860004446A6421C60C8BF00202DDDC6EB080729
:10087000B7F5804F33DB80037B1C90FBF3F0FFF771
:10088000C7FF404A404B15881B88C0F3C61909FBB7
:1008900005F57F2D8246A8BF7F252BB3A64253DCEA
:1008A0004445D4BFC6EB0404C6EB08049F42CCBF4A
:1008B00003FB04445C43354BC8BF013794FBF7F797
:1008C0001F6013E034461E60C6EB0807A045D4BF86
:1008D000C6EB0800C6EB0400B7F5804FCBDAC0EBDF
:1008E000803090FBF7F0CAE7284A1360284C236851
:1008F000994508D0274B1B88002B34D1264B1B88E9
:100900006BBBC4F80090254C23689A4506D0214B58
:100910001B885A1F032A19D9C4F800A0204C236849
:100920009D420FD01F4B188848B11A4B1E4A1B8896
:10093000D35C834203D0C0B2E9B209F095F92560D7
:10094000BDE8F087BDE8F0870024AFE7164AD05C29
:100950002030C0B20AF07F0109F086F9DCE7484692
:1009600009F022FACDE7104A4946D05C09F07CF93B
:10097000C4E700BFF09DFF1F549FFF1FBA9FFF1FDA
:10098000109DFF1F209DFF1F229DFF1FC09FFF1F67
:10099000849DFF1F3C9FFF1FE29DFF1F409DFF1F87
:1009A000E49DFF1F4A9FFF1F148AFF1F2DE9F04F90
:1009B00001208BB00EF0E6F9DFF850B3CBF8000061
:1009C00000200EF0DFF9B34BB34A1B8810600C2BEC
:1009D00000F00582B14A00211F2B117037D0B04FB3
:1009E000B04B3A88B04E53F8225000233370AF4BCF
:1009F000AF4A1B88AF491288013B012A31F91330F5
:100A0000059300F00682AC4B0193AC4B0293DFF8E8
:100A10000083DFF8009300230093A94B1B88012B70
:100A200000F04D82DFF8F0A2A64B0393DAF8004005
:100A3000A54B04930023A54A1288013A032A00F229
:100A40008682DFE812F00101DC0011007101A04B89
:100A5000934F1B783988934A934E52F821500033B4
:100A600018BF01233370C2E72046059310F0AEFC97
:100A7000984910F0FFFC059B0446184610F0A6FCB0
:100A8000954910F0F7FC0146204610F0EBFB10F002
:100A9000B7FE0446CAF80040D8F8000010F096FCF3
:100AA0008C4910F0E7FC8246009810F08FFC8A49D0
:100AB00010F0E0FC0146504610F0D4FB10F0A0FE10
:100AC000C8F80000854A864BB2F800E01988854BCB
:100AD000DBF800201B88DFF844C2CEEB040804EBEF
:100AE0000E0AC1EB000E08440499039CC1F800A053
:100AF0000199C4F80080C1F800E002999A420860A8
:100B0000BCF8001080F25281C3EB010C62486545CD
:100B10004FF0000E006880F256816C1C83420CF18D
:100B2000010C0EFB04FE9EFBFCFE00F3928381424F
:100B3000A8BF0146C91A04FB01F191FBFCF19A42DE
:100B400000F317818342C0F21481DFF8D4A1DAF8F0
:100B5000000010F03BFC644910F08CFC634910F07D
:100B600081FB10F04DFEA0F5FF531C3B082B98BFF6
:100B70004FF40050D9F80040DFF8A881044443F650
:100B8000FF77BC42A8BF3C4624EAE4742046CAF87A
:100B9000004010F01BFC8146307805FB00F010F09F
:100BA00015FC4FF07A5110F065FC0146484610F0F4
:100BB00057FB10F025FE4E4BB842A8BF38461B78B5
:100BC00020EAE070C8F80000002B00F0E380B4F5E4
:100BD000005F00F0DF8006F0E5F8464BD8F8000033
:100BE00001221A70444C2368834205D080B209F078
:100BF0000BF8D8F8003023600BB0BDE8F08F20462A
:100C0000059310F0E3FB3D4910F034FC059B0446CE
:100C1000184610F0DBFB3A4910F02CFC0146204648
:100C200010F020FB10F0ECFD0446CAF80040D8F8A4
:100C3000000010F0CBFB314910F01CFC82460098FC
:100C400010F0C4FB2E4933E72046059310F0BEFB9D
:100C50002C4910F00FFC059B0446184610F0B6FB1B
:100C6000294910F007FC0146204610F0FBFA10F06D
:100C7000C7FD0446CAF80040D8F8000010F0A6FBF3
:100C8000204910F0F7FB8246009810F09FFB1E49A8
:100C90000EE700BF869FFF1F3C9DFF1F169DFF1F95
:100CA0007A9DFF1F9089FF1F6A9FFF1F2089FF1FEA
:100CB0005A9FFF1F1C340100E89FFF1FB49DFF1FB8
:100CC000EC9EFF1F789FFF1FF09EFF1F6489FF1F90
:100CD0002E9DFF1FCDCC4C3FCDCC4C3E208AFF1F1C
:100CE0005C89FF1F509FFF1F9A99193FCDCC4C453F
:100CF0009EA0FF1FE09DFF1F2489FF1F6666663FC1
:100D0000CDCCCC3D3333733FCDCC4C3D749DFF1FD8
:100D1000089DFF1F909FFF1F749FFF1F589DFF1F7F
:100D2000C889FF1F6089FF1F2046059310F04EFB06
:100D3000C54910F09FFB059B0446184610F046FB82
:100D4000C24910F097FB0146204610F08BFA10F0D4
:100D500057FD0446CAF80040D8F8000010F036FBF2
:100D6000B94910F087FB8246009810F02FFBB74975
:100D70009EE63B88002B3FF4E8AEC1EB0E03002B50
:100D8000B8BF5B42092B00F3E5804FF40050DFF859
:100D900008A3EFE6AE4C2378002B3FF423AF05F019
:100DA000FDFF0023D8F8000023701BE7C3EB010C04
:100DB000A8488A42D4BFC3EB020EC3EB010E6545BF
:100DC0000068FFF6AAAE83420EFB05FEC8BF0024F2
:100DD0009EFBFCFE40F3348294FBFCF1AFE69E4B9D
:100DE0001B78002B00F0D5809C4F9D4B39889D4A85
:100DF00053F821009C4E012100231170337010F034
:100E0000E5FA4FF07C5110F035FB10F0F9FC054687
:100E1000EDE5964B964A1B8896491278013B31F9CD
:100E20001340002A40F0B08011200DF0ABFF00907D
:100E3000914B0193D3F80090009B994540F3AC800F
:100E40008E4BDFF858821B888D4A012BD8F8003072
:100E5000B2F800A08B4A02922846A3EB040400F0EB
:100E6000CE8010F0B3FA029A52F82A1010F002FB6A
:100E70000146002010F0F4F910F0C2FC009BC9EB11
:100E800004029C42B8BF1C469042C9EB040480F2A5
:100E9000CA8000FB0444013294FBF2F47A4BDFF881
:100EA00000920293D9F80030234403EBD3735B1014
:100EB000C9F80030754B1B88012B7FF4B3AD744B20
:100EC00003931C460F200DF05DFF226804929042B0
:100ED000034680F2E980694A1288012A00F02E81D7
:100EE000674A07901288674C0692284610F06EFAFF
:100EF000069ADFF8B0A154F82210DAF8004010F09A
:100F0000B9FA0146002010F0ABF9059BE21A0592F0
:100F100010F076FC059A079B04999A42C1EB020EE9
:100F2000B8BF1A46704580F23381521A00FB022284
:100F30000EF1010192FBF1F2D9F80010554804902E
:100F40000A4402EBD2725210C9F8002073E5D8F8B7
:100F50000000B7E50EF500500130401A10F036FAE7
:100F60003A49DFF834A110F085FA0446DAF80000B7
:100F700010F02CFA344910F07DFA0146204610F0AA
:100F800071F910F03DFCF5E515200CF0DFFD009047
:100F90004EE7344A137022E53B4B0293D3F800909E
:100FA000009B994544DA354BDFF8F0801B88344AC2
:100FB000012BD8F80030B2F800A0324A039228463C
:100FC0001C4400F0EC8010F001FA039A52F82A1049
:100FD00010F050FA10F014FC009B9C42C9EB040284
:100FE000A8BF1C46C9EB04049042BABF00FB0444EE
:100FF0000132444394FBF2F4DFF8A49052E710F07E
:10100000E5F9029A52F82A1010F034FA10F0F8FBC1
:10101000009BC9EB04029C42B8BF1C468242C9EB4C
:1010200004043FF736AF00FB04F494FBF2F435E719
:10103000DFF86C90DFF86480D9F8003003EBD373ED
:101040005B10C9F80030E8E49A99193FCDCCCC3E4A
:10105000E09DFF1F3C9DFF1F2E9DFF1F7A9DFF1FE0
:101060009089FF1F169DFF1F6A9FFF1F6C8AFF1F3D
:101070000C9FFF1F38300100E89FFF1FC69DFF1F18
:10108000609DFF1F34340100B49DFF1FEC9EFF1FC5
:10109000789FFF1FF09EFF1FC889FF1F089DFF1F3D
:1010A000909FFF1F749FFF1F6B4A04921268069265
:1010B000904237DD694A1288012A00F08E80684A22
:1010C00009901188674A08912846079210F07EF926
:1010D000079A0899DFF890A152F82110DAF8004039
:1010E00010F0C8F9059B2344059310F089FB05997E
:1010F000099B069A9942C2EB010EA8BF194670459A
:1011000080F29080891A00FB01110EF1010291FB1F
:10111000F2F2D9F800100A4402EBD2725210C9F868
:10112000002088E4D9F80020DFF83CA102EBD2725D
:101130005210DAF80040C9F800207CE4484A0890D0
:101140001188484A07912846069210F03FF9069AFE
:101150000799DFF814A152F82110DAF8004010F0D6
:1011600089F9059BE11A059110F04AFB0599089B46
:10117000049A9942C2EB010EB8BF1946704558DA7D
:10118000891A00FB01110EF1010291FBF2F2D3E684
:101190000499521A00FB02F292FBFEF2CCE610F028
:1011A00015F9039A52F82A1010F064F9014600204C
:1011B00010F056F810F024FB009A9442C9EB040397
:1011C000A8BF1446C9EB04049842BABF00FB04440C
:1011D0000133444394FBF3F40EE72149214A08907C
:1011E00028460C88079210F0F1F8079ADFF878A0EB
:1011F00052F82410DAF8004010F03CF901460020C3
:1012000010F02EF8059B2344059310F0F9FA059988
:10121000089B069A9942C2EB010EA8BF1946704579
:10122000FFF670AF069A891A00FB01F191FBFEF2FE
:101230006FE7049A891A00FB01F191FBFEF27BE64D
:101240008842D4BFC3EB0004C3EB010405FB04F4E4
:10125000C2E519466EE400BFF09EFF1FC69DFF1F4A
:10126000609DFF1F34340100749FFF1F08B5244B9D
:101270001B88FBB1234B1B78FBB1234B1B78E3B1DD
:10128000224B1B78CBB1224B1B78B3B1214B2248A8
:101290001A78C2B9214A2249008812880968024492
:1012A000B1EB620F09DD01221A706420BDE808402D
:1012B00005F08CBD174A117801B908BD1370BDE85F
:1012C000084008F045BD154A16490088128809688B
:1012D0000244B1EB620FF0DD00221A7008F038FD15
:1012E000642005F073FD642005F070FD642005F0B6
:1012F0006DFD4FF41670BDE808400DF079B900BFE0
:10130000FE9EFF1FB69FFF1FB79FFF1FB89FFF1FC7
:10131000B99FFF1F449DFF1F589DFF1F509FFF1F38
:10132000749DFF1F3C9DFF1F38B5114C232025786D
:101330000CF00CFC0F4A42F82500131F02F1C40008
:10134000002253F8041F83420A44FAD123780A4941
:1013500007480A4C0133DBB2322B81FB025108BF34
:101360000023D217C2EB21120370226038BD00BFE8
:10137000249DFF1F009EFF1F1F85EB514C9FFF1FE9
:101380002DE9F04FB74DB84E2868B84C83B010F037
:101390001DF8B74910F06EF8074610200DF0F2FC6A
:1013A00010F014F8B34910F065F839460FF05AFF01
:1013B00010F026FA31882860884223887EDA1F469A
:1013C00000225B1ADFF8D482DFF8D4E27F2BCABF99
:1013D000D201C2EBC212013392FBF3F3B8F8002042
:1013E000CEF80030192A00F0DF801A2A00F02B8195
:1013F0001E2A00F05B814FF00108C1469E4B1B88FE
:10140000002B66D09D4A1288032A00F20981884287
:10141000C0F25F81B842D4BFC1EB0000C1EB07004E
:10142000791A8B42B4BF03FB00005843944F954B8D
:10143000B8BF013190FBF1F01860388800284FD018
:101440003188D5F800E0884ADFF818A2714500F32A
:101450008280DFF83CC29CF80030002B4CD14FF06A
:10146000010B04288CF800B046D1B8F1000F40F011
:10147000CB81854B1888F0B1B9F1000F1BD02B68D8
:10148000318822888B4280F29C810023541A7E2C62
:101490007E4DD5BFC3EB8313C3EBC3135B00013495
:1014A00093FBF4F42B680134A34203D0C0B2E1B241
:1014B00008F0DAFB2C6003B0BDE8F08F9842D4BF8F
:1014C000C1EB0002C1EB03021F467AE799464FF0D9
:1014D00001081E2A00F0D281694F38880028AFD158
:1014E000694B1B88002BABD1694A11780029E2D0E7
:1014F000137003B0BDE8F08F012800F012810228BC
:1015000000F003810328B4D1624B1B88092BB0D0B3
:10151000B8F1000FADD02B6837882288BB4280F22B
:1015200095810023D71B7E2FDFF86CB1D5BFC3EBAD
:101530008313C3EBC3135B00013793FBF7F7DBF8AF
:1015400000300137BB4203D0F9B24A2008F08CFBCF
:10155000CBF800708DE74E4B1A78002AABD00024F0
:1015600001281C7000F0C280022840F03181B8F1DF
:10157000000F00F0C280484D2B68002B00F0BD80AA
:101580000420214608F070FB3F4B2C60188800288F
:1015900091D0B9F1000F8ED0C0B2002108F064FBE9
:1015A0003A4B00221A6086E7DFF8F8A0DFF8F890DF
:1015B0009AF80030BBB1DFF8D0E0BEF800E0BEF131
:1015C000000F10D099F800C09C4500F099805FFA98
:1015D0008EF07F2108F048FB9AF80030B8F8002020
:1015E00089F800300FE099F800E09E4500F088800F
:1015F000254B0021187808F037FB9AF80030B8F82E
:10160000002089F800301C4B1B88002B3FF45EAF94
:101610001E2A40F02B814FF001084FF0000951E0E5
:10162000884258DBB842A1EB0701A8BF38468B427D
:10163000A0EB070055DA03FB00004B1C90FBF3F313
:10164000104A136048E7DFF85CA09AF80030002BDE
:101650000BBF4FF001084FF000084FF000094FF0AA
:101660000109CBE6689DFF1F049FFF1F009FFF1F1E
:101670009A99193FCDCCCC3EC49FFF1F7C9FFF1F82
:10168000709DFF1FF89DFF1F989FFF1F4C9DFF1F20
:101690008C9FFF1F3C9FFF1FFC9DFF1F869FFF1F0E
:1016A0006C9FFF1F2E9DFF1F2A9DFF1FDFF8E8A1E3
:1016B000744B9AF800801B88B8FA88F84FEA5818DB
:1016C0004FF000099AF8002042B328683188278833
:1016D00098E60020A4E60846C91B8B42A0EB070051
:1016E000A9DB03FB00F393FBF1F3A9E7B8F1000FCB
:1016F00003D0654D2B68002B7FD1644B188846E7DB
:101700004FF001084FF0000978E6B8F1000F3FF400
:10171000B0AEDFF874B1DBF8003030E05C4B1A603B
:10172000DAE6B8F1000F3FF4A4AEB4F800A0F24539
:10173000D4BFC1EB0A03C1EB0E03C1EB0A0ABAF135
:101740007E0FDFF844B1D5BFC3EB8313C3EBC313E4
:101750005B000AF1010A93FBFAFADBF800300AF1A8
:10176000010A534504D05FFA8AF1012008F07CFA9F
:101770003888CBF800A002287FF4C4AE53462A680C
:10178000B6F800A02188524559DA0022CAEB010AB6
:10179000BAF17E0FD3BFC2EB8212C2EBC2120AF1C2
:1017A000010A520092FBFAFA0AF1010A9A4504D0A2
:1017B0005FFA8AF1042008F057FA3888CBF800A0C5
:1017C000A0E69342D4BFC1EB0303C1EB02035DE685
:1017D000032828D12F4B1B88092B8ED0B8F1000F7E
:1017E0008BD0294D2B68002B87D04A20214608F04A
:1017F0003BFA264B2C601888C9E6214608F034FADB
:10180000224B2C601888C2E640207F218DE80C0016
:1018100008F02AFA388858459DE80C001DD00228A7
:101820007FF470AE75E704287FF467AFB8F1000F5E
:101830003FF463AF2146402008F016FA5DE78A4284
:10184000D4BFCAEB0202CAEB01029FE79342D4BFA6
:10185000C7EB0303C7EB020364E6DAF800E0118884
:10186000B4F800A08E45FFF668AF60E728683188BD
:1018700027884FF001084FF00009C3E50023DFF887
:1018800018A01FE7C49FFF1FFC9DFF1F989FFF1F0D
:10189000F89DFF1F3C9FFF1F2E9DFF1F08B5114B9A
:1018A0001B88022B09D0052B07D0032B15D0042B46
:1018B0000BD00D4B01221A7008BD7F21412008F08A
:1018C000D3F9094B01221A7008BD7F21092008F0C5
:1018D000CBF9054B01221A7008BD4021092008F000
:1018E000C3F9E6E7F69DFF1F969DFF1F38B5074B2E
:1018F000074D1B88052B044606D02B68834203D076
:10190000C1B2052008F0B0F92C6038BDF69DFF1F6C
:10191000A09FFF1F38B5124D124C2B88052B12D0FB
:1019200022684AB9022B0ED0033B012B13D90E4A71
:1019300000231370236038BD0021052008F094F9BE
:101940002B88022B04D10021412008F08DF9EEE70D
:10195000052BE9D1F7E70021092008F085F9E6E732
:10196000F69DFF1FA09FFF1F969DFF1F464B1B88E4
:101970001D2B70B541D0454D0024454B1B88022BD3
:1019800016D0444B1B88022B54D02888424B002C85
:101990001B780ADB8442A8BF044634B1002B3AD03E
:1019A0002046BDE87040FFF7A1BF002B2FD170BDCE
:1019B0003A4B1B78002B37D015200CF0C7F8384B6A
:1019C0001860384A1288002ADBD0374A1868118814
:1019D0008142D6DC354B2A881B888342A3EB010663
:1019E000A8BF03465B1AB242BABF02FB03330136FB
:1019F000534393FBF6F31C44C3E72A4B1C888CB17A
:101A00002B4B224D1C78002CB7D02C88B5E7BDE8B5
:101A10007040FFF77FBFFFF741FF2046BDE87040F1
:101A2000FFF764BF194DA8E711200DF0ABF91C4B6F
:101A30001860C6E70F200DF0A5F91A4B1D4A1B8848
:101A40001060002BA1D01C4AC0F53B6311880833FD
:101A50008B429ADB194A288812889342A2EB01052F
:101A6000A8BF1346A842A3EB010306DA00FB033329
:101A7000013593FBF5F31C4488E700FB03F292FB6E
:101A8000F5F31C4482E700BF869FFF1F8E9FFF1F58
:101A90005A9FFF1FEC9EFF1F969DFF1F0C9FFF1F6D
:101AA000189DFF1FF69DFF1F929DFF1F849FFF1F24
:101AB0002E9DFF1F309DFF1FF49DFF1F709FFF1F76
:101AC000F8B510200DF05EF9C830B0F5FA7FC0F21D
:101AD0009680B0F57A6F0146A8BF4FF47A6101F5A0
:101AE0001673B3F57A6FA8BF4FF47A639BB289B2CD
:101AF000914A924C11802220238008F00FFA21880D
:101B00008F4D904C242008F009FA0E200CF01EF89E
:101B100040F6FF71C8308842A8BF084620EAE0704E
:101B200000F2DC5283B28A42A8BF0A46022019465C
:101B300022802B8008F0F2F92188042008F0EEF9C9
:101B400001200DF01FF9044600200DF01BF9A04202
:101B5000B8BF204600F1C801B1F5FA7FC0F2D180CC
:101B6000B1F57A6FA8BF4FF47A6101F54873B3F508
:101B70007A6FA8BF4FF47A639BB289B2724A734CF2
:101B800011800A20238008F0C9F921880C2008F070
:101B9000C5F90F200DF0F6F8C0F53F610431B1F53D
:101BA000AF6FC0F2AB80B1F5FA6FA8BF4FF4FA6126
:101BB00089B2674BC0F54360B0F5AF6F1980C0F2D2
:101BC0009A80B0F5FA6FA8BF4FF4FA6083B2614C07
:101BD000A420238008F0A2F92188A62008F09EF90D
:101BE00015200BF0B3FF00F59671B1F52F7F0BDBDD
:101BF00041F25C23994240F38980194608E040F2A3
:101C00004C434FF4FA7173E740F214534FF42F71C1
:101C1000514A1180514C524D2380062008F07EF924
:101C20002188504E082008F079F900274FF4AF744E
:101C3000F9B24D4809F0C8FF55F8043BC3F5967357
:101C400000FB03F086FB0023C017C0EB6310844247
:101C500007F10107A8BF0446062FE9D1434F414EC3
:101C60000025E9B2424809F0AFFF57F8043BC3F53D
:101C7000967300FB03F086FB0023C017C0EB6310D4
:101C8000844205F10105A8BF04460C2DE9D1394F66
:101C9000344E0025E9B2384809F096FF57F8043B66
:101CA000304AC3F5967300FB03F086FB0013C017A0
:101CB000C0EB6310844205F10105A8BF04460C2D5A
:101CC000E8D1A4F11401312931DD40F23A73A4F5D1
:101CD000B97403FB04F482FB0432E417A4EB621230
:101CE00089B232322548264B01801A602A20BDE88D
:101CF000F84008F013B94FF4AF6368E74FF4AF61F1
:101D000057E740F214534FF4FA7137E7124A00F5DF
:101D1000617089B2B0F52F7F1180B8BF4FF42F7377
:101D2000FFF678AF8342A8BF03469BB272E740F24A
:101D30006C723221D6E700BF049FFF1F009FFF1F78
:101D4000F09DFF1FBA9FFF1F509FFF1F589DFF1F51
:101D5000F49DFF1F709FFF1F929DFF1F849FFF1F19
:101D6000548AFF1FB5814E1B489DFF1F248AFF1F09
:101D7000789DFF1F2C89FF1FE89DFF1FB49FFF1F49
:101D8000108AFF1F2DE9F84F0C200BF0ABFE0C2042
:101D90000CF060FBCB49DFF8B4A314200CF06AFB15
:101DA000C949CA4809F0A2FB022103200CF0F8FB44
:101DB000022104200CF0F4FB022105200CF0F0FBC2
:101DC000022106200CF0ECFB01210A200CF0E8FBBC
:101DD000012109200CF0E4FB01210D200CF0E0FBB7
:101DE000012128200CF0DCFB012114200CF0D8FB91
:101DF000012116200CF0D4FB012117200CF0D0FBA0
:101E0000012121200CF0CCFB02211C200CF0C8FB8E
:101E100001211B200CF0C4FB00211B200CF0ACFBAB
:101E20001C200CF0AFFBB0FA80F35B091A208AF893
:101E300000300CF04BFD1F2000210CF00DFD0420A4
:101E40000CF0A0FB002800F0318105200CF09AFB7B
:101E5000002800F0A68100239D4C062023700CF082
:101E600091FBB0FA80F35B094FF0000B994A1370B5
:101E700006F0DCFB2478002C40F01481584608F072
:101E800077F8954B954A1B8815889549954840F2F7
:101E90003A72A3F5AF7302FB03F381FB0312DB1766
:101EA000A3EB6213323303608F4B01210D201D70B1
:101EB0000CF062FB64200CF09BFB4FF416710A20BF
:101EC0000CF0CAF95D21894809F0BAFE002800F03B
:101ED000A58164200CF08CFB21460A200CF0BCF993
:101EE0004FF4967109200CF0B7F95C21804809F095
:101EF000A7FE002800F07F8164200CF079FB2146CA
:101F000009200CF0A9F94FF4967116200CF0A4F9F1
:101F10005B21784809F094FE002800F04981642094
:101F20000CF066FB214616200CF096F94FF49671E2
:101F300017200CF091F964200CF05AFB2146172071
:101F40000CF08AF964200CF053FB21460D200CF0B4
:101F500013FB694A69481268DFF8F491684F694DCC
:101F6000694EDFF8F08100230121FEF79DFA01237D
:101F70003C602C60346089F8003004240F200CF0A1
:101F800001FF336803440E2033600BF0DFFD3B6834
:101F900099F8002018443860002A7CD015200BF0F6
:101FA000D5FD2B681844286004F0010080F0010082
:101FB00004F0FCFEB8F80030002B14BF4B20DC20EE
:101FC0000CF016FB013CD9D1336839684C4A2868BB
:101FD0004E4F002BB8BF03330029B8BF033189101F
:101FE00011604B494B4A098814889B1000283360C4
:101FF000B8BF0330484E8210581A19442A60316025
:102000003860464D46484749161B22442E60026000
:102010000B60BBF1000F40F0AC80B8F80030002B33
:1020200000F09A80404B012404201C600CF0AAFAB6
:1020300018B93E4B2C4A1C7010703D4B1B881C2B52
:1020400000F09F803B4C04F1C80523200BF07EFD7F
:1020500044F8040F01200CF0CBFAA542F5D19AF810
:10206000003023B1344B1B78002B40F095800021C9
:1020700021200CF081FA314A314B1078187007F0AA
:102080007FFD04F08BFE45F6BF522E492E48BDE879
:10209000F84F0BF013BB11200CF074FE2B681844A2
:1020A000286081E7BDE8F84F09F030B906200CF050
:1020B00069FA00287FF4C9AE054C034620704FF042
:1020C000010BD3E6001B374640420F00F491FF1F7F
:1020D0004A9DFF1FF49EFF1FB49FFF1F889FFF1F95
:1020E000B5814E1B108AFF1FB09DFF1F489DFF1F2B
:1020F000E89DFF1F789DFF1F2889FF1F189FFF1F66
:102100001C9DFF1F089DFF1F749FFF1F789FFF1FCF
:10211000208AFF1F5C89FF1FF09EFF1FE89FFF1FA3
:10212000B49DFF1FCC9FFF1F809FFF1F349DFF1F8B
:10213000869FFF1FFC9DFF1F069FFF1F089FFF1F1D
:10214000EB9EFF1FA5050000A89FFF1FEE9EFF1F2F
:102150000C9FFF1F469FFF1F4FF4FA7004F036FEDE
:1021600004F020FE06F0ACFD4FF4AF600CF040FA36
:1021700058E7FFF7A5FCB8F80030002B7FF452AF0A
:10218000EAE7294B188800283FF45CAF274BC0B220
:10219000197807F069FD55E7012121200CF0ECF9D1
:1021A00069E703200CF0EEF9B0FA80F35B0953E61F
:1021B00003200CF0E7F90028FAD104200CF0E2F932
:1021C0000028F5D105200CF0DDF90028F0D106201B
:1021D0000CF0D8F90028EBD10CF0F4FE04200CF040
:1021E000D1F940B905200CF0CDF920B906200CF04A
:1021F000C9F90028F0D003200CF0C4F90028FAD166
:10220000ECE704200CF0BEF940B905200CF0BAF957
:1022100020B906200CF0B6F90028DDD003200CF020
:10222000B1F90028FAD1ECE7B89DFF1F649DFF1FAC
:102230002DE9F04FAD4C2678012E95B000F0558277
:10224000C0F00B82022E00F0D880A949A94A91F86B
:1022500000801178A84ADFF83CE3A84DA84FA948B0
:10226000A94B0292A94A0092A94A9EF800B0019295
:102270002D78A84A3F7890F800E01B78DFF818A383
:10228000DFF818C3DFF818930392012E84BF0022F1
:102290002270A14AA1481370A14A80F800B01570BD
:1022A000A048A14A077082F80080A048A04A0370A5
:1022B0009CBF013626701170BEF1000F40F0748192
:1022C0009C4A10880D2800F0B9819B4C002020709A
:1022D000024604462DB197480088002840F0BA8194
:1022E0000546964806882544002E40F067819448AC
:1022F000944C019E0078367824780130A0EB46009B
:10230000002C40F05682039C94F800E0CEEB0004D1
:10231000BEF1000F40F076820026DFF874E20298EA
:102320009EF800E00078A41BA4EB4E043C44CBEBE9
:10233000040410B1B7FA87F040099CF80060271830
:10234000BC1B1EB11EF1000618BF0126009F99F8A4
:10235000000097F800909AF800C07B4FC6EB040E7F
:10236000C0EB0E00A0EB49008044C3EB0803A3EBD5
:1023700041010C2313FB0C113960744B744F754CE5
:1023800075481B880088D7F800C0744E2788744CA5
:102390003688D4F800E0033BC0EBC00403EB4303F2
:1023A000C7EBC70001EB830364446E4F33447044B2
:1023B0006D4E57F8244056F820000C3B1D44254430
:1023C00005440AB1694B1960694A13689D4200F0DF
:1023D0003181684B684819680791079901601B684B
:1023E00008936648089B008815605B1A834284BF87
:1023F000634B1D6015B0BDE8F08FDFF8A881614E1A
:1024000008AF0025E9B2604809F0DEFB58F8043B4C
:10241000C3F5967300FB03F086FB00230135C0175C
:10242000C0EB63100C2D47F8040BEBD1574B384D24
:102430000195384DB3F800C00395109D09980F9988
:10244000404EDFF8C0A0DFF8B490DFF8BC806545EF
:1024500011AA8CCAAE46ACBF4FF0000E4FF0010E71
:102460008445D4BF0020012030708C4528480B9D46
:102470001F4E8AF800E0D4BF00210121017094456D
:102480002449DFF814A1D4BF002201220A709C4520
:102490003F4AD4BF00230123BC45AB46D4BF00272D
:1024A00001271370AC45164B0C9D1F70D4BF4FF025
:1024B000000B4FF0010B374B0F4A0292AC45DFF88F
:1024C00034C0124A83F800B0D4BF0025012589F832
:1024D000005098F800309CF8001096F80080DFF863
:1024E000BCC02678DFF8B8900092CEE6EA9EFF1FC7
:1024F000389FFF1F3A9FFF1F499DFF1F3F9FFF1FF0
:10250000949DFF1FF49FFF1F399FFF1F8A9FFF1F8E
:102510009D9FFF1F9E9FFF1FEE9FFF1FEF9FFF1FAF
:10252000F09FFF1FF19FFF1FF29FFF1FF39FFF1FF1
:102530008B9FFF1FF69FFF1F2E9DFF1F149DFF1FE8
:10254000228AFF1FD89FFF1F409FFF1F5E9FFF1F14
:10255000F89DFF1F989DFF1F7C9FFF1F269DFF1F5B
:10256000C09FFF1FF8310100802B0100D09FFF1F8B
:102570008C9DFF1FDCA0FF1F7C9DFF1F969FFF1FF0
:10258000DC9FFF1FB5814E1BE89DFF1FB49FFF1FFF
:102590009F9FFF1F959DFF1FF59EFF1FED9FFF1F34
:1025A000B29FFF1F2C89FF1FAF4AB0481488012239
:1025B000182C027040F2058100248BE6012E00F0F9
:1025C0008F81022E00F0EE81032EA94B00F01F81B7
:1025D0001E78009B9CF800E01C78019B99F800C0D5
:1025E0001878029B93F80080039B1F78A6EB4E039C
:1025F000A4EB8404CCEB030CC0EB80760CEB04035F
:10260000C0EB8600034403EB480303EB810327B1CF
:1026100098490978002940F0608201269AF8001054
:102620009548C1F1060101EB4101334403EB8101FF
:102630000160A2E69149924B0968D0E6002D3FF473
:1026400044AE894A894E14880122182C327040F217
:10265000B8807446A0F10D0543E6DFF87092894F0B
:102660000DF120080025E9B2874809F0ADFA59F8C4
:10267000043BC3F5967300FB03F087FB0023013591
:10268000C017C0EB6310062D48F8040BEBD17F4B4D
:10269000DFF83CA219880D9B00228B428AF80020AB
:1026A00080F2A2807A4B8AF800507A497A4A7B48B5
:1026B00091F8008011787A4A1D7002920378794A65
:1026C000DFF810C2DFF810920092774A774E784D0B
:1026D000784892F800E0784A0192784A96F800B07B
:1026E0002D78077826780392CFE5DFF8F081654EE4
:1026F00008AF0025E9B2724809F066FA58F8043BC1
:10270000C3F5967300FB03F086FB00230135C01769
:10271000C0EB63100C2D47F8040BEBD15B4B0C9D09
:102720001F885F4B02935F4B00930B9B0A98099A9B
:10273000DFF8A0C1089EDFF8A0910F99BB429E462A
:10274000ACBF4FF0000E4FF0010EAF42D4BF0025DA
:1027500001258742109B8CF80050D4BF0020012037
:10276000504D89F800009742D4BF00220122B742A1
:10277000D4BF4FF000084FF001082A709F42474A2B
:102780004448474E80F80080D4BF002301231370D3
:10279000129A414886F800E08F42D4BF00210121FF
:1027A000974201701ADC00224648DFF824A102702B
:1027B0008BE7039C46B12678002E40F06081441ED2
:1027C000ABE50C3C012285E594F800E00138CEEB46
:1027D0000004BEF1000F7FF4A0AD9DE5119A974271
:1027E000D4BF00220122DFE70C9A374B9142CCBFC5
:1027F000012200221A7040F3458105258AF8005015
:10280000234B52E7002E3FF487AD012685E51C7867
:10281000009B029893F80080019B9CF800601B7855
:1028200090F800C099F800700398A4EB4604E71BE9
:1028300090F800E0C3EB8374A8EB88003844C3EB46
:102840008403034403EB4C0303EB8103BEF1000F4D
:1028500040F0488101269AF80010074833440C24C0
:1028600014FB0131016088E5869FFF1F2E9DFF1F2D
:10287000228AFF1F9F9FFF1F409FFF1F7C9DFF1FFE
:10288000DCA0FF1FB5814E1B489DFF1FB49FFF1F9B
:10289000029FFF1F389FFF1F3A9FFF1F399FFF1F97
:1028A000499DFF1F8A9FFF1FF49FFF1F959DFF1FDC
:1028B0003F9FFF1F949DFF1F9D9FFF1F9E9FFF1F18
:1028C000789DFF1F5E9DFF1FB99FFF1F548AFF1F4A
:1028D000F59EFF1FED9FFF1FB29FFF1F248AFF1F62
:1028E000A34CDFF89CE2207805909EF80040019808
:1028F0000494059C007801900134A4EB40040498F2
:10290000002840F0AF80039890F800E00498261A61
:10291000CEEB06000390BEF1000F40F09E8074469F
:102920000298944E00780290039836780496041B1F
:10293000A4EB460402983C44CBEB0404002800F0CE
:102940008780B7FA87F040099CF800602044871B15
:102950001EB10498061C18BF0126009C99F80000BF
:102960002478BE1B301AA0EB440080440198C3EBCE
:102970000803A3EB4103002867D1BEF1000F40F02C
:10298000BB807344002C5ED100290CBF00206FF087
:1029900009009AF80010784C03440C2010FB013118
:1029A0002160EAE4039E019C36780396009E247819
:1029B000019434786F4E714899F800E0009496F8CD
:1029C00000906F4C9DF80C6086709DF80460067056
:1029D00080F806E09DF8006080F803909CF800C045
:1029E0002478DFF8B491DDF804E080F808800771FE
:1029F00080F805C0C671417244704FF00008012094
:102A0000009500215D4C0D465FFA88FC4F467646E6
:102A100007E0022809D00A290BD014F8016F17F833
:102A2000010F864201F10101F3D101350A29EDB20E
:102A3000F3D1092D72D808F10108B8F1100F36D082
:102A400019F80A0FDDE70020A3E74FF0000E98E722
:102A5000029879E7CEEB040003900198041C18BF9C
:102A600001245DE7019800284ED0039890F800E01B
:102A7000BEF1000FEED1601E0390744650E7841B38
:102A800001264AE40B9A3F4B9142CCBF012200221F
:102A90001A703EDC0A9A3C4B9142CCBF01220022C4
:102AA0001A7052DD03258AF80050384BFDE5304896
:102AB00037490478C86B0299009D09780134204495
:102AC000CBEB0000084400219AF800402A4B401A42
:102AD0000C2111FB040119604FE41BF1000618BF23
:102AE00001269BE52349097800293FF4B3AE1BF189
:102AF000000618BF0126AEE6049800280CBF4FF070
:102B0000000E4FF0090E3CE7039890F800E03046C5
:102B1000FDE604258AF800501C4BC6E514481C4904
:102B2000047851F828000299009D09780134204466
:102B3000CBEB000066460844002BC4D0002EC2D167
:102B4000BBF1000FBFD00121BEE7099A114B9142A2
:102B5000CCBF012200221A7004DD02258AF8005041
:102B60000A4BA2E5089B994218DD01259AE500BFB2
:102B7000228AFF1F9F9FFF1F409FFF1FBC9DFF1FBB
:102B8000D89FFF1FB89FFF1FB79FFF1F029FFF1F08
:102B9000D089FF1FB69FFF1FC8300100154B1D785D
:102BA000012D25D9144A8AF800501288D2B1134A4F
:102BB0001288013A92B2062A14D8114A12788AB1C0
:102BC000104A1268012A7FF470AD0F4A0F4E106848
:102BD0000C2290FBF2F102FB110232800C4A03211D
:102BE000117062E5074A1268012A7FF45EADF5E7CD
:102BF00035465AE5029FFF1F689FFF1F0A9FFF1F70
:102C0000F29DFF1F809FFF1FDC9FFF1F449FFF1F40
:102C1000C489FF1F2DE9F04F3A4B1B788BB0002B76
:102C20006BD10E200AF092FF0EF0D0FB0146364821
:102C3000364E374DFDF77EFC3348FDF751FC0EF064
:102C4000DFFD80F30C003060FFF7F2FA2C68012CF6
:102C50007AD0022C00F0C582032C00F02B842D4E7C
:102C60002D4C33682D4A2E4E0993099B31681288EA
:102C70002360591A013A9142274F00F2AD82294E42
:102C800032689A1A092A00F29682274E32689A1AF6
:102C90000D2A00F28B82254E32689A1A252A1AD9FB
:102CA000234B1B88002B40F05B81224B1B78002BB1
:102CB00040F05681FEF738FB1F4B1B881B3B9BB235
:102CC000022B04D81D4B1B78002B40F04C8104F0E4
:102CD0008FF8236833601A4D2A689B1A502B00F234
:102CE0000D82184B1B88012B00F0258206F040FF57
:102CF00006F024FE0BB0BDE8F08F08F08FF90BB0A2
:102D0000BDE8F08F4A9DFF1F189FFF1F549FFF1FB4
:102D1000809FFF1FDCA0FF1F149FFF1FCC89FF1F98
:102D2000EC9DFF1FD49DFF1FA89DFF1FAC9DFF1FA3
:102D3000FE9EFF1F449DFF1F869FFF1F2E9DFF1FAE
:102D4000F89EFF1F589FFF1FDFF820939F4AB9F896
:102D500000001378834204D0C3B21846137006F003
:102D6000F9FEDFF804839A4AB8F8003011789942E6
:102D700004D0984F3978002940F05887964A336834
:102D80001288964E9A42C0F2F880954A1278002A2C
:102D900040F0F380DFF8D8A2BAF8003023B9914BA5
:102DA0001B88002B00F069858F4A904B11881B8887
:102DB0008F4A0B4412685B1093428E4A126880F26D
:102DC0000B8500219342B4BF01230B46049100936D
:102DD000ACBF4FF0010B8B4605910E200AF0B6FEFA
:102DE000854B864A1B68176803930133A7F252325A
:102DF000002B8446029240F32A87802BA8BF8023B1
:102E00007F4A804912780191002A00F0C080097839
:102E1000914200F0BC80B8F80010DFF84CE2994213
:102E200001F015816B49AEF80030774B4FF0010E81
:102E300081F800E01978DFF83CE2019B8EF8001081
:102E40001A70009B002B00F01781BAF80030002B9D
:102E500000F012816D4B1B685A1C002A40F3FB8660
:102E6000802A00F3F7866A4C6A496B4824880988EF
:102E700000682144B0EB610FC1F25A83A3F148020C
:102E80000F2A02D8473BA9F800300E200AF05EFE58
:102E90006FF454731F44874202DC604B00221A70A7
:102EA0005F4B1B88002B00F08E845E4B5E4A1B78C4
:102EB0001178994243D0002B41D05C490C78002C0A
:102EC00000F08D875A4991F800C0BCF1000F40F026
:102ED0008487584F0097584F58480297554F0078AD
:102EE00087F800C0544F4FF0010E87F800C081F8FA
:102EF00000E0002841F0FB8051490978002901F0E9
:102F00004F80504903910C460978002941F04580D3
:102F10004D48494F0078397001210297217070B1F6
:102F2000444843490090494803270770002008702F
:102F30000099029F0870039901243C700870137077
:102F4000434B1B88A3F11B02012A40F233861D2B41
:102F50007FF486AE3C4A3F4B12781A703E4C80E6B6
:102F6000FEF784F9A6E63D4B1B78002B3FF4AFAE8D
:102F70002B68012B7FF4ABAEABE63168384A069183
:102F800006983849106002220B602A6002E71E4949
:102F9000DFF8E0E0097800293FF44FAF9EF8000029
:102FA00081423FF44AAF03984B2841F3178018330E
:102FB000802BB8F80000A8BF802398423FF43DAFB3
:102FC0002948038003480123037036E7EB9EFF1F67
:102FD000B09DFF1F349DFF1FF09DFF1FDCA0FF1F52
:102FE000449DFF1FDA9DFF1F589DFF1F509FFF1F2D
:102FF000749DFF1F3C9DFF1FD09FFF1F1C9DFF1F47
:10300000C69FFF1F889DFF1FC79FFF1F409FFF1F79
:10301000049FFF1F009FFF1F689DFF1F509DFF1F04
:103020000A9FFF1F5E9DFF1F0C9DFF1FF19FFF1F4B
:10303000489FFF1F9C9FFF1FF29DFF1FF29FFF1FD6
:10304000EE9FFF1F0D9DFF1F2E9DFF1FC489FF1FB9
:10305000869FFF1F2A9DFF1F149FFF1F8B9FFF1F2F
:103060009C9DFF1F109FFF1F889FFF1F089FFF1F32
:10307000909DFF1F899DFF1F029B9C45BFF605AFDA
:10308000954B1B88002B3FF400AFBBF1000F7FF482
:10309000E1AE924B1B881BB1059B002B7FF4DAAE8F
:1030A000049B002B3FF4F1AE8D4B1A78002A7FF47D
:1030B000ECAEDFF8B09299F8004001221A70002CB3
:1030C00040F0A883874B1B78002B02F0CA80864B08
:1030D0001B78002B02F09E83844B1B78002B7FF41F
:1030E000D4AE834B1B78002B3FF4CFAEB8F8003042
:1030F00080490A3BA8F800300A70C6E605F0DEFAFF
:103100007D4B1B7873B97D4B1B785BB97C4B1B786F
:1031100043B97C4B1B782BB97B4B1B7813B903F05D
:103120003DFE01E003F046FE23682B60774B1B88D1
:10313000012B7FF4DBAD764B764A19681778764E13
:10314000A92303FB01F10029744BB8BF01F57F519E
:103150001868734BB8BF3F3189132A225439183885
:1031600002FB00111D786FF0140202FB071232609F
:103170006C49002D00F04E810B689A4200F3BE832B
:1031800080F24881684D2878002840F09D87674884
:103190000568D5F17F0548BF0335AD1001355B1BD0
:1031A0009A4200F337810B601A4634E1FEF7DEFBEA
:1031B000236833606FE5FDF7F9FBFEF7E1F85C4B40
:1031C0001B88032B00F067855A4B1B88032B00F0EC
:1031D0005E852368336058E5FDF734FB3B68336058
:1031E0004DE5554A34681288A24204DB464B1B78F1
:1031F000002B00F0B383514E514833680793514B75
:10320000079900681B88091A994200F2B180002BC7
:1032100000F0AE804C4B198800293FF421AD4B4B98
:103220004B481B680088A342B8BF23469A4241F32B
:103230007881484B1A60DFF8308188F80010374FEA
:10324000FDF700FB38687F2840F3C385424B7F3889
:1032500083FB0032C317C3EB620303EB4303A0EB12
:10326000830073303D4B01931B883860002B40F086
:10327000E786234B00931B78002B00F01C84384C0E
:103280002378002B00F01784DFF8E090DFF8C8A067
:103290004FF0000B0CE003F17300C0B298F800107F
:1032A00006F012FD23780BF1010B5B4540F303841C
:1032B0003B6859F8040F1844A0F17F038AFB0321EF
:1032C000DA17C2EB610202EB42027F28A3EB820312
:1032D000E1DCFDF7D7F9E0E7DA9DFF1F0E9FFF1F46
:1032E000509DFF1FEE9FFF1FEF9FFF1FF09FFF1FCF
:1032F000F19FFF1F349DFF1FF29DFF1F489FFF1F7F
:103300009C9FFF1F0D9DFF1F449DFF1F589FFF1F88
:10331000C889FF1F6A9FFF1FCC9DFF1FDC9FFF1FF7
:10332000969DFF1FDC9DFF1FA49FFF1FA09FFF1FF7
:103330005A9FFF1FEC9EFF1FF09DFF1FDCA0FF1F89
:103340009C9DFF1FD89DFF1F2C9DFF1F109FFF1FDF
:10335000BA9FFF1F109DFF1FABAAAA2A6E9DFF1FD9
:103360008C89FF1FF59EFF1FC89DFF1F6489FF1FEB
:103370007E4B7F491B6808887E49A342B8BF23461D
:103380009A4200F3D2827C4C09888342A8BF03464C
:10339000236000297FF44FAF9A42C8BF0B4640F329
:1033A000CB82801AB0F5804FAABF9B03C3EB833357
:1033B000013093FBF0F0FDF72BFAC0F3C6100EF0CE
:1033C00005F86E4B044618880EF000F86C49074665
:1033D00020460EF04FF8014638460EF04BF82146D5
:1033E0000DF040FF4FF07E5104460EF0E1F9002849
:1033F00041F07B80634920460EF0F8F9002840F048
:10340000708620460EF022FAC0B2DFF8BC8188F840
:10341000000014E70A605C4B188858B35B4B2568C2
:1034200053F82040B5FBF4F3772C04FB135300F35F
:103430002882C3EBC30303EB031393FBF4F3544859
:10344000544C50F823002468534BA0F2FF7004FB47
:1034500000F000F57D3000F5607000EB4004C0EB3B
:10346000C40083FB00430344C017C0EBA3400B38E8
:1034700002440A6049494A4B0888198800F27C7066
:103480004300B3F57C6FA1F164014FEA4100B5BF81
:103490004449454903FB02225A4381FB023111444E
:1034A000D317C3EBE123C11881F30C0128200AF0E4
:1034B000D3FE1BE43D4BD6F800801988414540F30C
:1034C00087803B4B1B78002B40F08280DFF8FC901C
:1034D00099F800007F2840F3F385A3F155337F3836
:1034E00003F1004383FB0032C317C3EB620303EB1A
:1034F0004303A0EB830073302E4B01931B88C0B2B3
:1035000089F80000002B40F0EC872B4B00931B78D0
:10351000002B00F09184294C2378002B00F08C8440
:10352000274FDFF8A0804FF0000A0AE003F1730094
:10353000C0B206F0EDFB23780AF1010A534540F3CF
:103540007B8457F8043F99F800001844A0F17F03EA
:1035500088FB0321DA17C2EB610202EB42027F28EB
:10356000A3EB8203E2DCFDF78DF8E1E7109FFF1F7C
:10357000BA9FFF1F2C9DFF1F109DFF1FC89FFF1F9D
:10358000CDCCCC3D0000FE42289DFF1FA4300100A1
:103590007C2901006C9FFF1F4D261281E09FFF1FB9
:1035A000A09DFF1F81DFFF8183200882F09DFF1F08
:1035B000449DFF1F6E9DFF1F9C9FFF1F8C89FF1F57
:1035C0006489FF1FABAAAA2AC89DFF1F3E9FFF1F49
:1035D000AF4F38687F2840F3B681AE4B7F3883FB0E
:1035E0000032C317C3EB620303EB4303A0EB83007A
:1035F0007330DFF8F89299F80040844200F00082BE
:10360000A54B1B88002B43D1A44AA548126800880B
:10361000914205DC8242D4BFC1EB0203C1EB00033F
:10362000411AB1F5804FA6BF9B030131C3EB833331
:1036300093FBF1F0FDF7ECF8C0F3C6100DF0C6FEF9
:10364000984B804618880DF0C1FE97498246404647
:103650000DF010FF014650460DF00CFF41460DF0F5
:1036600001FE4FF07E5180460EF0A2F8002840F097
:10367000A8868E4940460EF0B9F8002840F02E8505
:1036800040460EF0E3F8C0B2DFF8648288F800002C
:103690007F2C40F390837F487F3C80FB0430E3170E
:1036A000C3EB600000EB4000A4EB80007330804B64
:1036B00000931B78C0B289F80000002B40F0F28222
:1036C0007C4B03931B78002B40F0DD847A4B0293F4
:1036D0001B78002B40F01D87784B0193029B1B78D1
:1036E000FBB1774B1B88012B00F06285022B00F0A9
:1036F0007187032B01F00881042B01F01283052B45
:1037000001F0B283062B01F07885072B01F0DC85F0
:10371000082B01F0EE87092B02F037810A2B02F00B
:103720003883009B1B78002B00F04A84019B634C7C
:103730001988002900F0A08438687F2840F3AF8200
:10374000544B7F3883FB0032C317C3EB620303EB98
:103750004303A0EB830073303860002940F04F84AE
:10376000009B1B78002B00F05781564C2378002BD0
:1037700000F05281DFF87CA1DFF874814FF0000B7C
:103780000CE003F17300C0B298F8001006F09CFA48
:1037900023780BF1010B5B4540F33E813B685AF8FF
:1037A000040F3C4A1844A0F17F0382FB0321DA177F
:1037B000C2EB610202EB42027F28A3EB8203E0DC52
:1037C000FCF760FFDFE73C4C3F483949394A23703A
:1037D00003700B70FFF7B3BB93424FF0000B80F206
:1037E000B5800123CDF800B0CDF814B00493FFF7F5
:1037F000F4BA364B1B78002B7FF447AB039B344A5B
:10380000243B83F34703D9B25B20136006F02CFA04
:1038100099F80040032C30D1DFF8DC8098F80030B4
:10382000002B42F044812B4F3B78002B42F0328139
:10383000264C2378002B42F02081274B1B78002B4D
:1038400042F00E81254A1380254B1B78002B42F055
:103850003A81114B7F221A8098F800306BB93B787F
:103860005BB923784BB91F4A7F210720138006F0EC
:10387000FBF97F210B2006F0F7F91B4B1F68FFF7C0
:1038800004BBC3EB0313D800631C90FBF3F3D6E532
:10389000DC9FFF1FABAAAA2A2C9DFF1F109DFF1FB4
:1038A000BA9FFF1FC89FFF1FCDCCCC3D0000FE423A
:1038B0009C9FFF1F0D9DFF1FF29DFF1F6E9DFF1F11
:1038C0000A9FFF1F8C89FF1F489FFF1FF19FFF1F4B
:1038D000549DFF1FF09FFF1FEF9FFF1FE29DFF1FE3
:1038E000F29FFF1F3C9FFF1F1C9DFF1F3E9FFF1F5E
:1038F000C89DFF1F6489FF1FEE9FFF1FB648057814
:10390000002D40F04083B5480068D0F17F0048BFEB
:10391000033003EBA000431CB1480B609A42B8BFD0
:103920000260FFF678AD1A4675E5AE4B09881A605D
:1039300000297FF480AC13469842D4BFC2EB000349
:10394000C2EB03032DE5FCF79DFE52E60123CDF803
:1039500010B0CDF800B00593FFF73FBA01232B60FC
:10396000FFF77DB9029B1B78FBB19F4B1B88012B96
:1039700000F0A084022B00F0AB86032B01F03A800C
:10398000042B01F0F381052B01F0E482062B01F0FA
:103990003D84072B01F03785082B01F0E286092BC7
:1039A00001F0BC870A2B02F0B981019B1B88002B18
:1039B00000F02E83009B1B783BB9039B1B7823B937
:1039C000029B1B78002B01F08E80884B1B78002B0C
:1039D00000F0008186490B78082B00F2FB808548B7
:1039E0003A680068844C0133DBB25F1E101A44F859
:1039F00027000B70814BD6F80080198889F80020C9
:103A000088457F4E7FF72CA932687E4B0892089A32
:103A10007D4C1A60FFF725B9039B1B78002BA1D0C2
:103A20003B68A3F10C007F2840F3418377488B3B30
:103A300080FB0320DA17C2EB600000EB4000A3EB31
:103A4000800303F17300DFF8D881C0B298F800104A
:103A500006F03AF9009B1B78002B83D0644C237846
:103A6000002B3FF47FAFDFF8BCA14FF0000B0CE060
:103A700003F17300C0B298F8001006F025F923781E
:103A80000BF1010B5B457FF76DAF3B685AF8040FF4
:103A90005E4A1844A0F18B0382FB0321DA17C2EBC4
:103AA00061020C3802EB42027F28A3EB8203DFDCC9
:103AB000FCF7E8FDDEE74D4B1B78002B40F0B582AC
:103AC0003B68534A1278002A45D0A3F10C007F28A6
:103AD00040F3F3824D4A8B3B82FB0321DA17C2EBA2
:103AE000610202EB4202A3EB820303F17300C0B256
:103AF00098F8001006F0E8F8009B1B7853B33C4C94
:103B000023783BB3DFF81C91DFF800A14FF0000BE6
:103B10000BE003F17300C0B298F8001006F0D4F87F
:103B200023780BF1010B5B4514DD3B6859F8040F5A
:103B30001844A0F18B038AFB0321DA17C2EB610260
:103B40000C3802EB42027F28A3EB8203E1DCFCF796
:103B500099FDE0E73B682F4A1278FAB1224A1288B1
:103B6000012A00F03184022A00F03386032A00F093
:103B7000CC87042A01F02181052A01F05E82062A01
:103B800001F04C83072A01F0F184082A01F05586E0
:103B9000092A01F026870A2A02F08980019A1288F0
:103BA000002A00F03B821C4A174C137003232B6041
:103BB000FFF757B8DFF8708098F80030002B40F01E
:103BC000FE80164F3B78002B40F0C8840E4C3B70B3
:103BD000FFF747B83A680DE7A49FFF1FA09FFF1F9C
:103BE000DC9DFF1F109DFF1F0A9FFF1F489FFF1FA7
:103BF0008C89FF1F389DFF1F6889FF1FF09DFF1FE5
:103C0000DCA0FF1F88A0FF1F149FFF1FABAAAA2ADA
:103C10000D9DFF1FF29DFF1F3E9FFF1F2A9DFF1F4F
:103C2000C89DFF1F6489FF1F2E9DFF1FDBB2184632
:103C3000137006F0D7F8A54BA5491A46A54B1846B0
:103C400000230B703B7013700370FFF797B80123CC
:103C5000FFF7D6B88024A049A04BA14A09881B8849
:103C600012680B44B2EB630FBFF60FA99D4B1B7894
:103C7000002B40F0F281B8F800309B4AA3423FF499
:103C800004A99A4B148001221A70FFF7FEB8FCF7C2
:103C900061FDFFF79EBAFCF707FDFFF795BAFCF749
:103CA000F1FC59E5924B01931B8863BB894B03934D
:103CB000904B0293904C23787BB3DFF85882DFF867
:103CC0003CA24FF0000B09E003F17300C0B206F014
:103CD0001FF823780BF1010B5B451EDD58F8043FFC
:103CE00099F800001844A0F17F038AFB0321DA173A
:103CF000C2EB610202EB42027F28A3EB8203E3DC0A
:103D0000FCF7C0FCE2E7734B03937A4B029305F098
:103D1000FFFF009B1B78002BCCD1039B1B78002B53
:103D20003FF4DCAC99F80030A3F10C007F2840F39D
:103D3000C18172488B3B80FB0320DA17C2EB600025
:103D400000EB4000A3EB800303F17300C0B205F069
:103D5000DFFF009B1B78002B00F09E81664C2378D0
:103D6000002B01F07782DFF8AC81DFF890A14FF0F3
:103D7000000B0AE003F17300C0B205F0C9FF23781D
:103D80000BF1010B5B457FF7A9AC58F8043F99F89C
:103D900000001844A0F18B038AFB0321DA17C2EB61
:103DA00061020C3802EB42027F28A3EB8203E1DCC4
:103DB000FCF768FCE0E72046FCF764FC77E4504A37
:103DC0001278002A40F0A0814E4F4F4C3B70FEF716
:103DD00048BFFCF757FCFFF745BA002008704B4975
:103DE000087840B1394900910978002900F07C81B8
:103DF000009F002139704649097800297FF481A885
:103E0000002C40F0CD80002840F0CA80354C2F4F68
:103E100094F800E02F4C0394364C02942D4C2C491E
:103E20002070344C0097087038702070BEF1000F7D
:103E30007FF479A8FFF783B8264B1B78002B6BD053
:103E400099F80030A3F10C007F2840F392832B4AAD
:103E50008B3B82FB0321DA17C2EB610202EB4202C9
:103E6000A3EB820303F17300C0B205F051FF009B86
:103E70001B78002B50D0204C2378002B4CD0254FA2
:103E8000DFF878804FF0000A09E003F17300C0B258
:103E900005F03EFF23780AF1010A53453CDD57F84F
:103EA000043F99F800001844A0F18B0388FB03211C
:103EB000DA17C2EB61020C3802EB42027F28A3EB57
:103EC0008203E2DCFCF7DEFBE1E700BF9C9FFF1F03
:103ED000489FFF1F0D9DFF1F009FFF1F049FFF1F97
:103EE000689DFF1F2E9DFF1F889FFF1F349DFF1F92
:103EF0006E9DFF1FF29DFF1F8C89FF1FABAAAA2A90
:103F00008B9FFF1F2A9DFF1F149FFF1FF29FFF1F04
:103F1000EE9FFF1F6489FF1F914B1B78FBB1914BF4
:103F20001B88012B00F07686022B00F07087032B94
:103F300001F0EA80042B01F07881052B01F0BB83AE
:103F4000062B01F0E084072B01F0CA85082B01F055
:103F50007D86092B01F08B870A2B01F06887019B76
:103F60001B88002B00F0B8827F4B1B78002B40F0A1
:103F7000AE827E4B7E4A1988D6F80080002001234D
:103F800010602B603CE50135EDB2022D86BF0022AA
:103F9000027005701A46FFF73EBA039800210170BF
:103FA0007449097800293EF4CAAF6D490291097835
:103FB000002900F05287029800210170FEF7BFBF70
:103FC000039B1B78002B7FF4B1AB029B1B78002B6B
:103FD0007FF4ACAB019B1988FFF7AEBB243B002BF1
:103FE000B8F8000040F3748498423EF426AF9BB2C8
:103FF0006148A8F8003001230370FEF71EBFDFF808
:104000007C81C0B298F8001005F05EFEFFF7A8BBF7
:104010005A4B3878197805F057FECBE4D8B298F8A7
:10402000001005F051FE3B68BDE57F21402005F002
:104030001BFE5349534A3B680B600021117040E559
:10404000C0B298F8001005F03FFEFFF712B94E4BD2
:10405000DFF854E11978FEF7F0BE4B2C40F34882AC
:104060001834802CB8F80030484AA8BF8024A342F6
:104070007FF407AEFEF709BF99F8000005F048FE8F
:104080002188FFF759BB424B01931B88002B41F05D
:104090003487334B029345E6029B1B78002B7FF459
:1040A00020AB039B1B78002B7FF440AB92E7FCF71F
:1040B000E9FAC8E4FCF7E6FA48E6FCF7E3FA16E5A5
:1040C000FCF7E0FAFFF718BA421CD2B2022A40F21B
:1040D000568200222A701A46FFF79DB97F20FFF70B
:1040E000D3BA7F20FFF791B91D4F1F4902974FF0B8
:1040F000000C81F800C0009F02994FF0010E87F874
:1041000000E081F800C076E6224F387802F0DAFE4F
:10411000214B1B78002B00F040823B887E2B00F265
:104120003C821E4CDFF884902268D9F80010521AA5
:104130000F2A40F229821A4A0133108899B2398035
:10414000002800F04382C9B2C0B205F08DFD154FC2
:10415000226898F80030C9F800203B70FEF781BD56
:10416000F29DFF1F0A9FFF1F489FFF1FF09DFF1F2B
:10417000109DFF1F2E9DFF1F349DFF1FC89DFF1F19
:10418000389DFF1F8C89FF1FC79FFF1F889FFF1F40
:104190006E9DFF1F649DFF1FF39FFF1F149FFF1F56
:1041A000B89DFF1F2A9DFF1F899DFF1FD49FFF1FE2
:1041B000DFF89CA399F80000BAF80030DF4AE04C21
:1041C000C31A82FB031ED917C1EB6E0101EB41013B
:1041D000A3EB810303EB430354F8233018447F28F7
:1041E00040F38F847F3882FB0032C317C3EB620336
:1041F00003EB4303A0EB83007330DFF858B3C0B286
:1042000005F086FDBBF80030022B7FF68AAA99F8EC
:104210000010BAF80030C94ACB1A82FB030ED81737
:10422000C0EB6E0000EB4000A3EB800303EB430305
:1042300004EB8303586808447F2840F3FA867F38EC
:1042400082FB0032C317C3EB620202EB4202A0EB17
:1042500082007330C0B205F05BFDBBF80030032B69
:104260007FF65FAA99F80010BAF80030B34ACB1A6B
:1042700082FB030ED817C0EB6E0000EB4000A3EBEF
:10428000800303EB430304EB8304A06808447F2806
:1042900040F351817F3882FB0032C317C3EB6202C7
:1042A00002EB4202A0EB82007330C0B205F030FD99
:1042B000FFF737BADFF898A23868BAF800309F4A9B
:1042C0009F4CC31A82FB031ED917C1EB6E0101EB91
:1042D0004101A3EB810303EB430354F8233018445B
:1042E0007F2840F30A847F3882FB0032C317C3EB78
:1042F000620303EB4303A0EB83007330DFF85882C3
:10430000DFF850B298F80010C0B205F0DDFCBBF841
:104310000030022B7FF649AB3968BAF80030874A83
:10432000CB1A82FB030ED817C0EB6E0000EB4000E7
:10433000A3EB800303EB430304EB830358680844B7
:104340007F2840F372867F3882FB0032C317C3EBAD
:10435000620202EB4202A0EB82007330C0B298F816
:10436000001005F0B1FCBBF80030032B7FF61DAB4D
:104370003968BAF80030714ACB1A82FB030ED8179D
:10438000C0EB6E0000EB4000A3EB800303EB4303A4
:1043900004EB8304A06808447F2840F3FB807F3847
:1043A00082FB0032C317C3EB620202EB4202A0EBB6
:1043B0008200733098F80010C0B205F085FCFFF75A
:1043C000F4BA0120FFF760B9DFF884A15B49BAF8BD
:1043D00000205B4C9A1A81FB020ED017C0EB6E00D6
:1043E00000EB4000A2EB800202EB420254F82200F4
:1043F00018447F2840F30084A0F17F0381FB032150
:10440000DA17C2EB610000EB4000A3EB80007330D1
:10441000DFF840B198F80010C0B205F055FCBBF8C9
:104420000030022B50D93968BAF80030434ACB1A11
:1044300082FB030ED817C0EB6E0000EB4000A3EB2D
:10444000800303EB430304EB8303586808447F288D
:1044500040F356867F3882FB0032C317C3EB6202FB
:1044600002EB4202A0EB82007330C0B298F8001059
:1044700005F02AFCBBF80030032B25D93868BAF8C0
:1044800000302E4AC31A82FB031ED917C1EB6E01FE
:1044900001EB4101A3EB810303EB430304EB830432
:1044A000A36818447F2867DD7F3882FB0032C3177A
:1044B000C3EB620202EB4202A0EB82007330C0B297
:1044C00098F8001005F000FC3B68FFF767BB00217F
:1044D000402005F0C9FB4CE599F8000005F018FCF8
:1044E00042E505F015FCFFF710B80120FEF78DBF7F
:1044F000243C002CB8F8003040F39185A3423EF4F0
:10450000C4ACA4B20F4BA8F8004001221A70FEF709
:10451000BCBC0D4B01931B88002B3FF4DFA8FFF7B9
:10452000F6BB0A4A8342A8BF03461360FEF783BE68
:104530001446FFF79BBBFCF7A5F8B6E6ABAAAA2A80
:10454000A82F0100349DFF1F6E9DFF1F109DFF1FB0
:10455000449FFF1FB09FFF1FC89DFF1FDF4BE04C14
:1045600019886A2005F0DAFC98F800303B70FEF7F5
:1045700078BBFCF787F877E4FCF784F89FE72A70AC
:104580001A46FEF748BFD64CD64F98F800303B701D
:10459000FEF767BBFCF776F80CE7D34B1B78002BD4
:1045A000F1D03B88CD4F002BEDD0CD4CDFF84893B8
:1045B0002268D9F80010521A0F2AE5D9CB4A013BDC
:1045C000108899B2398000287FF4BDADC8B205F0DB
:1045D000EBFBBCE5DFF824A399F80000BAF8003043
:1045E000C34AC44CC31A82FB031ED917C1EB6E0128
:1045F00001EB4101A3EB810303EB430354F82330A8
:1046000018447F2840F3FD837F3882FB0032C317B4
:10461000C3EB620303EB4303A0EB83007330DFF8CB
:10462000E0B2C0B205F074FBBBF80030022B7FF69D
:1046300078A899F80010BAF80030AD4ACB1A82FB7E
:10464000030ED817C0EB6E0000EB4000A3EB800315
:1046500003EB430304EB8303586808447F2840F3CB
:10466000F1857F3882FB0032C317C3EB620303EB93
:104670004303A0EB83007330C0B205F049FBBBF8E5
:104680000030032B7FF64DA899F80010BAF80030DF
:10469000974ACB1A82FB030ED817C0EB6E0000EBD3
:1046A0004000A3EB800303EB430304EB8304A06807
:1046B00008447F287FF73FAF7F3882FB0032C31763
:1046C000C3EB620303EB4303A0EB83007330ECE521
:1046D000DFF828A23868BAF80030854A854CC31A3A
:1046E00082FB031ED917C1EB6E0101EB4101A3EB65
:1046F000810303EB430354F8233018447F2840F32D
:1047000059837F3882FB0032C317C3EB620303EB8C
:104710004303A0EB83007330DFF8E881DFF8E0B1FA
:1047200098F80010C0B205F0CFFABBF80030022BA9
:104730007FF63BA93968BAF800306D4ACB1A82FB84
:10474000030ED817C0EB6E0000EB4000A3EB800314
:1047500003EB430304EB8303586808447F2840F3CA
:104760006D857F3882FB0032C317C3EB620303EB16
:104770004303A0EB83007330C0B298F8001005F03B
:10478000A3FABBF80030032B7FF60FA93868BAF8FC
:104790000030574AC31A82FB031ED917C1EB6E01C2
:1047A00001EB4101A3EB810303EB430304EB83041F
:1047B000A36818447F287FF7EDAE7F3882FB003274
:1047C000C317C3EB620303EB4303A0EB8300733017
:1047D000F0E5DFF828A14649BAF80020454C9A1ABE
:1047E00081FB020ED017C0EB6E0000EB4000A2EB85
:1047F000800202EB420254F8220018447F2840F362
:104800000383A0F17F0381FB0321DA17C2EB610070
:1048100000EB4000A3EB80007330DFF8E4B098F8C1
:104820000010C0B205F050FABBF80030022B7FF642
:104830004BAE3968BAF800302D4ACB1A82FB030E12
:10484000D817C0EB6E0000EB4000A3EB800303EB36
:10485000430304EB8303586808447F2840F3F6843D
:104860007F3882FB0032C317C3EB620303EB4303C1
:10487000A0EB83007330C0B298F8001005F024FA62
:10488000BBF80030032B7FF61FAE3868BAF8003053
:10489000174AC31A82FB031ED917C1EB6E0101EB45
:1048A0004101A3EB810303EB430304EB8304A368FF
:1048B00018447F287FF760AE7F3882FB0032C31731
:1048C000C3EB620303EB4303A0EB83007330F6E515
:1048D00001283EF4B2AA0123FFF78ABB649DFF1FA3
:1048E000149FFF1F2A9DFF1FF29FFF1FB89DFF1FF0
:1048F000ABAAAA2AD8320100D49FFF1F449FFF1FF2
:10490000B09FFF1FC89DFF1FDFF8FCA299F80000B1
:10491000BAF80030BA4ABB4CC31A82FB031ED9173F
:10492000C1EB6E0101EB4101A3EB810303EB4303F8
:1049300054F8233018447F2840F3E7817F3882FB06
:104940000032C317C3EB620202EB4202A0EB82000B
:104950007330DFF8B8B2C0B205F0DAF9BBF8003056
:10496000022B7EF6DEAE99F80000BAF80030A44AB9
:10497000C31A82FB0321DA17C2EB610202EB420287
:10498000A3EB820303EB430304EB83035B6818444C
:104990007F2840F328847F380C2290FBF2F302FB3F
:1049A00013007330C0B205F0B3F9BBF80030032B2D
:1049B0007EF6B7AE99F80000BAF80030904AC31AF4
:1049C00082FB0321DA17C2EB610202EB4202A3EB86
:1049D000820303EB430304EB8304A36818447F289A
:1049E0007FF7A9AD7F380C2290FBF2F302FB130096
:1049F00073305AE4DFF810A23868BAF80030804A01
:104A0000804CC31A82FB031ED917C1EB6E0101EB68
:104A10004101A3EB810303EB430354F82330184413
:104A20007F2840F36F817F3882FB0032C317C3EBCE
:104A3000620202EB4202A0EB82007330DFF8D08109
:104A4000DFF8C8B198F80010C0B205F03DF9BBF826
:104A50000030022B7EF6A9AF3868BAF80030684AF9
:104A6000C31A82FB0321DA17C2EB610202EB420296
:104A7000A3EB820303EB430304EB83035B6818445B
:104A80007F2840F3AD837F380C2290FBF2F302FBCA
:104A900013007330C0B298F8001005F015F9BBF898
:104AA0000030032B7EF681AF3868BAF80030544AE4
:104AB000C31A82FB0321DA17C2EB610202EB420246
:104AC000A3EB820303EB430304EB8304A3681844C2
:104AD0007F287FF75FAD7F380C2290FBF2F302FB5B
:104AE0001300733066E44FF47A43013BFDD199F82B
:104AF000000005F00DF9FEF768BFFBF7C3FDFFF7F7
:104B0000FDBBFBF7BFFDFFF778BBDFF8FCA03C491E
:104B1000BAF800203B4C9A1A81FB020ED017C0EB6A
:104B20006E0000EB4000A2EB800202EB420254F860
:104B3000220018447F2840F3EB80A0F17F0381FB23
:104B40000321DA17C2EB610101EB4101A3EB810004
:104B50007330DFF8B8B098F80010C0B205F0B4F8C0
:104B6000BBF80030022B7FF6AFAC3868BAF80030E3
:104B7000234AC31A82FB0321DA17C2EB610202EB5C
:104B80004202A3EB820303EB430304EB83035B6862
:104B900018447F2840F32E837F380C2290FBF2F3D9
:104BA00002FB13007330C0B298F8001005F08CF8C7
:104BB000BBF80030032B7FF687AC3868BAF80030BA
:104BC0000F4AC31A82FB0321DA17C2EB610202EB20
:104BD0004202A3EB820303EB430304EB8304A368C9
:104BE00018447F287FF7C8AC7F380C2290FBF2F383
:104BF00002FB1300733062E4FBF744FD08E400BFDE
:104C0000ABAAAA2A68330100449FFF1FB09FFF1F71
:104C1000C89DFF1FDFF834A399F80000BAF80030F0
:104C2000C24AC34CC31A82FB0317D917C1EB6701F1
:104C300001EB4101A3EB810303EB430354F8233061
:104C400018447F286ADD7F3882FB0032C317C3EB2C
:104C5000620202EB4202A0EB82007330DFF8F0B296
:104C6000C0B205F055F8BBF80030022B7FF677A9EB
:104C700099F80000BAF80030AC4AC31A82FB03214D
:104C8000DA17C2EB610202EB4202A3EB820303EBF1
:104C9000430304EB83035B6818447F2840F3A78237
:104CA0007F380C2290FBF2F302FB13007330C0B28A
:104CB00005F02EF8BBF80030032B7FF650A999F8C9
:104CC0000000BAF80030994AC31A82FB0321DA17B0
:104CD000C2EB610202EB4202A3EB820303EB43034C
:104CE00004EB8304A36818447F2814DD7F380C226A
:104CF00090FBF2F302FB13007330C0B205F008F82A
:104D0000FFF72DB9FBF7BEFC98E6FBF7BBFC20E6EE
:104D1000FBF7B8FC1DE7FBF7B5FCEEE7FBF7B2FCD1
:104D20009CE7DFF828A299F80000BAF800307F4A23
:104D3000804CC31A82FB031ED917C1EB6E0101EB35
:104D40004101A3EB810303EB430354F823301844E0
:104D50007F28DADD7F3882FB0032C317C3EB6203A2
:104D600003EB4303A0EB83007330F2E5DFF8DCA133
:104D70003868BAF800306D4A6E4CC31A82FB031EC5
:104D8000D917C1EB6E0101EB4101A3EB810303EBEA
:104D9000430354F8233018447F28B3DD7F3882FB67
:104DA0000032C317C3EB620303EB4303A0EB8300A2
:104DB000733043E6FBF766FCAEE4DFF890A15B4995
:104DC000BAF800205B4C9A1A81FB020ED017C0EB98
:104DD0006E0000EB4000A2EB800202EB420254F8AE
:104DE000220018447F2893DDA0F17F0381FB03217B
:104DF000DA17C2EB610000EB4000A3EB80007330D8
:104E0000A7E6FBF73FFC0AE4FBF73CFC05E5DFF80F
:104E10003CA199F80000BAF80030444A464CC31A45
:104E200082FB0317D917C1EB670101EB4101A3EB2B
:104E3000810303EB430354F8233018447F287FF7A2
:104E40006DAF7F3882FB0032C317C3EB620303EB05
:104E50004303A0EB8300733000E7384800903848E4
:104E600038490390FEF75FB8DFF8E0A099F800003A
:104E7000BAF800302D4A344CC31A82FB0321DA17EA
:104E8000C2EB610202EB4202A3EB820303EB43039A
:104E900054F8233018447F2840F39F817F380C2238
:104EA00090FBF2F302FB13007330DFF8A4B0C0B242
:104EB00004F02EFFBBF80030022B19D999F800003E
:104EC000BAF800300C22C11A91FBF2F302FB131363
:104ED00002FB03435B6818447F2840F33B847F3820
:104EE00090FBF2F302FB13007330C0B204F010FF2A
:104EF000BBF80030032B7EF614ACBAF8003099F8FA
:104F000000000C22C11A91FBF2F302FB131302FB07
:104F10000344A36818447F287FF70DAB7F3890FBCC
:104F2000F2F302FB13007330FFF7BFB9ABAAAA2A52
:104F3000A82F0100142C0100D83201009C9FFF1FF4
:104F40000D9DFF1F489FFF1F68310100449FFF1FF9
:104F5000B09FFF1FDFF864A33868BAF80030CE4A6C
:104F6000CE4CC31A82FB0321DA17C2EB610202EBBB
:104F70004202A3EB820303EB430354F823301844AB
:104F80007F2840F327817F380C2290FBF2F302FB4D
:104F900013007330DFF82883DFF828B398F8001087
:104FA000C0B204F091FEBBF80030022B1AD9386869
:104FB000BAF800300C22C11A91FBF2F302FB131372
:104FC00002FB03435B6818447F2840F3C7837F38A4
:104FD00090FBF2F302FB13007330C0B298F800109C
:104FE00004F072FEBBF80030032B7EF6DEACBAF89C
:104FF000003038680C22C11A91FBF2F302FB131344
:1050000002FB0344A36818447F287FF7C3AA7F38B4
:1050100090FBF2F302FB13007330FFF7CBB9012BC7
:105020003DF433AF0124FFF76DBAFBF72BFBFFF71D
:1050300095B9FBF727FBFFF70DB9DFF880A296497A
:10504000BAF80020954C9A1A81FB0210D117C1EBD7
:10505000600101EB4101A2EB810202EB420254F834
:10506000220018447F2840F3B280A0F17F030C2077
:1050700093FBF0F200FB12307330DFF848B298F87F
:105080000010C0B204F020FEBBF80030022B1AD989
:105090003868BAF800300C22C11A91FBF2F302FB17
:1050A000131302FB03435B6818447F2840F31E83FD
:1050B0007F3890FBF2F302FB13007330C0B298F814
:1050C000001004F001FEBBF80030032B7FF6FCA9B2
:1050D000BAF8003038680C22C11A91FBF2F302FBD7
:1050E000131302FB0344A36818447F287FF744AAE4
:1050F0007F3890FBF2F302FB13007330FFF7DFB948
:10510000FBF7C0FAFFF7B1B9DFF8B0A199F80000DA
:10511000BAF80030604A624CC31A82FB0321DA17E6
:10512000C2EB610202EB4202A3EB820303EB4303F7
:1051300054F8233018447F2846DD7F380C2290FB3A
:10514000F2F302FB13007330DFF878B1C0B204F061
:10515000DFFDBBF80030022B19D999F80000BAF82E
:1051600000300C22C11A91FBF2F302FB131302FB75
:1051700003435B6818447F2840F38B807F3890FBA3
:10518000F2F302FB13007330C0B204F0C1FDBBF8B0
:105190000030032B7EF6E3AEBAF8003099F8000039
:1051A0000C22C11A91FBF2F302FB131302FB03441E
:1051B000A36818447F287FF7AEAD7F3890FBF2F3E9
:1051C00002FB1300733098E5FBF75CFABCE7FBF7D2
:1051D00059FA52E7FBF756FADCE6FBF753FA64E6B6
:1051E000FBF750FA56E4FBF74DFAFFF7DBBBFBF792
:1051F00049FA5CE5FBF746FAD5E4DFF8C0A099F878
:105200000000BAF80030244A264C35E6DFF8ACA09E
:105210003868BAF80030204A224CA2E6DFF89CA099
:105220001D49BAF800201F4C0DE7DFF890A099F84F
:105230000000BAF80030184A1B4C6DE7FBF722FA61
:10524000FFF79ABAFBF71EFAFFF716BAFBF71AFA3E
:10525000FFF711BB029B1B78002B7EF442AAFEF7DE
:1052600065BA124B1B78002B00F0C182104B1B78E3
:10527000002B7DF40AAE0F4B1B78002B3DF405AEDE
:10528000B8F800300C490A33A8F800300A70FDF76E
:10529000FCBDFBF7F7F977E7ABAAAA2A6831010052
:1052A000683301005C340100142C0100EF9FFF1FE4
:1052B000F09FFF1FF19FFF1F349DFF1F449FFF1FA3
:1052C000C89DFF1FB09FFF1FA14C2388002B40F0FB
:1052D0007D83DFF894B29F499F4A098899F80000BE
:1052E000B2F800E0DFF87882C1EB000C0C229CFBE6
:1052F000F2F102FB11C14FF0900C0CFB0EFE02FB11
:1053000001E16FF00B0E58F8011008440EFB03008A
:105310007F2840F35F85A0F17F0393FBF2F002FB4F
:1053200010307330C0B204F0F3FCBBF800202388C7
:105330001344022B22DD874A874B118899F800001D
:10534000B3F800C0DFF818E2411A0C2291FBF2F327
:1053500002FB1311902303FB0CF302FB0133734494
:105360005B6818447F2840F353857F3890FBF2F345
:1053700002FB13007330C0B204F0CAFCBBF800207B
:1053800023881344032B22DD724A734B118899F84A
:105390000000B3F800C0DFF8C8E1411A0C2291FB0D
:1053A000F2F302FB1311902303FB0CF302FB013316
:1053B00073449B6818447F2840F310857F3890FB26
:1053C000F2F302FB13007330C0B204F0A1FCBBF88F
:1053D000002023881344042B7EF7A3A95F4B1B886E
:1053E000012B7EF49EA999F80020A2F10C007F28E1
:1053F0007FF7A1A88B3A0C2092FBF0F300FB13205F
:105400007330FEF752BF524C2388002B40F01D83AF
:10541000DFF854B14F49504A0988D7F80080B2F8F4
:1054200000E04F48C1EB080C0C229CFBF2F102FBA0
:1054300011C14FF0900C0CFB0EFE02FB01E16FF06E
:105440000B0E405880440EFB03807F2840F39D8460
:10545000A0F17F0393FBF2F002FB10307330414B5D
:10546000C0B2197804F030FCBBF800202388134444
:10547000022B23DD374A384B11883868B3F800C057
:10548000DFF8DCE0411A0C2291FBF2F302FB13116E
:10549000902303FB0CF302FB013373445B68184455
:1054A0007F2840F3AB847F3890FBF2F302FB1300BC
:1054B00073302C4BC0B2197804F006FCBBF8002006
:1054C00023881344032B23DD224A234B1188386899
:1054D000B3F800C0DFF888E0411A0C2291FBF2F328
:1054E00002FB1311902303FB0CF302FB0133734403
:1054F0009B6818447F2840F38F847F3890FBF2F339
:1055000002FB13007330174BC0B2197804F0DCFBB8
:10551000BBF8002023881344042B7EF746AA0F4BC8
:105520001B88012B7EF441AA3A68A2F10C007F2867
:1055300040F3E6818B3A0C2092FBF0F300FB132042
:105540007330084BC0B2197804F0BEFBFEF72DBAD9
:10555000D09DFF1F449FFF1FF69EFF1F629DFF1FF0
:10556000A42C0100C89DFF1FB09FFF1FCD4C2288B7
:10557000002A00F0D081CC49DFF858B30988BBF885
:1055800000000331884227DDC848C9490088B1F8C6
:1055900000E0DFF844C3181A0C2190FBF1F901FB7D
:1055A00019004FF0900909FB0EFE01FB00E06FF0BF
:1055B0000B0E5CF8000003440EFB02307F2840F322
:1055C000AA837F3890FBF1F301FB13007330C0B264
:1055D00098F8001004F078FBBBF8002023881344EF
:1055E000022B23DDB14BB24A38681B88B2F800C0E9
:1055F000DFF8E4E2C31A0C2193FBF1F201FB123253
:10560000902303FB0CF301FB023373445B681844E3
:105610007F2840F308847F3890FBF1F301FB1300EF
:105620007330C0B298F8001004F04EFBBBF80020B5
:1056300023881344032B23DD9C4B9D4A38681B8829
:10564000B2F800C0DFF890E2C31A0C2193FBF1F22C
:1056500001FB1232902303FB0CF301FB0233734472
:105660009B6818447F2840F3DB837F3890FBF1F37D
:1056700001FB13007330C0B298F8001004F024FB53
:10568000BBF8002023881344042B7EF71DAF864B04
:105690001B88012B7EF418AF3A68A2F10C007F281A
:1056A0007EF76AAF8B3A0C2092FBF0F300FB1320DD
:1056B0007330FEF704BFDFF8F4A199F80000BAF8E0
:1056C00000307C4CC11A0C2291FBF2F302FB131345
:1056D00002FB03F3E35818447F287FF775AD7F384A
:1056E00090FBF2F302FB130073302DE5FAF7CAFFCB
:1056F000E4E4714B1B88182B12D099F80020134456
:10570000A3F118007F2840F376830C20973B93FB8E
:10571000F0F200FB123303F17300C0B204F0F8FAA8
:10572000664A674B127833F81230182B3DF4F9AF04
:1057300099F800201344A3F118007F287EF7FBAEF0
:105740000C20973B93FBF0F200FB123303F1730044
:10575000FEF7ABBDFAF796FFFFF7C7BBFAF792FF6C
:105760003BE4554B1A88182A13D03B681344A3F125
:1057700018007F2840F33C830C20973B93FBF0F20A
:1057800000FB123303F173004E4BC0B2197804F0E2
:105790009BFA4A4B4A491A78022A94BF01320022E6
:1057A0001A701A7831F81200182810D10424022A2D
:1057B00002F10100C2B288BF002231F8120018289D
:1057C00004D1013CF3D11A70FEF7EFB81A703B68B0
:1057D0000344A3F118007F2840F392800C20973BEC
:1057E00093FBF0F200FB123303F17300A9E6364B92
:1057F0001B78002B7DF4FDAF344B1B78002B3DF460
:1058000044ABB8F8003032490133A8F800300A70D0
:10581000FDF73BBB2C4B1B78002B7DF436AB2B4BA1
:105820001B78002B3DF431ABB8F800302849013B20
:10583000A8F800300A70FDF728BB1F4A1288182A02
:1058400012D01344A3F118007F2840F3CE820C201D
:10585000973B93FBF0F200FB123303F17300C0B2ED
:1058600098F8001004F030FA144B15491A78022AFF
:1058700094BF013200221A701A7831F812001828E9
:105880002DD10424022A02F10100C2B288BF0022F5
:1058900031F81200182821D1013CF3D11A703B686D
:1058A000FEF77CB9D09DFF1F629DFF1F449FFF1F25
:1058B000F69EFF1F683101009A9FFF1FC489FF1FDA
:1058C000609FFF1FC89DFF1FF09FFF1FF19FFF1FDD
:1058D000349DFF1FB09FFF1FA42C01001A703B686E
:1058E0000344A3F118007F287EF746AE0C20973BB7
:1058F00093FBF0F200FB123303F17300FEF7DFBD00
:10590000FAF7C0FE1DE6DFF834A399F80000BAF8F4
:105910000030C04CD6E6DFF830B335E6BE4B1A880F
:10592000182A13D03B681344A3F118007F2840F3D2
:1059300069820C20973B93FBF0F200FB123303F1DA
:105940007300B64BC0B2197804F0BEF9B44BB54938
:105950001A78022A94BF013200221A701A7831F89C
:10596000120018287FF433AF0424022A02F1010246
:1059700094BFD2B2002231F8120018287FF426AF6B
:10598000013CF2D11A70FEF710B8A34B1B88182BFC
:1059900012D099F800201344A3F118007F2840F397
:1059A00034820C20973B93FBF0F200FB123303F19F
:1059B0007300C0B204F0ACF9994A9A4B127833F8EC
:1059C0001230182B7FF4B4AEFDF7ABBE964ADFF869
:1059D00078B21288BBF80010033291427FF7A5AC71
:1059E00079E48D4A1288182A12D01344A3F11800C2
:1059F0007F2840F3F7810C20973B93FBF0F200FBEC
:105A0000123303F17300C0B298F8001004F05CF98F
:105A1000834B84491A78022A94BF013200221A70FB
:105A20001A7831F8120018287FF459AF0424022A9A
:105A300002F1010294BFD2B2002231F812001828FC
:105A40007FF44CAF013CF2D128E7774ADFF8F8B198
:105A50001288BBF80010033291427FF705ADD9E4FC
:105A6000724B01227F2107201A8004F0FDF87F216C
:105A70000B2004F0F9F8FDF7E7BE6D4B04227F21FF
:105A800007201A8004F0F0F800210B2004F0ECF855
:105A9000FDF7D3BE664B02227F2107201A8004F057
:105AA000E3F87F210B2004F0DFF8FDF7C1BE604B67
:105AB000002107201C8004F0D7F87F210B2004F080
:105AC000D3F8FDF7B0BE5B4B00227F2107201A8080
:105AD00004F0CAF87F210B2004F0C6F8FDF7BCBE25
:105AE000554C2388002B40F0E581DFF85CB1534929
:105AF00099F80000524A09881788DFF848E1411AEE
:105B00000C2291FBF2FC02FB1C114FF0900C0CFBE1
:105B100007F702FB01716FF00B075EF801100144FB
:105B200007FB03107F2840F3C2817F3890FBF2F31C
:105B300002FB13007330C0B204F0EAF8BBF8002097
:105B400023881344022B21DD3C4B3D4A99F8000089
:105B50001B88B2F800E03B4FC31A0C2193FBF1F213
:105B600001FB1232902303FB0EF301FB02333B4493
:105B70005B6818447F2840F3B4817F3890FBF1F3D1
:105B800001FB13007330C0B204F0C2F8BBF8002070
:105B900023881344032B21DD284B294A99F8000060
:105BA0001B88B2F800E0274FC31A0C2193FBF1F2D7
:105BB00001FB1232902303FB0EF301FB02333B4443
:105BC0009B6818447F2840F389817F3890FBF1F36C
:105BD00001FB13007330C0B204F09AF8BBF8002048
:105BE00023881344042B7EF7BAA90F4B1B88012B83
:105BF0007EF4B5A999F80020A2F10C007F287FF768
:105C00008AA88B3A0C2092FBF0F300FB1320733030
:105C1000FFF773B85C3401005A9DFF1FC89DFF1F3A
:105C2000C489FF1FD89EFF1F629DFF1FE29DFF1FBB
:105C30003C9FFF1F2C9DFF1FD09DFF1F449FFF1FF8
:105C4000F69EFF1FA42C0100B09FFF1FAD4B1B88C9
:105C5000182B12D099F800201344A3F118007F28C4
:105C600040F342810C20973B93FBF0F200FB123390
:105C700003F17300C0B204F04BF8A34AA34B1278AF
:105C800033F81230182B3EF46AA999F80020134417
:105C9000A3F118007F287FF73EA80C20973B93FBC9
:105CA000F0F200FB123303F17300FFF726B8984AB5
:105CB0001288182A12D01344A3F118007F2840F349
:105CC0000A810C20973B93FBF0F200FB123303F1A7
:105CD0007300C0B298F8001003F0F6FF8A4B8D49AC
:105CE0001A78022A94BF013200221A701A7831F809
:105CF000120018287FF4F3AD0424022A02F10102F5
:105D000094BFD2B2002231F8120018287FF4E6AD19
:105D1000013CF2D1C2E5FAF7B5FC58E47C4B1A8895
:105D2000182A13D03B681344A3F118007F2840F3CE
:105D3000E1800C20973B93FBF0F200FB123303F160
:105D40007300754BC0B2197803F0BEFF6E4B7149FA
:105D50001A78022A94BF013200221A701A7831F898
:105D6000120018287FF433AD0424022A02F1010244
:105D700094BFD2B2002231F8120018287FF426AD69
:105D8000013CF2D11A70FDF710BEFAF77BFCFFF769
:105D900066BB5F4B1B88182B12D099F80020134468
:105DA000A3F118007F2840F3A2800C20973B93FBBF
:105DB000F0F200FB123303F17300C0B203F0A8FF4E
:105DC000514A544B127833F81230182B7FF4B0AC90
:105DD000FDF7A7BCFAF756FCFFF7A4BAFAF752FC96
:105DE000FFF7F2BAFAF74EFC0DE6FAF74BFC36E590
:105DF000FAF748FCC8E4FAF745FC8EE4FAF742FCEF
:105E0000FFF757BBFAF73EFC9BE5FAF73BFCD0E502
:105E1000FAF738FCFFF7AFBAFAF734FCFFF773BBB9
:105E2000FAF730FC27E4FAF72DFCFFF7FABB384B02
:105E30001B88182B11D099F800201344A3F11800E7
:105E40007F2845DD0C20973B93FBF0F200FB1233DB
:105E500003F17300C0B203F05BFF2B4A2D4B1278A5
:105E600033F81230182B7FF410AFFEF778B82B4BB5
:105E70001B88182B11D099F800201344A3F11800A7
:105E80007F2822DD0C20973B93FBF0F200FB1233BE
:105E900003F17300C0B203F03BFF1B4A204B1278A2
:105EA00033F81230182B7FF4F0AEFEF758B8FAF73B
:105EB000E9FB40E61B4ADFF874B01288BBF800101B
:105EC000033291427FF73AAE11E6FAF7DBFBE1E7E6
:105ED000FAF7D8FBBEE7FAF7D5FBFAE6FAF7D2FBFA
:105EE00079E6FAF7CFFB4EE6FAF7CCFBC2E6FAF713
:105EF000C9FB62E7FAF7C6FB23E70B4B0293FDF7FA
:105F000006BF00BF9A9FFF1FC489FF1F609FFF1F2E
:105F10005C9DFF1FE09EFF1FC89DFF1F5A9DFF1F36
:105F2000D89EFF1F629DFF1FF29DFF1FB09FFF1FA6
:105F300038B507F0A7FE0E4805F0DEFD0D4805F068
:105F4000DBFD0D4805F0D8FD00234FF07E52012106
:105F50000A48FAF78BFA0A4B0A4A0B4980240025B3
:105F60001C7118461D60BDE838400BF08FBC00BFA7
:105F7000489DFF1F789DFF1FE89DFF1F189FFF1F73
:105F8000A89FFF1F1C89FF1F2906000010B50446AB
:105F9000A4206368198803F0C1FFE368A62019886C
:105FA000BDE8104003F0BABF43682A20198803F007
:105FB000B5BF00BF10B5044622206368198803F0FE
:105FC000ADFFE36824201988BDE8104003F0A6BFA8
:105FD00010B504460A206368198803F09FFFE36840
:105FE0000C201988BDE8104003F098BF10B5044696
:105FF00006206368198803F091FFE3680820198878
:10600000BDE8104003F08ABF10B504460220636863
:10601000198803F083FFE36804201988BDE8104065
:1060200003F07CBF70B50E4C84B01225042201230E
:1060300006460390029320468DE824001423102185
:1060400006F05EFF0622092302930396019520467F
:1060500000921423102106F053FF04B070BD00BF5E
:1060600024A0FF1FF8B5B04CB4F90030032B00F0AA
:106070001281002B6AD0022B00F08A80052B00F0E1
:10608000B580012B00F0DD80042B00D0F8BDA74FB8
:10609000A74E00254FF4AF74E9B2A64805F094FD71
:1060A00057F8043BC3F5967300FB03F086FB00230F
:1060B000C017C0EB6310844205F10105A8BF044678
:1060C000062DE9D19C4F9A4E0025E9B29B4805F078
:1060D0007BFD57F8043BC3F5967300FB03F086FB8A
:1060E0000023C017C0EB6310844205F10105A8BF6F
:1060F00004460C2DE9D1924F8D4E0025E9B291480E
:1061000005F062FD57F8043B894AC3F5967300FB1E
:1061100003F086FB0013C017C0EB6310844205F147
:106120000105A8BF04460C2DE8D1A4F114013129C2
:1061300000F3A38040F26C7232218348834B0180CC
:106140001A602A20BDE8F84003F0E8BE0E2007F0F0
:10615000FDFC40F6FF71C8308842A8BF084620EA1F
:10616000E07000F2DC5283B28A42794D794EA8BFCA
:106170000A460220194633802A8003F0CFFE298880
:10618000042003F0CBFEB4F90030022B7FF476AF8D
:10619000012008F0F7FD0546002008F0F3FDA842B5
:1061A000B8BF284600F1C801B1F5FA7FC0F2B4804B
:1061B000B1F57A6FA8BF4FF47A6101F54873B3F572
:1061C0007A6FA8BF4FF47A639BB289B2624A634D7B
:1061D00011800A202B8003F0A1FE29880C2003F0F7
:1061E0009DFEB4F90030052B7FF44BAF0F2008F073
:1061F000C9FDC0F53F630433B3F5AF6FC0F28980CA
:10620000B3F5FA6FA8BF4FF4FA6399B2544BC0F5D7
:106210004360B0F5AF6F198061DBB0F5FA6FA8BFCE
:106220004FF4FA6083B24F4DA4202B8003F076FE2A
:106230002988A62003F072FEB4F90030012B7FF408
:1062400023AF152007F082FC00F59671B1F52F7F82
:106250004DDB41F25C23994263DC434A00F56170F7
:1062600089B2B0F52F7F1180B8BF4FF42F7344DB94
:106270008342A8BF03469BB23FE040F23A73A4F5C5
:10628000B97403FB04F482FB0432E417A4EB62123A
:1062900089B2323251E7102008F074FDC830B0F5F1
:1062A000FA7F1FDBB0F57A6F0146A8BF4FF47A6121
:1062B00001F51673B3F57A6FA8BF4FF47A639BB2FA
:1062C00089B22A4A2A4D118022202B8003F026FE13
:1062D0002988242003F022FEB4F90030C9E64FF4E7
:1062E000AF63A0E740F24C434FF4FA71E9E740F2A4
:1062F00014534FF42F711C4A11801E4D06202B8021
:1063000003F00CFE2988082003F008FEB4F90030E1
:10631000BAE64FF4AF6179E740F214534FF4FA71E3
:1063200054E71946E7E700BFFE9FFF1F548AFF1F8F
:10633000B5814E1B489DFF1F248AFF1F789DFF1FBC
:106340002C89FF1FE89DFF1FB49FFF1F108AFF1FAE
:10635000BA9FFF1FF09DFF1F509FFF1F589DFF1FFB
:10636000F49DFF1F709FFF1F929DFF1F049FFF1F43
:10637000009FFF1F849FFF1F2DE9F041224D82B037
:10638000012602B284B20092284601967823192190
:1063900006F0FCFC04F10C0212B28DE84400284621
:1063A000A7197823192104F1020806F0EFFC3FB287
:1063B0000FFA88F819233A46284619460196CDF86F
:1063C000008006F0E3FC78233A4628461946CDF8CB
:1063D0000080019604F10A070B3406F0D7FC3FB2A7
:1063E00024B278233A46284619468DE8500006F034
:1063F000CDFC192300943A4601962846194606F02A
:10640000C5FC02B0BDE8F08124A0FF1F30B583B009
:1064100000230C4605B2009326225B231C210C4866
:1064200006F004FA294601232622094805F00EFD4C
:10643000002C24B205DB214601232622044805F066
:1064400005FD044A044B15801C8003B030BD00BF1D
:1064500024A0FF1F6E8AFF1F708AFF1F2DE9F041E5
:10646000BB4C237882B01BB1BA4B4FF6FF721A8037
:10647000B94BB3F90030CBB9B84AB64B1068B3F991
:10648000002080F30C005B2303FB00F000131C30A2
:1064900082424BD04FF0FF31FFF7B8FFB04806F013
:1064A00029FA0023237002B0BDE8F081012B1BD034
:1064B000022B5AD0032B3FD0042B00F09980052BE0
:1064C000EFD10F2008F05EFCC0F53B600830B0F55E
:1064D000AF6F48DBB0F5FA6FA8BF4FF4FA60A0F5D4
:1064E000AF625B239F4835E09F4B1B78002B75D034
:1064F000152007F02BFB9D4B1860B0F52F7F32DB8A
:1065000041F25C239842A8BF1846A0F52F735B2286
:10651000974802FB03F380FB0320DB17C3EBA020AB
:106520001C308C4BB3F900308342B3D1914BB3F99B
:1065300000300133AED1B4E78F4B1B68B3F5FA7F5F
:1065400011DBB3F57A6FA8BF4FF47A638B48A3F5DC
:10655000FA725B2303FB02F380FB0320DB17C3EB20
:1065600020201C30DDE71C20DBE7854B1B68B3F5E2
:10657000FA7F3BDBB3F57A6FA8BF4FF47A63A3F5DC
:10658000FA727E485B2303FB02F380FB0320DB17D8
:10659000C3EB20201C307B4B1B68B3F5FA7F23DB59
:1065A000B3F57A6FA8BF4FF47A63A3F5FA72734913
:1065B0005B2303FB02F381FB0321DB17C3EB2121E8
:1065C0001C31644BB3F9003083427FF465AF694BF3
:1065D000B3F900308B427FF45FAF62E7112008F01F
:1065E000D1FB624B186088E71C21EAE71C20D2E748
:1065F000252200258DE8240076231C215848624E70
:10660000624FDFF8A08106F0C1FB16E0B0F5AF7F66
:10661000A8BF4FF4AF70323802FB00F088FB0031A6
:10662000C017C0EB61111C3109B201231D442522A2
:106630004B4805F00BFC0C2D14D0E9B2544805F082
:10664000C3FA56F8043BC3F5967300FB03F087FBCF
:106650000013C017C0EB631031284FF05B02D5DC8C
:106660001C21E2E7262200258DE8240076231C2148
:106670003B48484E454FDFF82C8106F087FB16E07B
:10668000B0F5AF7FA8BF4FF4AF70323802FB00F017
:1066900088FB0031C017C0EB61111C3109B2012326
:1066A0001D4426222E4805F0D1FB0C2D14D0E9B252
:1066B000394805F089FA56F8043BC3F5967300FB98
:1066C00003F087FB0013C017C0EB631031284FF0B5
:1066D0005B02D5DC1C21E2E7272200258DE824009F
:1066E00076231C211E482D4E284FDFF8B88006F077
:1066F0004DFB17E0B0F5AF7FA8BF4FF4AF70323855
:1067000002FB00F088FB0031C017C0EB61111C31A7
:1067100009B201231D442722114805F097FB062DDD
:106720003FF4BCAEE9B21E4805F04EFA56F8043B01
:10673000C3F5967300FB03F087FB0013C017C0EB93
:10674000631031284FF05B02D4DC1C21E1E700BF6D
:10675000F89FFF1F6E8AFF1FFE9FFF1F549FFF1FA2
:1067600024A0FF1F37800B6D0C9FFF1F189DFF1F7C
:10677000D3058541708AFF1F689DFF1F011FB81256
:10678000749DFF1F3C9DFF1F248AFF1FB5814E1B78
:10679000789DFF1F2C89FF1FE89DFF1F548AFF1F54
:1067A000489DFF1F4B48371B2DE9F041044682B03E
:1067B00071482768E56805F091FF1120FFF7DCFDBF
:1067C000012619234FF02808194624226A48019609
:1067D000CDF8008006F0DAFA7823194624226648BC
:1067E0000196CDF8008006F0D1FA3146624806F0F5
:1067F00063FE02221921604806F05AFE38460BF06B
:106800001FFE394602465C4806F0ECFF5A4806F087
:10681000FFFF14220021584806F04AFE0322574980
:10682000554806F0DFFF544806F0F2FF232200210E
:10683000514806F03DFE032251494F4806F0D2FF71
:106840004D4806F0E5FF7DB12F20FFF795FD322280
:106850000021494806F02CFE03224A49464806F02A
:10686000C1FF454806F0D4FF0123474A184613707C
:10687000FFF7D8FB2189638962685B1A5C2B128859
:1068800054DD521A02EB4202C2EB4212013392FB78
:10689000F3F31B333D4A3848138001261A221BB2FA
:1068A0008DE844001946142206F070FA002D4FD0EE
:1068B000218A638AE2685B1A5C2B12883EDC511ADB
:1068C0005C2202FB01F292FBF3F31B33304A2A48AD
:1068D000138001251BB2382219468DE8240032228C
:1068E00006F054FA4023002209218DE806002248D0
:1068F000194606F019FA29461F4806F0DDFD022266
:1069000044211D4806F0D4FD63681B48198806F031
:10691000CFFF2A461F49184806F064FFE36816486F
:10692000198802B0BDE8F04106F0C2BF511A5C22DE
:1069300002FB01F292FBF3F31B33ABE7521A02EBBB
:106940004202C2EB4212334492FBF3F31B33BDE726
:10695000402309212A46009107480195194606F06F
:10696000E3F93146044806F0A7FD022268210248F7
:1069700006F09EFD6368D2E724A0FF1FC435010026
:10698000C8350100CC3501009DA0FF1FFA9FFF1FF5
:10699000FC9FFF1FD03501002DE9F0471F4682B054
:1069A0001446002A4ED0052A0646D0F80C8000F086
:1069B000AB800B9B894A00EBC305012CB5F80AE0BC
:1069C00029896868C1EB0E0382FB03C21A444FEAAF
:1069D000E373C3EBA213028851D0042C00F08D8026
:1069E0000022402309218DE806007D48194606F063
:1069F0009BF901217A4806F05FFD0222B8F1000FF1
:106A000000F0E1804421764806F052FD7368744836
:106A1000198806F04DFF73497148012206F0E2FE25
:106A2000F3686F48198806F043FF6F4B022CB3F9E7
:106A3000001000F0A680082C00F0C280012002B0F7
:106A4000BDE8F087694E6A4A33681268CB1A9342F0
:106A50000D4655D9674A3B8811786148012918BF0E
:106A6000012414700A9A06321BB212B28DE8140087
:106A70001946BDF9282006F089F93560DEE79BB29A
:106A8000D31A994203DC9E457146A8BF19460A9A5B
:106A90000180B7F90030BDF928A0514802F106097C
:106AA0004FF0000E0FFA89F919465246CDF80090C2
:106AB000CDF804E006F06AF929896A896868521AF3
:106AC00003885C2AA3EB010373DD03EB430301326C
:106AD000C3EB431393FBF2F303F11B0213B2012048
:106AE0003A80194652460190CDF800903C4806F095
:106AF0004DF9404B00221A7072E712FA83F3C0E797
:106B0000204602B0BDE8F08707254FF000095A2360
:106B100023228DE820021A21314806F005F90121CF
:106B20002F4806F0C9FC01212D4806F0CBFC23229A
:106B300035212B4806F0BCFC2A462F49284806F090
:106B400051FE274806F064FE254805F0D3FE4FF4B9
:106B5000FA6007F04DFDFFF785FA5A2323221A2128
:106B60008DE820021E4806F0DFF81D4805F0C2FE41
:106B70003046FFF719FE214B01221A70FFF76EFC19
:106B80002EE74A1C12B21A8091423FF457AF0A9A7C
:106B9000B7F9003012480632012412B200921946A9
:106BA0000194BDF9282006F0F1F8204602B0BDE8B6
:106BB000F0875C2101FB03F393FBF2F21B328DE7BC
:106BC00000221A80E0E76821054806F071FC73682E
:106BD0000348198806F06CFE27E700BFC94216B2C9
:106BE00024A0FF1FD035010002A0FF1F88A0FF1FB7
:106BF000E04501009DA0FF1FD4350100F89FFF1F55
:106C00002DE9F04F5A4E5B4DB6F900704C7855F8AF
:106C1000277085B08146984604B10C78DFF874A1DE
:106C20001AB99AF80030002B39D0534D002338465A
:106C30002B808AF80030FFF7B7FD504A504BB5F96A
:106C40000000012111704FF6FF721A8060B3012815
:106C50005ED0012032232246019000934946494BE1
:106C60003846FFF799FE00240346B5F90020022AB2
:106C700039DD00222A80B6F900203D49002A3BDB9D
:106C8000052AC4BF00220A80B8F1000F39D1002CB8
:106C90000CBF18464FF0FF3005B0BDE8F08F364D01
:106CA000B5F900000028D2D1DFF8ECB0364ADBF8A5
:106CB00000301268C3EB0903934227D9334B1A788B
:106CC000012A18BF01201870FFF7ACF90123CBF897
:106CD0000090012C2AD0042C35D0022C3AD0082C5C
:106CE0003ED00024C1E7C6D1FA68002AC1D0B6F967
:106CF00000201F49002AC3DA05220A80B8F1000FDC
:106D0000C5D00393FFF7AAFB039BC0E70346E0E768
:106D10004FF0000E142322468DE8084049461C4BD4
:106D200038467446FFF738FE03469EE732888AF8F5
:106D30000040013232807A6982B1002438460393E0
:106D40009047039B91E732880121013A32808AF80B
:106D50000010F0E701222A8000248CE7144684E723
:106D60007A69002129804FF0FF34002AE6D182E7BA
:106D7000FE9FFF1F748AFF1F02A0FF1FF89FFF1FC7
:106D80006E8AFF1FFC9FFF1FE04501009DA0FF1FB3
:106D9000FA9FFF1F00A0FF1F88A0FF1F01210D20E9
:106DA00007F0EABB00210D2007F0E6BB01460D20ED
:106DB00007F0E2BB08B50D2007F0E4FBB0FA80F164
:106DC00049090D20BDE8084007F0D6BB10B50021E9
:106DD00044080D2007F0D0FB204607F009FC0D20E9
:106DE000012107F0C9FB2046BDE8104007F000BCB8
:106DF0002D4A2E4B10881B68984210B549DA2C4A50
:106E00001288141A9A42A8BF1A46B4F5157F36DACA
:106E1000121A40F2532303FB02F393FBF4F1053102
:106E20000A2007F019FA234B1978C9B3224B2349DA
:106E30001B6840F2271283F3070302FB03F381FB75
:106E400003211944DB17C3EBA1110531092007F019
:106E500003FA1B4B1968F1B181F3070140F22712C5
:106E6000164802FB01F380FB03211944DB17C3EB37
:106E7000A11105311620BDE8104007F0EDB9131A35
:106E80004FF41572611C02FB03F393FBF1F1053122
:106E9000C6E70021C4E71620BDE8104007F0DCB9C2
:106EA000092007F0D9F9D4E7F09DFF1F109DFF1FBF
:106EB000BA9FFF1F969DFF1FA09FFF1F090402811D
:106EC0006C9FFF1F7F2838B5A8BF7F200F4C4FF461
:106ED000167202FB00F284FB02311144D217054600
:106EE000C2EBA1110A2007F0B7F97F3D4FF496736A
:106EF00003FB05F384FB03211944DB17A3EBA1116A
:106F00000920BDE8384007F0A7B900BF0904028195
:106F1000C368B3F9003030B583EAE374A4EBE374DB
:106F2000002BA0B218DB012300E0134603EB830221
:106F300052009442F9DA0A4D90FBF3F285FB03E428
:106F400003FB1200DB173032D3EBA40380B201F84D
:106F5000012BF1D10B7030BD2D230B700131E2E715
:106F60006766666638B5094D8224204602F0F0FF58
:106F700035F8021B00B28842204601D002F0CEFF55
:106F80000234A4B28A2CF0D138BD00BFE09EFF1FAE
:106F9000024B8020198802F0C1BF00BF5C9DFF1F1B
:106FA00038B5094D7824204602F0D2FF35F8021B8F
:106FB00000B28842204601D002F0B0FF0234A4B2F1
:106FC000802CF0D138BD00BFD89EFF1F024B762029
:106FD000198802F0A3BF00BF5A9DFF1F38B5094DA5
:106FE0004624204602F0B4FF35F8021B00B2884266
:106FF000204601D002F092FF0234A4B24E2CF0D110
:1070000038BD00BF609FFF1F024B4420198802F06B
:1070100085BF00BF9A9FFF1F024B4E20198802F0C8
:107020007DBF00BF6E9DFF1F024B9A20198802F0A2
:1070300075BF00BFD09DFF1F024B9820198802F03A
:107040006DBF00BF629DFF1F024B8C20198802F0AC
:1070500065BF00BFF69EFF1F024B9C20198802F0FF
:107060005DBF00BFB09FFF1F024BA020198802F038
:1070700055BF00BF689FFF1F024B9620198802F082
:107080004DBF00BF449FFF1F024B8A20198802F0AA
:1070900045BF00BF0A9FFF1F024B1020198802F056
:1070A0003DBF00BF089FFF1F024B2C20198802F034
:1070B00035BF00BF469DFF1F024B1E20198802F0FE
:1070C0002DBF00BF609DFF1FC3680E20198802F00E
:1070D00025BF00BF024B2820198802F01FBF00BF48
:1070E0005E9FFF1F024B6420198802F017BF00BF8C
:1070F000589FFF1F024BB420198802F00FBF00BF3A
:10710000A09DFF1F024BB620198802F007BF00BFE9
:10711000E09FFF1F024B5A20198802F0FFBE00BFFC
:10712000209DFF1F024B1620198802F0F7BE00BFFA
:107130002C9DFF1F024B2E20198802F0EFBE00BFCE
:10714000D89DFF1F024B3020198802F0E7BE00BF18
:10715000C89FFF1F024B9E20198802F0DFBE00BFB0
:10716000CC89FF1F024BAC20198802F0D7BE00BFAC
:107170005A9FFF1F024BAE20198802F0CFBE00BFFE
:107180006C9DFF1F024BB020198802F0C7BE00BFE4
:10719000EC9EFF1F024BB220198802F0BFBE00BF59
:1071A0008A9DFF1F024B1820198802F0B7BE00BF4E
:1071B000F69DFF1F024BA220198802F0AFBE00BF50
:1071C0008E9FFF1F024B1A20198802F0A7BE00BF36
:1071D0007A9DFF1F024B1C20198802F09FBE00BF42
:1071E000709DFF1F024B6620198802F097BE00BFFA
:1071F000989FFF1F024B7220198802F08FBE00BFBC
:10720000C49FFF1F024B2020198802F087BE00BFD9
:10721000969FFF1F024B3220198802F07FBE00BFED
:10722000869FFF1F024B6820198802F077BE00BFBF
:10723000B89DFF1F024B6C20198802F06FBE00BF83
:10724000149DFF1F024B6E20198802F067BE00BF1D
:10725000F69FFF1F024B5220198802F05FBE00BF4D
:107260006489FF1F024B5020198802F057BE00BFEF
:107270002089FF1F024B5420198802F04FBE00BF27
:10728000208AFF1F024B5C20198802F047BE00BF16
:107290006C8AFF1F024B5E20198802F03FBE00BFC0
:1072A0005C89FF1F024B5620198802F037BE00BFD1
:1072B000C69DFF1F244B1B880B2B43D8DFE803F030
:1072C0000B10151A1F24292E33383D0608460422B8
:1072D0001E490BF073B9084604221D490BF06EB924
:1072E000084604221B490BF069B9084604221A49D2
:1072F0000BF064B90846042218490BF05FB9084640
:10730000042217490BF05AB90846042215490BF01C
:1073100055B90846042214490BF050B90846042216
:1073200012490BF04BB90846042211490BF046B93B
:10733000084604220F490BF041B9084604220E49C1
:107340000BF03CB9704700BF449FFF1F8042010013
:10735000CC3F01002C3E0100683F0100303E01009F
:10736000C4430100343E0100383E010018410100D1
:107370003C3E01008C420100403E0100064B074AA2
:1073800010B41C88064B0846002C14BF1146194641
:10739000042210BC0BF012B9909DFF1F443E010067
:1073A000483E0100064B074A10B41C88064B0846AD
:1073B000002C14BF11461946042210BC0BF0FEB875
:1073C000DA9DFF1F443E0100483E0100064B074A7C
:1073D00010B41C88064B0846002C14BF11461946F1
:1073E000042210BC0BF0EAB8FE9EFF1F443E0100D1
:1073F000483E0100064B074A10B41C88064B08465D
:10740000002C14BF11461946042210BC0BF0D6B84C
:10741000469FFF1F443E0100483E0100064B074ABD
:1074200010B41C88064B0846002C14BF11461946A0
:10743000042210BC0BF0C2B8E29DFF1F443E0100C5
:10744000483E01001B4B1B880A2B0AD8DFE803F0DB
:107450000A0E12161A1E22262A2E0600164B18682D
:1074600008607047154B186808607047144B18681F
:1074700008607047134B186808607047124B186813
:1074800008607047114B186808607047104B186807
:10749000086070470F4B1868086070470E4B1868FB
:1074A000086070470D4B1868086070470C4B1868EF
:1074B000086070470A9FFF1F703E0100483E0100B0
:1074C0004C3E0100503E0100543E0100583E010078
:1074D0005C3E0100603E0100643E0100683E010028
:1074E0006C3E0100F0B52B4E2B4FDFF8C4E0054693
:1074F0000FCE87B06C460FC496E803003B68274A5E
:10750000274F44F8040B40F6CC308342C8BF3A46BC
:10751000BEF800602180012E11889278ADF80D1020
:107520008DF80F202AD032D340F6CA02022E18BF9F
:1075300000229A4226DAA3F698031A491A4AC3EBA4
:10754000031381FB03011944DB17C3EB61232433CD
:1075500082FB0321DA17C2EBA10202EB8201A3EB4B
:107560004103303330328DF813308DF811206946E5
:10757000284616220BF022F807B0F0BD40F698021C
:107580009A42D8DB094B1868CDF81100EFE740F6B6
:10759000FC02CEE7843E01004C9FFF1F783E0100B5
:1075A000743E01003B773B98676666667C3E01004F
:1075B000E89EFF1FF8B5174C174E2278174D337809
:1075C0002F888E46003218BF012201467046FFF711
:1075D00017FB002398423370237015DB14BF012082
:1075E00000202B889F420ED040F23A72A3F5AF7371
:1075F0000B490C4C02FB03F381FB0312DB17A3EBDB
:10760000621332332360F8BD0749012218460A701D
:107610002270E6E71C8BFF1F11A0FF1FB49FFF1F06
:10762000B5814E1B108AFF1F9CA0FF1F014B1878CD
:1076300002F00CBC84A0FF1F014B187802F020BCA4
:10764000D891FF1F134BB3F9003030B583EAE374D0
:10765000A4EBE374002BA0B218DB012300E0134677
:1076600003EB830252009442F9DA0B4D90FBF3F2E4
:1076700085FB03E403FB1200DB173032D3EBA403DA
:1076800080B201F8012BF1D10B7030BD2D230B70AE
:107690000131E2E7D891FF1F67666666144BB3F9C4
:1076A000003070B583EAE375A5EBE375002BACB24F
:1076B0001ADB012300E0034603EB83004000854210
:1076C000F9DA0C4E94FBF3F086FB03E503FB104460
:1076D000DB173030D3EBA503A4B201F8010BF1D1D5
:1076E00005480B70106070BD2D230B700131E0E771
:1076F000209DFF1F676666669C3E0100134BB3F931
:10770000003030B583EAE374A4EBE374002BA0B23D
:1077100018DB012300E0134603EB8302520094427E
:10772000F9DA0B4D90FBF3F285FB03E403FB120047
:10773000DB173032D3EBA40380B201F8012BF1D177
:107740000B7030BD2D230B700131E2E7CC89FF1F98
:1077500067666666134BB3F9003030B583EAE374AD
:10776000A4EBE374002BA0B218DB012300E0134666
:1077700003EB830252009442F9DA0B4D90FBF3F2D3
:1077800085FB03E403FB1200DB173032D3EBA403C9
:1077900080B201F8012BF1D10B7030BD2D230B709D
:1077A0000131E2E76C9DFF1F67666666134BB3F914
:1077B000003030B583EAE374A4EBE374002BA0B28D
:1077C00018DB012300E0134603EB830252009442CE
:1077D000F9DA0B4D90FBF3F285FB03E403FB120097
:1077E000DB173032D3EBA40380B201F8012BF1D1C7
:1077F0000B7030BD2D230B700131E2E78A9DFF1F16
:1078000067666666134BB3F9003030B583EAE374FC
:10781000A4EBE374002BA0B218DB012300E01346B5
:1078200003EB830252009442F9DA0B4D90FBF3F222
:1078300085FB03E403FB1200DB173032D3EBA40318
:1078400080B201F8012BF1D10B7030BD2D230B70EC
:107850000131E2E78E9FFF1F67666666134BB3F93F
:10786000003030B583EAE374A4EBE374002BA0B2DC
:1078700018DB012300E0134603EB8302520094421D
:10788000F9DA0B4D90FBF3F285FB03E403FB1200E6
:10789000DB173032D3EBA40380B201F8012BF1D116
:1078A0000B7030BD2D230B700131E2E76489FF1F9F
:1078B00067666666134BB3F9003030B583EAE3744C
:1078C000A4EBE374002BA0B218DB012300E0134605
:1078D00003EB830252009442F9DA0B4D90FBF3F272
:1078E00085FB03E403FB1200DB173032D3EBA40368
:1078F00080B201F8012BF1D10B7030BD2D230B703C
:107900000131E2E72089FF1F67666666134BB3F912
:10791000003030B583EAE374A4EBE374002BA0B22B
:1079200018DB012300E0134603EB8302520094426C
:10793000F9DA0B4D90FBF3F285FB03E403FB120035
:10794000DB173032D3EBA40380B201F8012BF1D165
:107950000B7030BD2D230B700131E2E7208AFF1F31
:1079600067666666134BB3F9003030B583EAE3749B
:10797000A4EBE374002BA0B218DB012300E0134654
:1079800003EB830252009442F9DA0B4D90FBF3F2C1
:1079900085FB03E403FB1200DB173032D3EBA403B7
:1079A00080B201F8012BF1D10B7030BD2D230B708B
:1079B0000131E2E76C8AFF1F67666666134BB3F915
:1079C000003030B583EAE374A4EBE374002BA0B27B
:1079D00018DB012300E0134603EB830252009442BC
:1079E000F9DA0B4D90FBF3F285FB03E403FB120085
:1079F000DB173032D3EBA40380B201F8012BF1D1B5
:107A00000B7030BD2D230B700131E2E75C89FF1F45
:107A10006766666608B5B82002F09AFA044B1988C2
:107A2000884204D0B820BDE8084002F077BA08BD0B
:107A3000289DFF1F08B5702002F08AFA044B1988B0
:107A4000884204D07020BDE8084002F067BA08BD43
:107A5000E89EFF1F08B5742002F07AFA044B1988DB
:107A6000884204D07420BDE8084002F057BA08BD2F
:107A70007C9FFF1F054B1B880846042213B904494D
:107A80000AF09CBD03490AF099BD00BF6E9DFF1F1F
:107A9000A43E0100A03E01000E4B1B88032B17D80B
:107AA000DFE803F0110C0702084604220A490AF035
:107AB00085BD0846042209490AF080BD0846042213
:107AC00007490AF07BBD0846042206490AF076BD44
:107AD000704700BFF69EFF1FB43E0100B03E01009C
:107AE000AC3E0100A83E010010B40A4B0A4C0A4605
:107AF00093E8030083B0238802AC04E9030004EB9D
:107B00008303104653F8081C052203B010BC0AF08A
:107B100055BD00BF54360100589FFF1F30B40A4BBB
:107B20000A4D0C4693E8070084B02B8804AD05E9A4
:107B3000070005EB8303204653F80C1C042204B015
:107B400030BC0AF03BBD00BF5C360100E89EFF1F61
:107B5000F0B40C4D0C4F0E460FCD8CB001AC0FC4E1
:107B60000FCD0FC495E807003B8884E807000CAAF6
:107B700002EB8303304653F82C1C04220CB0F0BCFB
:107B80000AF01CBD683601003C9FFF1F30B50A4B50
:107B90000A4D0C460FCB85B00DF1100E0EE90F000B
:107BA0002B880EEB8303204653F8101C042205B0EB
:107BB000BDE830400AF002BDA43601005A9FFF1F05
:107BC00030B50A4B0A4D0C460FCB85B00DF1100EA7
:107BD0000EE90F002B880EEB8303204653F8101C90
:107BE000042205B0BDE830400AF0E8BCA43601002C
:107BF000EC9EFF1FF0B40B4D0B4F0E460FCD86B021
:107C00006C460FC495E803003B8884E8030006AA8D
:107C100002EB8303304653F8181C042206B0F0BC74
:107C20000AF0CCBCB4360100F69DFF1FF0B40A4D3B
:107C30000A4F0E460FCD86B001AC0FC42A683B88B0
:107C4000226006AA02EB8303304653F8141C0C2270
:107C500006B0F0BC0AF0B2BCCC360100709DFF1F2C
:107C6000F0B40B4D0B4F0E460FCD88B06C460FC4D1
:107C700095E80F0084E80F003B8808AA02EB830315
:107C8000304653F8201C042208B0F0BC0AF096BC21
:107C9000E03601007C9FFF1F164B1B880BB31BB205
:107CA00083EAE370A0EBE370002B30B584B21DDBF8
:107CB000012300E0134603EB830252009042F9DAFD
:107CC0000D4894FBF3F280FB03E503FB1244DB1742
:107CD0003032D3EBA503A4B201F8012BF1D10B7024
:107CE00030BD0846042205490AF068BC2D230B70FC
:107CF0000131DDE7B89DFF1F67666666B83E01008B
:107D0000F0B40A4D0A4F0E460FCD86B001AC0FC439
:107D10002A683B88226006AA02EB8303304653F8A8
:107D2000141C042206B0F0BC0AF048BC0037010065
:107D3000149DFF1F054B1B881BB9054B1868086075
:107D400070470846042203490AF038BCD09DFF1F43
:107D5000483E0100443E0100164B1B880BB31BB28A
:107D600030B583EAE374A4EBE374002BA0B21CDB10
:107D7000012300E0134603EB830252009442F9DA38
:107D80000D4D90FBF3F285FB03E403FB1200DB17C0
:107D90003032D3EBA40380B201F8012BF1D10B7088
:107DA00030BD064B1868086070472D230B700131F9
:107DB000DEE700BF609DFF1F67666666483E010004
:107DC000164B1B880BB31BB230B583EAE374A4EBEC
:107DD000E374002BA0B21CDB012300E0134603EB8D
:107DE000830252009442F9DA0D4D90FBF3F285FBC9
:107DF00003E403FB1200DB173032D3EBA40380B2A1
:107E000001F8012BF1D10B7030BD064B18680860EA
:107E100070472D230B700131DEE700BF289DFF1F47
:107E200067666666483E0100164B1B880BB31BB2A3
:107E300030B583EAE374A4EBE374002BA0B21CDB3F
:107E4000012300E0134603EB830252009442F9DA67
:107E50000D4D90FBF3F285FB03E403FB1200DB17EF
:107E60003032D3EBA40380B201F8012BF1D10B70B7
:107E700030BD064B1868086070472D230B70013128
:107E8000DEE700BF4A9FFF1F67666666483E010047
:107E9000164B1B880BB31BB230B583EAE374A4EB1B
:107EA000E374002BA0B21CDB012300E0134603EBBC
:107EB000830252009442F9DA0D4D90FBF3F285FBF8
:107EC00003E403FB1200DB173032D3EBA40380B2D0
:107ED00001F8012BF1D10B7030BD064B186808601A
:107EE00070472D230B700131DEE700BF2C9DFF1F73
:107EF00067666666BC3E0100174B1B881BB31BB24E
:107F000070B583EAE375A5EBE375002BACB21EDB1D
:107F1000012300E0034603EB830040008542F9DAC9
:107F20000E4E94FBF3F086FB03E503FB1044DB17D6
:107F30003030D3EBA503A4B201F8010BF1D108480E
:107F40000B70106070BD074B1868086070472D23D8
:107F50000B700131DCE700BFD89DFF1F67666666C6
:107F6000C03E0100483E0100164B1B880BB31BB2FC
:107F700030B583EAE374A4EBE374002BA0B21CDBFE
:107F8000012300E0134603EB830252009442F9DA26
:107F90000D4D90FBF3F285FB03E403FB1200DB17AE
:107FA0003032D3EBA40380B201F8012BF1D10B7076
:107FB00030BD064B1868086070472D230B700131E7
:107FC000DEE700BFC89FFF1F67666666483E010088
:107FD000164B1B880BB31BB230B583EAE374A4EBDA
:107FE000E374002BA0B21CDB012300E0134603EB7B
:107FF000830252009442F9DA0D4D90FBF3F285FBB7
:1080000003E403FB1200DB173032D3EBA40380B28E
:1080100001F8012BF1D10B7030BD064B18680860D8
:1080200070472D230B700131DEE700BF989FFF1FC3
:1080300067666666483E0100164B1B880BB31BB291
:1080400030B583EAE374A4EBE374002BA0B21CDB2D
:10805000012300E0134603EB830252009442F9DA55
:108060000D4D90FBF3F285FB03E403FB1200DB17DD
:108070003032D3EBA40380B201F8012BF1D10B70A5
:1080800030BD064B1868086070472D230B70013116
:10809000DEE700BFC49FFF1F67666666483E0100BB
:1080A000174B1B881BB31BB270B583EAE375A5EBB6
:1080B000E375002BACB21EDB012300E0034603EBAB
:1080C000830040008542F9DA0E4E94FBF3F086FB04
:1080D00003E503FB1044DB173030D3EBA503A4B258
:1080E00001F8010BF1D108480B70106070BD074B0F
:1080F0001868086070472D230B700131DCE700BF62
:10810000969FFF1F67666666C03E0100483E0100FD
:10811000054B1B881BB1054B186808607047044B62
:1081200018680860704700BFC69DFF1FD43E01005D
:10813000D03E010070B5FAF77BF8164B1B7813B1EF
:10814000154C237833B9154B1020198801F0E6FE41
:10815000012070BD124D134E2B783288B3FA83F391
:1081600082F008025B09114642202B70328001F038
:10817000D5FE23780BB12B782BB90021212006F0F6
:10818000FBF9002070BD0121212006F0F5F9002047
:1081900070BD00BF2E9DFF1FEE9EFF1F089FFF1F9B
:1081A000069FFF1FBC9FFF1F184B1A8852B3184A27
:1081B000128830B50A80B3F90030002B83EAE374EB
:1081C000A4EBE374BCBF2D238B70A0B2ACBF023113
:1081D0000331012300E0134603EB83025200944273
:1081E000F9DA0C4D90FBF3F285FB03E403FB12007C
:1081F000DB173032D3EBA40380B201F8012BF1D1AD
:108200000B7030BD044B1868086070477A9DFF1FE3
:10821000D83E010067666666483E010070B53C4D79
:108220002B780646002B35D11C4673780BB92046B7
:1082300070BDF9F7FDFF374A374B3848127831786F
:108240001B78007802EB43034A1E03EB80030E2ADF
:10825000EDD801A050F822F0C1820000E3820000B6
:108260002F820000C18200002F8200002F820000B8
:108270002F820000AF8200002F8200002F820000BA
:108280002F8200002F8200002F8200002F8200002A
:10829000AB820000AE21224803F0D0FF204804F05A
:1082A0001DFA00232B700124BFE706F08BFEAF21DF
:1082B0001B4803F0C3FF1B4A012313702B70B6E762
:1082C00083B91948038804294FF6FF7103F1FF327F
:1082D0000CBF01230B46134403F07F0301330380DB
:1082E0000FE073B1013B114A32F813304BB10E4E1F
:1082F0000F481049104A33800123002606700B7086
:108300001370084A0221012311702B70204670BDA2
:108310001C8BFF1F9D9FFF1F9E9FFF1F9F9FFF1F87
:1083200024A0FF1F9CA0FF1F889FFF1FC89EFF1F48
:10833000B09DFF1F349DFF1F9FA0FF1F10B5064B70
:10834000064C1A882046012101F0D6FD21884220E2
:10835000BDE8104001F0E2BD909DFF1FBC9FFF1FD4
:1083600010B5064B064C1A882046022101F0C4FDC8
:1083700021884220BDE8104001F0D0BDDA9DFF1FEA
:10838000BC9FFF1F10B5064B064C1A8820460421DF
:1083900001F0B2FD21884220BDE8104001F0BEBDD1
:1083A000FE9EFF1FBC9FFF1F10B5064B064C1A8890
:1083B0002046002101F0A0FD21884220BDE81040A8
:1083C00001F0ACBD469FFF1FBC9FFF1F08B51220E8
:1083D00001F0BEFD054B1988884206D0122001F03D
:1083E0009DFDBDE8084001F063BC08BD3C9FFF1F38
:1083F00008B5582001F0ACFD054B1988884206D01D
:10840000582001F08BFDBDE8084001F051BC08BDCB
:108410004A9FFF1F08B5142001F09AFD054B1988EB
:10842000884206D0142001F079FDBDE8084001F033
:108430003FBC08BDE29DFF1FF0B480EAE075A5EBEC
:10844000E0750028ACB21FDB1DBF2B230B704E1C48
:108450000E46012300E0134603EB830252009542CF
:10846000F9DA0B4F94FBF3F287FB030503FB12448D
:10847000DB173032D3EBA503A4B206F8012BF1D100
:1084800033700846F0BC70472D230B704E1CE0E79C
:1084900067666666084B188828B10D2807D00D3826
:1084A00000B2FFF7C9BF054A106808607047044A68
:1084B00010680860704700BFF69FFF1F483E01002C
:1084C000DC3E01001A4B18880C2815D0192817D04B
:1084D0001A2819D01B281BD01C281DD01D281FD0DE
:1084E0001E2821D01F2803D00C3800B2FFF7A4BFEC
:1084F000104A1068086070470F4A1068086070479B
:108500000E4A1068086070470D4A1068086070478E
:108510000C4A1068086070470B4A10680860704782
:108520000A4A106808607047094A10680860704776
:10853000869FFF1FFC3E0100E03E0100E43E01007B
:10854000E83E0100EC3E0100F03E0100F43E010077
:10855000F83E0100034B1888A0EB8000400000B2F9
:10856000FFF76ABF84A0FF1F024B1888643800B26F
:10857000FFF762BFE09FFF1F024B1888643800B20C
:10858000FFF75ABFA09DFF1F024B1888033800B2A7
:10859000FFF752BF5E9FFF1F024B18880C3800B2D6
:1085A000FFF74ABF269DFF1F024B1888183800B2FC
:1085B000FFF742BF5C9DFF1F024B1888183800B2BE
:1085C000FFF73ABF5A9DFF1F024B1888183800B2B8
:1085D000FFF732BF9A9FFF1FC3681888183800B290
:1085E000FFF72ABF054B1B881BB9054B18680860AD
:1085F000704708460422034909F0E0BF689FFF1F47
:10860000483E0100443E0100054B1B881BB9054B49
:1086100018680860704708460422034909F0CEBF75
:10862000629DFF1F483E0100443E010030B5134CDF
:1086300085B001252B463C2202212046009503F0FF
:1086400073FE204604F04AF8002240218023204691
:108650000191009311460A4B029504F0EDFC20466F
:1086600004F048F907480849084A0023036083805A
:108670000B608B801360938005B030BD24A0FF1F7A
:10868000B039010004A0FF1F1CA0FF1F8CA0FF1F1A
:1086900010B500EBC00000F10F02D2B293B284B06B
:1086A0009C1E981C3D2303918DE819003921024836
:1086B00004F026FC04B010BD24A0FF1F014B0122D2
:1086C0001A70704711A0FF1FF0B5784B784C794FA6
:1086D000794E7A4D85B004228DE80C000293204635
:1086E000774B4022802103F027FC2046754A7649CB
:1086F000764C09F0CBF8764B76489F61764FDF6178
:10870000764FB761764FF761764FAF61764FEF6185
:10871000764FA761764FE761764F87617649774F4D
:10872000C761774F8F61774A774FCF61774F9761F6
:10873000774B784FD761784F9F61784E784FDF61E4
:10874000784FB761784D794FF761794F794CAF61C8
:10875000794FEF61794F7A48A7617A4FE7617A4F95
:108760007A4987617A4FC7617A4F7B4A8F617B4F25
:10877000CF617B4F7B4B97617B4FD7617B4F7C4EAB
:108780009F617C4FDF617C4F7C4DB7617C4FF7610F
:108790007C4FAF617C4C7D4FEF617D4FA7617D4881
:1087A0007D4FE7617D4F87617D497E4FC7617E4F79
:1087B0008F617E4A7E4FCF617E4F97617E4B7F4FA8
:1087C000D7617F4F9F617F4E7F4FDF617F4FB761E2
:1087D0007F4D804FF761804FAF61804C804FEF61DC
:1087E000804FA7618048814FE761814F8761814950
:1087F000814FC761814F824A8F61824FCF61824F23
:10880000824B9761824FD761824F834E9F61834F26
:10881000DF61834F834DB761834FF761834F844C92
:10882000AF61844FEF61844F8448A761844FE76153
:10883000844F85498761854FC761854F8F61854A20
:10884000854FCF61854F9761854B864FD761864FA6
:108850009F61864E864FDF61864F874DB761874F98
:10886000F761874F874CAF61874F88488849EF6130
:10887000884F894DA761E561884F894D894CDFF8A4
:1088800048E2894A894B8761C5618C61884E894F6E
:10889000894D8A4CC1F81CE089488A499761D561A5
:1088A0009C61D861B16005B0F0BD00BF40420F00CF
:1088B00024A0FF1F99850000D88FFF1F248FFF1F62
:1088C000F491FF1F1C89FF1F91BF0000A48CFF1FA4
:1088D0000C8EFF1FFC8FFF1FC970000089850000F0
:1088E000D57000007D7300003D830000A57300007B
:1088F00061830000CD730000C48DFF1F85830000DD
:10890000E97A0000108DFF1FE5700000F57300008C
:10891000E88DFF1FA9830000798500008491FF1F67
:10892000F5700000698500006091FF1F057100006F
:10893000C17D0000A08DFF1F157A00005585000045
:108940007C8DFF1F2D76000045760000B48FFF1F41
:10895000397600001D7B0000388CFF1F357A00003F
:10896000517B00006890FF1FCD830000297E00002E
:10897000EC8CFF1FF18300009D760000F88BFF1F39
:10898000157100001D740000F890FF1F1584000091
:10899000917E0000C88CFF1F25710000F97E000049
:1089A000548EFF1F35710000697F0000808CFF1F0F
:1089B00045710000FD760000B08BFF1F557100006F
:1089C0008D7B0000B090FF1F65710000557700009F
:1089D0006C8FFF1F75710000C17B00008C8BFF1F27
:1089E00085710000AD770000308EFF1F957100008B
:1089F000F57B0000D48AFF1FA571000005780000F8
:108A0000348DFF1FB5710000A9810000908FFF1FFA
:108A1000C57100002D7C0000B491FF1FD5710000CE
:108A2000D17F0000008FFF1FE5710000398000003A
:108A3000688BFF1FF5710000617C00008C90FF1FA8
:108A4000557A0000A1800000488FFF1F05720000CA
:108A5000C5840000448BFF1F15720000997C000044
:108A6000208BFF1F25720000017D00008C8AFF1FF4
:108A70003572000095840000588DFF1F457200007C
:108A80005D7800005C8CFF1F55720000F88AFF1FA4
:108A9000D48BFF1FB5780000657200000D790000CF
:108AA00075720000657900002090FF1FB08AFF1FDB
:108AB000A891FF1FBD790000957200001181000090
:108AC000A57200008D90000085720000F0B5461C74
:108AD00083B00D460127032336B22AB2044631463D
:108AE0008DE888002348ADB204F0A0F90C23AA1C3D
:108AF00012B200930197052321B21E4804F096F9A3
:108B00001D4A1E4B12881B68BA422AD023D3022A60
:108B100010D11B4CA3F6CA0384FB03241C44DB17AF
:108B2000C3EB24140A2CA8BF0A2424EAE474A2B2DA
:108B300023B202E000231A461C460D35AA1A012072
:108B40000093019012B2314603230A4804F0ECF876
:108B5000204603B0F0BD0B4CA3F6FC0384FB0324BA
:108B6000DDE7094CA3F6980384FB0324DB17C3EB72
:108B7000A404D7E724A0FF1FE89EFF1F4C9FFF1F00
:108B800009CB3D8D1F85EB51398EE3382DE9F0433C
:108B90008FB283B0DFF84C80BD1D461D2DB204B2EC
:108BA00036B24FF001090AB22346314640460095DD
:108BB000CDF8049004F0EAF82A46334621464046B0
:108BC0008DE8200204F0E2F807F10C02009533462C
:108BD00012B22146CDF80490404604F0D7F803B015
:108BE000BDE8F08324A0FF1F2DE9F043804685B047
:108BF000002956D10121304804F05EFC2F4998F835
:108C0000062098F8083011F80290994522DA4FEAC8
:108C100089064D460C24D8F80C3027489B595F68CC
:108C200022B2002104F044FC384609F009FC394620
:108C30000246214804F0D6FD1F4804F0E9FD98F8EB
:108C4000083001350934AB42A4B206F1040601DD57
:108C5000422CE0D1B9F1000F13D109F10609994571
:108C60000CDA3C2301213B220391029300930192F1
:108C700039233F223A21104804F042F905B0BDE8FB
:108C8000F0830F2301213B22039102930093019271
:108C900039230C223A21084804F032F998F80830B8
:108CA000DBE700213423009301913F230C2202488B
:108CB00004F03AF89EE700BF24A0FF1F1CA0FF1F8E
:108CC00010B5104C0121204604F0FCFB2046012188
:108CD00004F0F2FB20463422552104F0E9FB204643
:108CE0000222094904F07EFD20460522074904F0CE
:108CF00079FD204604F08CFD2046BDE8104003F0CD
:108D0000F9BD00BF24A0FF1F483F01004C3F0100F8
:108D100070B50D46064609F093FB00EB4000840059
:108D2000002D36D0284609F08BFB00EB40004000B8
:108D300023185B1003F16001091A282209B21748B1
:108D4000C3F1600404F0B4FB0121144804F0B4FB47
:108D5000284609F075FB29460246104804F042FDFA
:108D60000E4804F055FD02210C4804F0A5FB21B289
:108D700021220A4804F09CFB304609F061FB314691
:108D80000246064804F02EFD0448BDE8704004F099
:108D90003FBD6410C4F16004E5E700BF24A0FF1FDD
:108DA00010B50D4B1B5C51F82340237884B013B1F0
:108DB000012004B010BD04AA01A942F8103D2046CC
:108DC000A3699847A38A9B07F2D401A80099FFF7EB
:108DD0009FFF012004B010BD04A0FF1F2DE9F04F3C
:108DE0002F4DDFF8CCB0DFF8C4A0DFF8C8900FCD6E
:108DF00091B003AC0FC40FCD0FC40FCD0FC42B68BF
:108E000023600025A8462F462E4600E09846BAF873
:108E1000003024495BF8232028461123F7F7E2FCB1
:108E200000EBC00400EB840089FB00340444C0174D
:108E3000C0EB6434C4F13C00C6F13C0207F14101CF
:108E4000012600B208F1410300901BB2019612B254
:108E500009B2154803F09AFF08EB060305F2111555
:108E60003C2B2646ADB24746D0D134226B210E486A
:108E700004F01EFB00210C4804F01EFB0B4B1B886A
:108E800010AA02EB830353F8344C204609F0D8FAB9
:108E900002460548214611B0BDE8F04F04F0A2BCDF
:108EA000143701008030010024A0FF1F469DFF1FE2
:108EB000E42E010009000280234B70B5B3F90030A5
:108EC00083EAE374A4EBE374002B82B0A1B234DB39
:108ED00068466D46012300E0134603EB830252000F
:108EE0009442F9DA194E91FBF3F286FB03E403FB9B
:108EF0001211DB173032D3EBA40389B205F8012B32
:108F0000F1D119462B70FFF703FF114B1B7813B1FA
:108F1000104B1B780BB902B070BD01210E4804F054
:108F2000CBFA332264210C4804F0C2FA04220B4924
:108F3000094804F057FC02B070BD2D238DF80030B5
:108F40000DF101056846C5E7089FFF1F6766666665
:108F5000EE9EFF1F069FFF1F24A0FF1F543F01002E
:108F600010B5424C424882B003F0B8FB2378C3B935
:108F700006213F4804F0A0FA2378012B37D90A22B2
:108F8000022B11463A486BD004F092FA3949032279
:108F9000374804F027FC364802B0BDE8104004F022
:108FA00037BC354B1A7801210523002A35D10191B0
:108FB000009311462E4803F039FF304B1A78002AEF
:108FC00036D0052301220192009300220A2128486D
:108FD00003F0AAFE2A4B1A78002A35D10121052375
:108FE000019100931421224803F020FFC0E7254C93
:108FF0002388092B32D9632B8CBF0A211F210A2217
:109000001B4804F055FA2188194804F051FC18480F
:1090100002B0BDE8104004F0FBBB002201910093B8
:109020001146134803F080FE144B1A78002AC8D169
:1090300005230121019100930A210D4803F0F6FE5A
:109040000F4B1A78002AC9D0012205230192009300
:1090500000221421064803F067FE89E73021CEE79D
:1090600004F026FA0322084992E700BF9FA0FF1FE1
:1090700024A0FF1F603F01009D9FFF1F9E9FFF1FB9
:109080009F9FFF1F889FFF1F5C3F0100F8B56D4D3C
:10909000287840B96C4B1B6899425CD36B4A01231A
:1090A00013702B70F8BD0C4600266948664F03F01C
:1090B00015FB04F6AC53324665483B6031212E70F7
:1090C00004F0F6F901216248624D04F0FBF93146E3
:1090D0005F4804F0F1F905225F495D4804F082FB26
:1090E0005B4804F095FB0C221021594804F0E0F98C
:1090F0000B225A49564804F075FB0522584954483A
:1091000004F070FB524804F083FB564B50481C6837
:10911000A4F69803C3EB031385FB03251D4410211C
:10912000DB172022C3EB652504F0C2F940F6CC33EF
:109130009C4205F124054FF022014FF004000BDCA6
:10914000FFF7C4FC484B1C88064674B3012C46D07C
:10915000022C41D00120F8BDFFF718FD0922434938
:109160003B4804F03FFB2A221021394804F0A0F9C3
:109170003F4C374884FB0534EB17C3EBA40421466E
:1091800004F096FB01223B49314804F02BFB04EB31
:109190008401A5EB41012E4804F08AFB01223649E7
:1091A0002B4804F01FFB0120F8BD34491022284849
:1091B00004F018FB264804F02BFB2A221021244837
:1091C00004F076F93146224804F072FB07222C495C
:1091D0001F4804F007FBCBE70C222A49E7E70C22E3
:1091E00029491B4804F0FEFA194804F011FB2A2211
:1091F0001021174804F05CF9314615481C4E04F064
:1092000057FB07221E49124804F0ECFA86FB05368C
:10921000EB17C3EBA60631460D4804F049FB224686
:1092200014490B4804F0DEFA06EB8601A5EB410178
:10923000074804F03DFB22460F49054804F0D2FAE6
:109240002046F8BD1C8BFF1F18A0FF1F9CA0FF1F0E
:1092500024A0FF1F3B773B98643F01006C3F010057
:109260004C3F01004C9FFF1FE89EFF1F783F01000D
:10927000676666666C470100DC460100843F0100BA
:10928000983F0100B03F0100A03F01002DE9F041EF
:10929000754C2278002A05460F4614BF4FF001088E
:1092A0004FF000084ED1714E3368CB1AB3F5FA6F08
:1092B00004D86B78A3B94046BDE8F0816C4B6D488B
:1092C0006D49DFF8D0E11A7001230370098823701B
:1092D00026208EF8002000F021FE6B78002BEAD0CB
:1092E0003760F8F7A5FF654A654B6649127828781C
:1092F0001B78097802EB4303421E03EB81030E2A1D
:10930000D9D801A151F822F0F9930000C5930000CB
:10931000B7920000F9930000B7920000B7920000E6
:10932000B7920000AD930000B79200005F93000079
:10933000B7920000B7920000B7920000B792000009
:109340005B930000AF215048484E02F077FFFFF7D3
:1093500007FE002337602370ABE705F033FE4A4871
:1093600003F0BCF90221484804F0A6F80F2223219B
:10937000454804F09DF805224449434804F032FA78
:10938000414804F045FA1E2223213F4804F090F89A
:1093900005223F493C4804F025FA3B4804F038FADE
:1093A000394803F0A7FA00F0D3FC84E7394D2B7855
:1093B000012B50D9304B2620198800F0AFFD002337
:1093C0002B7078E7002B3FF476AF013B324A32F83E
:1093D0001330002B3FF46FAF274C304825492D4AFE
:1093E00023804FF001080023037081F8008082F889
:1093F0000080FFF7B5FD5EE793B1013B264A32F8E6
:10940000131019B31C4B254D1A4C224A1980002603
:10941000012326202E702370137000F07FFD15E0CD
:10942000154C1E4922880B7004284FF6FF7002F17C
:10943000FF310CBF012202460A440E4E154D02F0C8
:109440007F0201320121228031702B70FFF788FDED
:109450004FF001082FE70649064A01230020087053
:1094600013702370A6E700BF1C8BFF1F98A0FF1F7F
:109470009CA0FF1F349DFF1F889FFF1F9D9FFF1F04
:109480009E9FFF1F9F9FFF1F24A0FF1FC03F010043
:10949000C83F01009FA0FF1FC89EFF1FB09DFF1F78
:1094A0002DE9F04F05468BB00F46AD480121164619
:1094B00004F008F8AA8812F0010440F0B080DFF848
:1094C000CC8298F80030002B7DD1AB79A54AD15CD5
:1094D000A1B9DFF8BCA279781AF8039041B33978C2
:1094E0000139072900F2B780DFE811F0F1005401DB
:1094F000B5006C01B500B500B500E9007C78002C22
:1095000000F0CA800139EC68387854F82170FC68A2
:10951000411EB4F80080072900F2A780DFE811F0AF
:1095200074015901A5006C01A500A500A5009F00CC
:10953000DFF854A2DAF80020B21AB2F5967F75D996
:10954000894A107801281ABF012010701170874ACB
:1095500018BF0146D05CC0EB0900C0B2FFF798F815
:109560000124CAF80060AB889B0770D57B78002B7C
:109570006DD0F8F75DFE7E4B7E4A7F481B781278EF
:1095800039780078022515FB02330A2903EB8003A2
:1095900000F04E810C295AD1002B58D003F119004C
:1095A000764E774A013B0021400080B226F8131026
:1095B0000123157088F8003000F0B0FC714B0322D5
:1095C00020461A702FE0664803F088F801216448AD
:1095D00003F072FF62482246214603F069FFAB8820
:1095E000580725D42C68204608F02AFF2146024659
:1095F0005B4804F0F7F85A4804F00AF909220123FD
:109600008DE80C0000217F23554803F0BFFB0021AB
:109610002846FFF7E9FA002388F8003055E7AB68E1
:109620003146384698470BB0BDE8F08F0846FAE758
:109630002B6804A8984704A808F002FF04A9024672
:10964000474804F0CFF8464804F0E2F8D6E7204651
:109650000BB0BDE8F08F00240AF8039083E70021E7
:10966000D1543846FB699847FC68A4F8008000276D
:1096700025223C238DE8840041211822384803F03C
:1096800053FBE968A879FFF78BFB374A3E4B17700D
:109690001E600BB0BDE8F08F3B490A68B21AB2F504
:1096A000967FD4D9304F0E603E78012E00F0B48002
:1096B000E968184601233B70FFF772FBB3E7304AB5
:1096C000E9791170012288F800200024C4E72A7A81
:1096D000013A4A45BFDD09F10104E4B2A145BAD01F
:1096E000224E16F803B0CBEB0900C0B20021FEF702
:1096F000CFFF2B7A052BD9461BD9CBEB0402042ACA
:1097000040F3AE80A4F1040BBBF1000FC0F2B080B7
:10971000063B5B45A8BF5B465FFA83F9AA7913480D
:10972000B15C994205D000F8029001212846FFF76C
:109730005BFAC9EB0400C0B201210B4EFEF7A8FF93
:1097400000213423019100930548317040230B22FE
:109750003F21A14603F0E8FA0124AB797CE700BF82
:1097600024A0FF1F8CA0FF1F9DA0FF1F1CA0FF1F98
:109770009D9FFF1F9E9FFF1F9F9FFF1FC89EFF1F54
:109780009CA0FF1F9FA0FF1F88A0FF1F1C8BFF1F17
:1097900004A0FF1F0FFA89F1E868604C50F82160BF
:1097A0002168049134785E4904980860002C71D0D7
:1097B000012C7FF450AF5B4A317A88F80040117079
:1097C000002449E7B9F1000F50D009F1FF34E4B2A9
:1097D00084E7B98A01F0040189B200293FF440AF5F
:1097E0003B6A03929847039A00283FF43DAFAB7958
:1097F000FC680021D15438E77B8A43453CD908F105
:1098000001081FFA88F830E73B8A43453BD208F14C
:10981000FF381FFA88F828E725238DE8180042480A
:109820003C703C231822412103F07EFA3046FAE6D0
:10983000002B3FF40CAF3D4A3D4E1188394A03F1ED
:109840001900013B400080B226F81310012388F86C
:109850000030157000F062FB364B20461D70E2E6CA
:10986000002A3FF755AF04F1FF3B4DE74C46F3E6C6
:109870004FF000094B4651E7BB8ADA077FF5F5AE9A
:10988000B7F81080F1E6BB8AD9077FF5EEAEB7F8DE
:109890001280EAE62849C85CC0EB090009F1010E14
:1098A000C0B201214FF0340B02F803E0FEF7F0FEE6
:1098B000B6681D48019440230B223F210124CDF8B6
:1098C00000B003F031FA40230B223F211648CDF8B7
:1098D00000B0019403F0AAFA2146134803F0ECFD0E
:1098E000304608F0ADFDA0EB800000F15F0109B249
:1098F0000F220D4803F0DCFD304608F0A1FD314693
:109900000246094803F06EFF074803F081FFE9684B
:10991000A879FFF745FAAB799EE600BFDCA0FF1FF0
:1099200088A0FF1F9CA0FF1F24A0FF1F889FFF1F70
:10993000C89EFF1F9FA0FF1F1CA0FF1F2DE9F0471F
:10994000DFF808926D4B99F800601B68DFF800A201
:1099500082B0003601934FF0030018BF0126019F2B
:109960009AF8008004F00EFE0546042004F00AFE7A
:109970000446052004F006FE800040EA4404062068
:1099800004F000FE2C4364B25D4944EAC0000A784A
:1099900080F00F03DBB29A425A4A3CD01760002293
:1099A00059480B7003788DF800808DF8012053B36F
:1099B000564A12684EF66021BA1A8A4219D8022B0A
:1099C00059D0012B5FD0062B48D0032B63D0042B3A
:1099D00069D0052B77D0072B7DD0082B00F0838032
:1099E000092B68D016B14A4802F084FF02B0BDE8E6
:1099F000F087484A484C002301212370037013600C
:109A0000938089F800103A4669464448FFF748FDBC
:109A10003043C6B2E6E71268BA1A1E2A6BD99AF822
:109A20000020934222D0394C3D488AF80030012B67
:109A3000276082EA030207609846B1D0042BAFD1B9
:109A400037480068381AB0F5C87FA9D9354C206866
:109A5000381A3228A4D927601A46A1E73A4669463F
:109A60003148FFF71DFD3043C6B2BBE7012B4FF075
:109A70000002E3D1E4E73A4669462C48FFF710FDBF
:109A80003043C6B2AEE73A4669462948FFF708FDBB
:109A90003043C6B2A6E73A4669462648FFF700FDBE
:109AA0003043C6B29EE73A4669462348FFF7F8FCC2
:109AB0003043C6B296E73A4669462048FFF7F0FCC5
:109AC0003043C6B28EE73A4669461D48FFF7E8FCC8
:109AD0003043C6B286E73A4669461A48FFF7E0FCCB
:109AE0003043C6B27EE73A4669461748FFF7D8FCCE
:109AF0003043C6B276E7002252E700BFDCA0FF1F6A
:109B0000A0A0FF1F0CA0FF1F9CA0FF1F94A0FF1F81
:109B100024A0FF1F8CA0FF1F9EA0FF1F8039010003
:109B2000A4A0FF1F14A0FF1FB03D0100D838010002
:109B3000DC370100783701002C460100CC370100EA
:109B400034380100BC380100A891FF1F1C8BFF1F97
:109B500010A0FF1F28B11028044BA8BF10201860C8
:109B60007047024B01201860704700BFA8A0FF1F7C
:109B700008B5002006F010F90028FAD108BD00BF92
:109B800010B504464FF4406005F01AF805F072F87D
:109B90000A4B1B7833B96CB1102C094BA8BF1024A9
:109BA0001C6010BD4FF4C05004F0E0FD04F014FF41
:109BB000002CF1D1024B01241C6010BDEE9EFF1F52
:109BC000A8A0FF1F70B50D461446064605F048F8DC
:109BD000284605F045F8204605F042F8084B1B786A
:109BE00013B1084B1B7803B970BD304604F09CFEDE
:109BF000284604F099FE2046BDE8704004F094BE6B
:109C0000EE9EFF1F069FFF1F38B5164D2B780446AA
:109C100041F6FF72A0F50050824203F1FF33A8BF66
:109C200002461B0202F5005203F47063100443F471
:109C3000604343F00E0300F4FE005204184302F0A8
:109C4000FE42104305F0DEFF2868013860F01F0077
:109C5000C4F3C61204F07F01C0B2BDE83840FFF77C
:109C6000B1BF00BFA8A0FF1F70B5104E3378013BF5
:109C70001B0203F47063044643F4304308062204D5
:109C800000F0FE4043F00B03034302F4FE001843D0
:109C90000D4605F0B7FF3068013860F04F002A46E6
:109CA0002146C0B2BDE87040FFF78CBFA8A0FF1FDF
:109CB00008B564210720FFF7D7FF7F210B20BDE8FF
:109CC0000840FFF7D1BF00BF70B5104E3378013B9D
:109CD0001B0203F47063044643F410430806220495
:109CE00000F0FE4043F00903034302F4FE00184372
:109CF0000D4605F087FF3068013860F06F002A4696
:109D00002146C0B2BDE87040FFF75CBFA8A0FF1FAE
:109D100038B50E4D2B78013B1B0203F470630446EB
:109D200043F41043000443F0090300F4FE00184319
:109D300005F068FF2868013860F06F002146C0B266
:109D40000022BDE83840FFF73DBF00BFA8A0FF1FBD
:109D500010B500217B20FFF787FF0024E0B2FFF75A
:109D6000D7FF0134022004F043FC802CF6D110BD53
:109D700038B50C46054604F073FF204604F070FF2A
:109D8000074B1B7813B1074B1B7803B938BD284626
:109D900004F0CAFD2046BDE8384004F0C5BD00BF50
:109DA000EE9EFF1F069FFF1F38B50D4D2B78013B20
:109DB0001B0203F47063044643F45043000443F071
:109DC0000D0300F4FE00184305F01CFF286801385D
:109DD00060F02F002146C0B2BDE83840FFF7C8BF91
:109DE000A8A0FF1F38B50E4D2B78013B01381B0290
:109DF000C4B203F47063200443F4404343F00C0303
:109E000000F4FE00184305F0FDFE2868013860F0FC
:109E10003F002146C0B2BDE83840FFF7A9BF00BFF0
:109E2000A8A0FF1F38B504460D46F02004F018FF27
:109E300035B1254414F8010B04F012FFAC42F9D1FE
:109E4000F720BDE8384004F00BBF00BF00B50B4B56
:109E500083B00246998818680090032AADF8041070
:109E600002D903B05DF804FB684606218DF8052091
:109E7000FFF7D8FF03B05DF804FB00BF9C4601006C
:109E800000B50B4B024683B0186899880090131FE9
:109E90004C2BADF8041002D903B05DF804FB684602
:109EA00006218DF80520FFF7BDFF03B05DF804FB28
:109EB000A4460100030203F4FE43C0F3C610184396
:109EC000704700BF03784078DB0103F47E5300F055
:109ED0007F001843704700BF82B002AA114642F8C3
:109EE000040D002012F8013B03F07F03914243EA86
:109EF0000020F7D102B07047003210B403884FF051
:109F0000010404FA01F418BF012202FA01F123EA64
:109F100004020A43028010BC704700BF70B5CEB285
:109F20000C46054603F0F6FE864203D0314628462D
:109F300003F00AFF0135284603F0ECFE240A8442B0
:109F400005D021462846BDE8704003F0FDBE70BD37
:109F500038B5054603F0DEFE4FF0000460F3070459
:109F6000681C03F0D7FE60F30F24A0B238BD00BF19
:109F7000F8B504460020FFF7EBFF002C00F0D18578
:109F80004FF4AF610220FFF7C9FF4FF47A6104205C
:109F9000FFF7C4FF4FF496610620FFF7BFFF4FF4B1
:109FA000FA610820FFF7BAFF4FF4FA610A20FFF7C1
:109FB000B5FF40F6B8310C20FFF7B0FF4FF42F612A
:109FC0002220FFF7ABFF40F6AC512420FFF7A6FF9D
:109FD0007D212A20FFF7A2FF0C210E20FFF79EFF14
:109FE00001211020FFF79AFF02211220FFF796FFB0
:109FF00000211420FFF792FF00211620FFF78EFFAB
:10A0000002211820FFF78AFF01211A20FFF786FF9F
:10A0100001211C20FFF782FF04211E20FFF77EFF95
:10A0200014212020FFF77AFF01212620FFF776FF79
:10A0300003212820FFF772FF04212C20FFF76EFF79
:10A0400014212E20FFF76AFF00213020FFF766FF62
:10A050000C213220FFF762FF00213420FFF75EFF62
:10A0600000213620FFF75AFF00213820FFF756FF66
:10A0700000213A20FFF752FF00213C20FFF74EFF5E
:10A0800000213E20FFF74AFF00214020FFF746FF56
:10A0900000214220FFF742FF1F214420FFF73EFF2F
:10A0A00013214620FFF73AFF0E214820FFF736FF25
:10A0B00011214A20FFF732FF0A214C20FFF72EFF23
:10A0C00000214E20FFF72AFF06215020FFF726FF30
:10A0D00002215220FFF722FF0C215420FFF71EFF20
:10A0E00000215620FFF71AFF00215820FFF716FF26
:10A0F00001215A20FFF712FF08215C20FFF70EFF15
:10A100000A215E20FFF70AFF00216020FFF706FF0B
:10A1100004216220FFF702FF01216420FFF7FEFE09
:10A1200000216620FFF7FAFE0B216820FFF7F6FEFC
:10A130007F216A20FFF7F2FE00216C20FFF7EEFE80
:10A1400000216E20FFF7EAFE00217020FFF7E6FEF7
:10A1500000217220FFF7E2FE00217420FFF7DEFEEF
:10A160001F217620FFF7DAFE13217820FFF7D6FEB5
:10A170000E217A20FFF7D2FE11217C20FFF7CEFEC0
:10A180000A217E20FFF7CAFE1F218020FFF7C6FEAE
:10A1900013218220FFF7C2FE0E218420FFF7BEFEAE
:10A1A00011218620FFF7BAFE0A218820FFF7B6FEAC
:10A1B00000218A20FFF7B2FE00218C20FFF7AEFEBF
:10A1C00000219620FFF7AAFE00219820FFF7A6FEA7
:10A1D00000219A20FFF7A2FE05219C20FFF79EFE9A
:10A1E00006219E20FFF79AFE0021A020FFF796FE91
:10A1F0007F21A220FFF792FE40F2A461A420FFF786
:10A200008DFE4FF4E161A620FFF788FE0021A82013
:10A21000FFF784FE0021AA20FFF780FE0221AC2078
:10A22000FFF77CFE0121AE20FFF778FE0121B02070
:10A23000FFF774FE0B21B220FFF770FE6421B420FB
:10A24000FFF76CFE6421B620FFF768FE0321B820FB
:10A25000FFF764FE2C210020FFF760FE0220FFF7CD
:10A2600077FEB0F5805F034680F03486D24A042042
:10A270001380FFF76DFEB0F5805F034680F0218606
:10A28000CE4A06201380FFF763FEA0F52F739BB222
:10A29000B3F57A6F024606D940F628210620FFF76B
:10A2A0003DFE40F62822C64B08201A80FFF750FEDC
:10A2B000A0F52F739BB2B3F57A6F024606D940F62C
:10A2C000E4410820FFF72AFE40F6E442BD4B0A2095
:10A2D0001A80FFF73DFEA0F5FA739BB240F6AC5131
:10A2E0008B42024606D94FF4FA610A20FFF716FEA8
:10A2F0004FF4FA62B44B0C201A80FFF729FEA0F548
:10A30000FA739BB240F6AC518B42024606D940F636
:10A31000B8310C20FFF702FE40F6B832AB4B0E20EE
:10A320001A80FFF715FE1828034600F2C385A84AD5
:10A3300010201380FFF70CFE431E9BB20F2B02462A
:10A3400004D901211020FFF7E9FD0122A14B1220C1
:10A350001A80FFF7FDFD0A28034600F2A4859E4AF5
:10A3600014201380FFF7F4FD0128034604D90021CF
:10A370001420FFF7D3FD0023984A16201380FFF71F
:10A38000E7FD7F28034600F28785954A1820138051
:10A39000FFF7DEFD0528034600F27785914A1A2073
:10A3A0001380FFF7D5FD0C28034600F267858E4A1F
:10A3B0001C201380FFF7CCFD0428034600F25785CC
:10A3C0008A4A1E201380FFF7C3FD0928034600F2C6
:10A3D0004785874A20201380FFF7BAFD46280346A9
:10A3E00000F23785834A22201380FFF7B1FDA0F5E4
:10A3F000FA739BB240F6AC518B42024606D94FF439
:10A400002F612220FFF78AFD4FF42F627A4B242020
:10A410001A80FFF79DFDA0F5FA739BB240F6AC548D
:10A42000A342024604D921462420FFF777FD2246A5
:10A43000724B26201A80FFF78BFD7F28034600F21F
:10A4400001856F4A28201380FFF782FD0628034606
:10A4500000F2F1846B4A2A201380FFF779FDA0F106
:10A4600032039BB2B3F5967F024604D97D212A20A0
:10A47000FFF754FD7D22644B2C201A80FFF768FD06
:10A480000C28034600F2D084604A2E201380FFF788
:10A490005FFD1E28034600F2C0845D4A3020138011
:10A4A000FFF756FD0928034600F2B084594A3220CE
:10A4B0001380FFF74DFD1F28034600F2A084564A83
:10A4C00034201380FFF744FD7F28034600F2908478
:10A4D000524C36202380FFF73BFD7F28034600F2D5
:10A4E000808438206380FFF733FD7F28034600F225
:10A4F00071843A20A380FFF72BFD7F28034600F2EA
:10A5000062843C20E380FFF723FD7F28034600F2AE
:10A5100053843E202381FFF71BFD7F28034600F272
:10A52000448440206381FFF713FD7F28034600F237
:10A5300035844220A381FFF70BFD394D288044204C
:10A54000FFF706FD3028034600F2FD83354A46201A
:10A550001380FFF7FDFC3028034600F2EE83324CF7
:10A5600048202380FFF7F4FC3028034600F2DF8305
:10A570004A206380FFF7ECFC3028034600F2D183C9
:10A580004C20A380FFF7E4FC3028034600F2C3838D
:10A590004E20E380FFF7DCFC0128034604D90021AC
:10A5A0004E20FFF7BBFC0023204A50201380FFF70A
:10A5B000CFFC431E3CE000BFF09DFF1FBA9FFF1F72
:10A5C000929DFF1F849FFF1F509FFF1F589DFF1FDD
:10A5D000269DFF1F089FFF1F3C9FFF1FE29DFF1F3F
:10A5E0002C9DFF1FF69DFF1F7A9DFF1F709DFF1F73
:10A5F000609DFF1F969FFF1F049FFF1F009FFF1F6F
:10A60000889FFF1F5E9FFF1FB49FFF1F469DFF1F78
:10A61000D89DFF1FC89FFF1F869FFF1FC89EFF1F5B
:10A62000BC9FFF1F9A9FFF1F609FFF1F6E9DFF1F14
:10A630009BB20B2B024604D906215020FFF76EFC7B
:10A640000622CF4B52201A80FFF782FC04280346D3
:10A6500000F25B83CB4A54201380FFF779FC431E42
:10A660009BB21D2B024604D90C215420FFF756FC47
:10A670000C22C54B56201A80FFF76AFC01280346BE
:10A6800004D900215620FFF749FC0023BF4A582077
:10A690001380FFF75DFC7F28034600F23083BC4A3D
:10A6A0005A201380FFF754FC431E9BB2092B02462D
:10A6B00004D901215A20FFF731FC0122B54B5C205F
:10A6C0001A80FFF745FC431E9BB2102B024604D9AB
:10A6D00008215C20FFF722FC0822AF4B5E201A8085
:10A6E000FFF736FC431E9BB21D2B024604D90A21FC
:10A6F0005E20FFF713FC0A22A84B60201A80FFF7A8
:10A7000027FC0228034600F2F482A54A6420138045
:10A71000FFF71EFC0128034604D901216420FFF73E
:10A72000FDFB01239F4A62201380FFF711FCC31E2B
:10A730009BB2012B024604D904216220FFF7EEFBF5
:10A740000422994B66201A80FFF702FC7F280346FB
:10A7500000F2C982954A68201380FFF7F9FB7F2831
:10A76000034600F2BA82924A6A201380FFF7F0FB98
:10A770007F28034600F2AB828E4A6C201380FFF7DD
:10A78000E7FB0428034600F29C828B4A6E2013806C
:10A79000FFF7DEFB1928034600F28D82874A7020FE
:10A7A0001380FFF7D5FB0228034600F27E82844A1D
:10A7B00072201380FFF7CCFB0628034600F26F825D
:10A7C000804A74201380FFF7C3FB0728034600F27A
:10A7D00060827D4A8A201380FFF7BAFB0A2803466D
:10A7E00000F25182794A8C201380FFF7B1FB0428D4
:10A7F000034600F24282764A98201380FFF7A8FBB6
:10A800000128034604D900219820FFF787FB002385
:10A81000704A9A201380FFF79BFB0128034604D956
:10A8200000219A20FFF77AFB00236B4A96201380C1
:10A83000FFF78EFB0B28034600F21982674A9C2023
:10A840001380FFF785FB831E9BB2032B024604D9BE
:10A8500005219C20FFF762FB0522614B76201A80C0
:10A86000FFF776FB3028034600F2FB815D4A782033
:10A870001380FFF76DFB3028034600F2EC815A4C41
:10A880007A202380FFF764FB3028034600F2DD8145
:10A890007C206380FFF75CFB3028034600F2CF8109
:10A8A0007E20A380FFF754FB3028034600F2C181CD
:10A8B0008020E380FFF74CFB3028034600F2B38191
:10A8C0004A4A82201380FFF743FB3028034600F2F8
:10A8D000A481474C84202380FFF73AFB30280346AD
:10A8E00000F2958186206380FFF732FB3028034613
:10A8F00000F287818820A380FFF72AFB30280346D7
:10A9000000F27981A020E380FFF722FB01280346B3
:10A9100004D90021A020FFF701FB0023354A9E2027
:10A920001380FFF715FBC31E9BB20C2B024604D904
:10A9300006219E20FFF7F2FA06222F4BA2201A8052
:10A94000FFF706FB431E9BB27E2B024604D97F21F4
:10A95000A220FFF7E3FA7F22284BA4201A80FFF7FA
:10A96000F7FAA0F5AF639BB2B3F5167F024647D95D
:10A9700040F2A461A420FFF7D1FA40F2A4623FE0C4
:10A980002089FF1F6489FF1F208AFF1FC69DFF1FAC
:10A990004A9FFF1F209DFF1F6C8AFF1F5C89FF1FBE
:10A9A000FC9EFF1F589FFF1F809DFF1F989FFF1F4A
:10A9B000B89DFF1F649DFF1F149DFF1FF69FFF1F83
:10A9C000E89EFF1FC49FFF1F7C9FFF1F0A9FFF1F62
:10A9D000F69EFF1F629DFF1FD09DFF1F449FFF1F1C
:10A9E000B09FFF1F5A9DFF1FD89EFF1F5C9DFF1F3A
:10A9F000E09EFF1F689FFF1FCC89FF1F8E9FFF1FD8
:10AA0000D44BA6201A80FFF7A3FAA0F5AF639BB240
:10AA1000B3F5167F024606D94FF4E161A620FFF791
:10AA20007DFA4FF4E162CC4BA8201A80FFF790FA30
:10AA30000628034600F2D980C84AAA201380FFF7EF
:10AA400087FA0328034600F2CA80C54AAC20138067
:10AA5000FFF77EFA0328034600F2BB80C14AB0200C
:10AA60001380FFF775FA0328034600F2AC80BE4A54
:10AA7000AE201380FFF76CFA7F28034600F29D801A
:10AA8000BA4AB2201380FFF763FA7F28034600F228
:10AA90008E80B74AB4201380FFF75AFA431E9BB248
:10AAA000C62B024604D96421B420FFF737FA64228A
:10AAB000B04BB6201A80FFF74BFA431E9BB2C62B51
:10AAC000024604D96421B620FFF728FA6422AA4B73
:10AAD000B8201A80FFF73CFA082862D82B88DFF8E4
:10AAE000B8E2A64FA64AA74DA74EA84CA84903F026
:10AAF000010CAEF800C0C3F3400EA7F800E0C3F3AA
:10AB000080071780C3F3C007A24A2F70C3F3001752
:10AB1000C3F34015C3F38013378025800B8010806A
:10AB2000F8BD4FF6FF7398423FF42AAA2C283FF451
:10AB300095AB17287FF624AA19287FF68DAA1B2823
:10AB40007FF6AAAA1C283FF4BFAA1E287FF6C4AA33
:10AB50001F283FF4C9AA20283FF4E2AA21283FF485
:10AB6000EBAA22283FF4F0AA23283FF4F9AA2428CC
:10AB70003FF42AAB25283FF42FAB26283FF430AB17
:10AB800027283FF435AB28283FF440AB29283FF471
:10AB900045AB2A283FF452AB2B287FF45BABFFF781
:10ABA00055BBB8200321FFF7B9F9032096E70B2125
:10ABB000B220FFF7B3F90B236BE70121AE20FFF7BB
:10ABC000ADF901235CE70121B020FFF7A7F90123CC
:10ABD0004DE70221AC20FFF7A1F902233EE7002157
:10ABE000AA20FFF79BF900232FE70021A820FFF7F9
:10ABF00095F9002320E70A218820FFF78FF90A231F
:10AC000080E611218620FFF789F9112372E60E21D3
:10AC10008420FFF783F90E2364E613218220FFF7D7
:10AC20007DF9132355E61F218020FFF777F91F23B5
:10AC300046E60A217E20FFF771F90A2338E6112142
:10AC40007C20FFF76BF911232AE60E217A20FFF70B
:10AC500065F90E231CE613217820FFF75FF9132313
:10AC60000DE61F217620FFF759F91F23FEE500218D
:10AC70009620FFF753F90023E0E500218C20FFF731
:10AC80004DF90023B7E500218A20FFF747F900239B
:10AC9000A8E500217420FFF741F9002399E5002180
:10ACA0007220FFF73BF900238AE500217020FFF7AF
:10ACB00035F900237BE500216E20FFF72FF90023F3
:10ACC0006CE500216C20FFF729F900235DE57F2169
:10ACD0006A20FFF723F97F234EE50B216820FFF759
:10ACE0001DF90B233FE500216620FFF717F900232C
:10ACF00030E500216020FFF711F9002305E5002170
:10AD00005820FFF70BF90023C9E402215220FFF776
:10AD100005F902239EE40A214C20FFF7FFF80A23DD
:10AD200036E411214A20FFF7F9F8112328E40E2117
:10AD30004820FFF7F3F80E231AE413214620FFF70B
:10AD4000EDF813230BE41F214420FFF7E7F81F233E
:10AD5000FFF7FCBBF49DFF1F709FFF1F229DFF1F8D
:10AD6000989DFF1F5A9FFF1FEC9EFF1F6C9DFF1FAA
:10AD70008A9DFF1FA09DFF1FE09FFF1F909DFF1F4B
:10AD8000DA9DFF1F069FFF1FFE9EFF1F5C9FFF1F98
:10AD90000E9FFF1F289DFF1F469FFF1F0021402081
:10ADA000FFF7BCF80023FFF7C4BB00213E20FFF7EC
:10ADB000B5F80023FFF7B5BB00213C20FFF7AEF844
:10ADC0000023FFF7A6BB00213A20FFF7A7F80023D6
:10ADD000FFF797BB00213820FFF7A0F80023FFF70B
:10ADE00088BB00213620FFF799F80023FFF779BBD5
:10ADF00000213420FFF792F80023FFF769BB0C21F4
:10AE00003220FFF78BF80C23FFF759BB00213020CD
:10AE1000FFF784F80023FFF749BB14212E20FFF72A
:10AE20007DF81423FFF739BB04212C20FFF776F8B7
:10AE30000423FFF729BB03212820FFF76FF8032322
:10AE4000FFF708BB01212620FFF768F80123FFF771
:10AE5000F8BA14212020FFF761F81423FFF7C2BAD3
:10AE600004211E20FFF75AF80423FFF7B2BA01218C
:10AE70001C20FFF753F80123FFF7A2BA01211A2083
:10AE8000FFF74CF80123FFF792BA02211820FFF7D1
:10AE900045F80223FFF782BA00211620FFF73EF89B
:10AEA0000023FFF772BA02211220FFF737F80223BE
:10AEB000FFF755BA0C210E20FFF730F80C23FFF7EF
:10AEC00036BA4FF47A610420FFF728F84FF47A631A
:10AED000FFF7D6B94FF4AF610220FFF71FF84FF428
:10AEE000AF63FFF7C3B900BFF8B5CB2006F008FD8C
:10AEF000204B214A054603CB1368C5F803001A0C02
:10AF0000BA20C5F807102B80AA70FEF7D3FF2E4693
:10AF1000002426F80B0FA0B2FFF71AF8FEF7CAFFBD
:10AF20000234BA2C26F8020FF5D16C1E05F1C606C4
:10AF30004FF0FF3014F8013F082758400F4B40F303
:10AF400000017A1E0B4012F0FF0783EA5000F5D192
:10AF5000B442EFD1C043FEF7BFFF3A46C5F8C70081
:10AF6000CB21284604F09CFE2846BDE8F84006F0B8
:10AF7000CFBC00BFB0460100AC4601002083B8ED55
:10AF8000F0B50E4B0E4C054693E8070085B02468DB
:10AF90002E88AD7801AB83E80700270C1846002205
:10AFA0000B21ADF804408DF80670ADF80C608DF8FB
:10AFB0000E5004F075FE05B0F0BD00BFBC460100A8
:10AFC000AC460100F0B5124B124D1E68124F0FCD6A
:10AFD00087B06C460FC495E8030044F8040B38684A
:10AFE0003B79CDF80D00320C2C2021808DF8022009
:10AFF0008DF81130ADF80060FEF75CFF0022ADF86F
:10B000000B001221684604F04BFE07B0F0BD00BFF4
:10B01000AC460100C84601004C3F0100002004F08E
:10B02000BBBE00BF02F02EBE70B5124C82B0002530
:10B03000402306462946204600930195802320227E
:10B0400001F072FE20222946204602F031FA204605
:10B05000012102F037FA304607F0F2F93146024694
:10B06000204602F0BFFB204602B0BDE8704001F070
:10B0700041BC00BF24A0FF1FF0B5CA2983B075D919
:10B080000546441E00F1C6064FF0FF3014F8012FAC
:10B0900008275040404A40F300017B1E0A4013F04D
:10B0A000FF0782EA5000F5D1B442EFD1C043FEF76A
:10B0B00013FF0146D5F8C7000190019A914202D0D2
:10B0C000B2F17F2F0BD105F10B00FEF7FBFEBA2882
:10B0D0000BD03248FFF7A8FF002003B0F0BD304886
:10B0E000FFF7A2FF384603B0F0BD05F10D00FEF7F3
:10B0F000E9FE2C2840D1002440F6AC5613E0042889
:10B100001AD0062821D008281FD00A2828D00C28B9
:10B1100022D1A1F5FA7292B2B24201D8FEF7FEFE38
:10B120000234BA2C0ED004F10D002844FEF7CAFEFA
:10B13000022C0146A0B2E2D1B1F5805FEED3023419
:10B14000BA2CF0D1012003B0F0BDA1F52F7292B25C
:10B15000B2F57A6FE4D8E1E7222801D0242811D192
:10B16000A1F5FA7292B2B242DAD8D7E70D48FFF7EA
:10B170005BFF002003B0F0BD0B48FFF755FF002038
:10B1800003B0F0BD2A28C9D1A1F1320292B2B2F5C2
:10B19000967FC5D8C2E700BF2083B8ED0C470100F9
:10B1A000F8460100E04601002047010003290CD9C0
:10B1B00070B5461C82B005460C46304603222A492B
:10B1C00007F0ACF910B102B070BD70470B2C05D977
:10B1D00005222649281D07F0A1F940B12448FFF7B0
:10B1E00023FF244802B0BDE87040FFF7C9BE05F157
:10B1F0000901032201A807F0E1F901A803221E4971
:10B2000007F08CF9D8B103221C4901A807F086F990
:10B2100008B301A803221A4907F080F9B0B9194808
:10B22000FFF702FFA11E89B23046FFF725FF002875
:10B23000C9D0154802B0BDE87040FFF7F5BE13480D
:10B24000FFF7F2FEFFF750FE1148F3E71148FFF752
:10B25000EBFE1148C6E71148FFF7E6FE02B0BDE875
:10B260007040FFF7AFBE00BFAC4601003847010099
:10B270004047010054470100584701008047010042
:10B28000984701009C470100B04701005C4701005E
:10B2900070470100C4470100D847010084470100FE
:10B2A0002DE9F043174D2B6883B081460F46904639
:10B2B000F3B1154E34880A1992B2184611463280FD
:10B2C00006F09CFE28603A464946204402F06CFD98
:10B2D000B8F1000F09D031882868FFF767FF2868A8
:10B2E00006F016FB00232B60338003B0BDE8F0832B
:10B2F000054E01930846318006F002FB019B286051
:10B300001C46E0E7B0A0FF1FACA0FF1F10B51F4C0C
:10B310004FF4FA70FBF75AFD204601F0DFF90022E6
:10B320001146204602F0C4F82046012102F0CAF876
:10B330002046002102F0C0F80B221549204602F0F9
:10B3400051FA204602F064FA0F221249204602F018
:10B3500049FA204602F05CFA0F490722204602F023
:10B3600041FA204602F054FA204601F0C3FA0B4B92
:10B370000B4A1A604FF4FA70FBF728FDFFF722FE24
:10B380000848BDE81040FFF74FBE00BF24A0FF1FD4
:10B39000DC470100E8470100F8470100E4A2FF1F75
:10B3A000A1B20000004801000020704790F8392049
:10B3B00090F83800101A704790F8383090F839201B
:10B3C0009A4205D95A1C034480F83820187E7047E9
:10B3D0004FF0FF30704700BF90F8383090F83920B8
:10B3E0009A4286BF1B18187E4FF0FF30704700BF8F
:10B3F000704700BF38B50546B0F85E0090B195F8CB
:10B400005D301446C3F1210294420CD805F13B0093
:10B410001844224602F0C8FC95F85D30234485F8B4
:10B420005D30204638BD012014462871EEE700BF8C
:10B43000B0F85E306BB190F85D30202B07D8C218A1
:10B44000013380F85D30012082F83B107047012302
:10B4500003710020704700BF0023426980F8383034
:10B4600080F8393080F85C3080F85D3080F85E30EC
:10B4700080F85F3006CA30B40D68046943662A4319
:10B4800083660A60A370426990F8613016491468B7
:10B4900013441D7A5B7B01EBC5051B026D6803F449
:10B4A000E06343F064032B6090F8623013449D7CAA
:10B4B000DB7D01EBC5011B02496803F4E06343F047
:10B4C00064030B6021685368194205D00369272281
:10B4D0005A70036904229A71036920225A71036920
:10B4E00080229A7030BC70473453010043690CCB02
:10B4F00012681A420CD0094B99420AD9084B99425A
:10B50000036994BF1A220D225A70036904229A71AA
:10B510007047036927225A70F7E700BF7F1A0600B9
:10B520003F420F0010B50269D378DBB2D90604465A
:10B530003DD510215806D17038D503F0040303F02F
:10B54000FF02002B51D03D49626E00230B7084F83E
:10B550005D30002A5BD0904794F85D30002B56D0C8
:10B560002369D0229A70236994F83B201A712369C9
:10B57000012284F85C200222DA7010BD304B84F87E
:10B5800060009C424AD02F4B9C4252D094F8391014
:10B5900013791F29DBB207D82848007820B160183A
:10B5A000013184F8391003760223D37010BD590697
:10B5B000C3D4917801F0100101F0FF000029DDD023
:10B5C00013F001031ED194F85C1094F85D008842DA
:10B5D00081BF4B1C091984F85C3091F83B30137122
:10B5E0002369D0229A702269DEE7236984F8392022
:10B5F000C0229A702369114A19790121117002221F
:10B60000DA7010BDC023937022691379CCE7012250
:10B61000002384F85D2084F83B30A1E7626994F848
:10B620006130094913440322187A02F043FD22696C
:10B63000ACE7626994F861300449F3E7B4A0FF1FF6
:10B64000F491FF1F6092FF1FADB60000B9B6000075
:10B650000369DB7803F0200373B190F860300133A5
:10B66000DBB2012B80F860301AD9426990F8613062
:10B670001344187A02F09ABD70B5426903F0FF05D1
:10B6800090F8613013440446187A02F08FFDA36EDF
:10B690005BB184F8385094F83900BDE87040184721
:10B6A00090F85F30002BE0D0704770BD0148FFF785
:10B6B000CFBF00BFF491FF1F0148FFF7C9BF00BF14
:10B6C0006092FF1F2DE9F047374FDFF8E0903B68AD
:10B6D000026982B006460093DDF800800021A025B3
:10B6E000D3789B065BD53B680193019BC8EB0303B2
:10B6F0000F2BF5D949B1102BF2D00020907033698F
:10B7000080229A7002B0BDE8F087726996F86130C5
:10B7100013440521187A02F043FF726996F86130EC
:10B720001344012193F812A0504602F039FF092476
:10B730000021504602F020FF2B46013BFDD10121A4
:10B74000504602F019FF2B46013BFDD1013CEFD1E1
:10B75000706996F8611001444FF4A0720C7A4B7B2B
:10B7600009EBC4011B02496803F4E06343F064037E
:10B770000B6096F862300344997CDB7D09EBC101D4
:10B780001B02496803F4E06343F064030B60013A71
:10B79000FDD13269D3789B064FF00101A3D401207B
:10B7A00002B0BDE8F08700BFDCA0FF1F34530100EA
:10B7B000F0B503691222DA700269937803F020036E
:10B7C00085B004460D46002B5ED0B42393703C49EF
:10B7D00022690B680093009E05E00B680193019BB2
:10B7E0009B1B042B42D8D37803F0200303F0FF0007
:10B7F000002BF2D094F85D30002B31D04FF0000ECA
:10B800004FF0020C04EB0E0393F83B3013710B68FE
:10B810000393039F206907E09B060DD50B680293F5
:10B82000029BDB1B052B28D8C378DBB203F0020296
:10B8300002F0FF06002AEFD080F803C02669F378F3
:10B84000DBB2DF0632462DD49F062BD5DB0731D481
:10B850000EF1010E94F85D305FFA8EFE7345D1D87B
:10B8600000201DBB002384F85E3004E09070236943
:10B8700080229A70042005B0F0BD86702369802272
:10B8800004209A7005B0F0BD03F0FF06FFF71AFF21
:10B8900010B9042005B0F0BD236984F85F60B022C0
:10B8A0009A7094E78023B3700420DAE72669802336
:10B8B000B370D7E7BEF1000F0CBF02200320F6E7FC
:10B8C000DCA0FF1F2DE9F04106690025122780F852
:10B8D000385080F83950F770D0F810C09CF802E06A
:10B8E0000EF0200E88B00446884615461E46BEF16E
:10B8F000000F49D0B4238CF80230784B21691A68C4
:10B900000092DDF800E006E01A6801920198CEEBA3
:10B910000000042830D8C87800F0200000F0FF07AD
:10B920000028F1D04FEA480242F00102D2B20A7177
:10B930001A680292DDF808E0206906E01A680392AE
:10B940000399CEEB010105292AD8C17801F0020143
:10B9500001F0FF070029F1D04FF0020C80F803C07E
:10B960002269D17811F0110722D12DBB002E0CBF16
:10B97000A0238023937003E08F70236980229A7044
:10B98000384608B0BDE8F0810EF0FF07FFF79AFED9
:10B990000028F5D0236984F85F70B0229A70ACE774
:10B9A00087702369802238469A7008B0BDE8F0811C
:10B9B000802393700027E3E7012D75D0A0219170BB
:10B9C00021690A79BE4667464FF0A80C1A680492AE
:10B9D000049805E01A680592059A121A052A4AD8B1
:10B9E000CA7802F0020202F0FF08002AF2D0CF70FB
:10B9F0002169CA78D2B212F0100F08465AD19206C5
:10BA000058D5013DEDB2012D49D0BEF11F0F3BD9F4
:10BA10000A79012DDAD11A680692069D05E01A68A6
:10BA20000792079A521B052A46D8C27802F00202F2
:10BA300002F0FF01002AF2D00223C3702269D378FA
:10BA4000DBB2D9063AD49B0634D5B023BEF11F0F22
:10BA500093703FD8226904EB0E0312791A760EF127
:10BA6000010E5FFA8EFE16B1236980229A7084F867
:10BA700039E0774684E781F80280236980229A7052
:10BA8000774684F839E07BE704EB0E0291F80480F6
:10BA900082F818800EF1010E5FFA8EFEB9E781F888
:10BAA00002C021690846B0E7A82191702069BE460E
:10BAB0000279B0E7774663E78170DEE71021A023C3
:10BAC000D170013BFDD12269937803F0F7037746EB
:10BAD000937055E723691B79C5E700BFDCA0FF1F02
:10BAE0000148FFF71FBD00BFF491FF1F0148FFF79A
:10BAF00019BD00BF6092FF1F704700BF38B5144CDE
:10BB0000037801225B000546204684F83B3084F828
:10BB10005E2084F85D20FFF78BFC20460021FFF7B4
:10BB200047FE0B4C2978012320461A46FFF7CAFE30
:10BB30000128F6D194F8383094F839209A4205D982
:10BB4000E218013384F83830107E38BDFF2038BD4C
:10BB5000F491FF1F38B51B4C037801225B000546AA
:10BB6000204684F83B3084F85E2084F85D20FFF79F
:10BB70005FFC20460021FFF71BFE124C297820466F
:10BB800001230222FFF79EFE0228F6D194F8382006
:10BB900094F839108A420FD2531CDBB2A018994294
:10BBA00084F83830007E0AD9234402321B7E84F8A0
:10BBB000382040EA032038BD4FF6FF7038BD40F40E
:10BBC0007F4038BDF491FF1F0C2901D90020704738
:10BBD0000231490001F0FE01FFF7BCBF70B50C4C0B
:10BBE0000378164601255B00204684F83B3084F834
:10BBF0005E5084F85D50FFF71BFC31462046FFF78E
:10BC000017FC29462046BDE87040FFF7D1BD00BFB4
:10BC1000F491FF1FF8B505460F461646412421460C
:10BC20003A462846FFF7DAFF611C0234C9B23246B1
:10BC30002846E4B2FFF7D2FF592CF0D1F8BD00BF7F
:10BC400038B504460D463548FFF706FC63228021CF
:10BC500020462570FFF7C2FF012002F0C9FC2046F4
:10BC600000225E21FFF7BAFF20465D21FFF746FF65
:10BC7000242801D0002038BD204606220C21FFF7E1
:10BC8000C9FF204601222B21FFF7A8FF20460122F1
:10BC90002C21FFF7A3FF20460E222D21FFF79EFF48
:10BCA000204600222E21FFF799FF204601222F2156
:10BCB000FFF794FF204605223021FFF78FFF204633
:10BCC00001223121FFF78AFF204600223221FFF7AF
:10BCD00085FF204600223321FFF780FF2046002207
:10BCE0003421FFF77BFF204600223521FFF776FF46
:10BCF000204600225B21FFF771FF204610225C21C5
:10BD0000FFF76CFF204620225D21FFF767FF2046EA
:10BD10008F225E21FFF762FF012038BDF491FF1FE3
:10BD200010B4047F4160022CC26002D010BC01F04C
:10BD3000D7BB836810BC184790E80C00F0B41C68AF
:10BD400059682568164F174E29432160164D17492B
:10BD50001760D66015611160417A154A5C180A3186
:10BD600094F8244053F8215002EBC40149680D6057
:10BD7000017A5C1803EB8101247ECD6902EBC401DA
:10BD800049680D60817A581803EB810390F8300000
:10BD9000596B02EBC002F0BC53681960704700BFDA
:10BDA00001401F00011000380110007800001F80C2
:10BDB00034530100704700BFF0B50C1EBDF814608D
:10BDC00034DBB0F906701919B942C4BF3B1B1BB272
:10BDD000002BA6461CDD002A1146B8BFD11D02F07B
:10BDE0000705CC10826A012007FB04E1A840012E60
:10BDF0000A44C0B21ED00CD3022E09D1013B12FA64
:10BE000083F3013A12F8011F41409A421170F9D1AF
:10BE1000F0BDC043013B12FA83F3C0B2013A12F8FD
:10BE2000011F014093421170F9D1F0BD23441BB2B0
:10BE30000024C6E7013B12FA83F3013A12F8011F0E
:10BE400001439A421170F9D1F0BD00BFF8B50D1E43
:10BE50000EDB14461F46064601F03AFBA84207DDFA
:10BE6000002C05DB304601F037FBA04201DCF8BDB9
:10BE7000F8BD304601F02AFB022853D003284BD0EE
:10BE8000012806D16540F3886C406540013B5D1B8D
:10BE90002DB2012F03D02AD3022F14D0F8BD002CCD
:10BEA0002246B6F90630B06AB8BFE21D42F3CF02AF
:10BEB00002FB035504F00704435D012101FA04F479
:10BEC0001C434455F8BD002C2246B6F90630B06A32
:10BED000B8BFE21D42F3CF0202FB035504F0070492
:10BEE000435D012101FA04F45C404455F8BD002C87
:10BEF0002246B6F90630B06AB8BFE21D42F3CF025F
:10BF000002FB035504F00704435D012101FA04F428
:10BF100023EA04044455F8BD3389013B591B2546E7
:10BF20000CB2B6E7F18832890139013A4D1B141B76
:10BF30002DB224B2ADE700BF2DE9F041079E9DF977
:10BF40001880089D04461F4600F0C0FF0D4B0E48A8
:10BF50000E4984F83380FF22002F08BF1F4684F863
:10BF60002F20002384F8302084F8312084F83220F8
:10BF70002060A665E565676261652362A36220466D
:10BF8000BDE8F081F491FF1F8C48010001100138D9
:10BF900010B50446806A034B236008B105F0B8FC75
:10BFA000204610BD8C480100F8B5436ADBB190F81B
:10BFB0002C200125AA4083F83B2083F85E5083F8AB
:10BFC0005D500446406A03680E461B68002198478E
:10BFD000606A036831461B6898472946606ABDE875
:10BFE000F840FFF7E5BBC26BC56C1368046A23EA2F
:10BFF000050313604CB122684FF00043D3625163D4
:10C00000D36A002BFCDA936BF8BD836B466B082573
:10C01000802410E03768426C3A4332601F68826CBB
:10C020003A431A601A68876C013D22EA07024FEA18
:10C0300054041A6007D02142ECD13268476C22EADE
:10C0400007023260EAE7F8BD70B50446406A0D4663
:10C0500000282BD0A16DFFF749FA002D20460CBF18
:10C06000A621A721FFF7A0FF606A20B1E16DBDE81E
:10C070007040FFF73BBA216C226D0868236A0243C7
:10C080000A6093B1DA7A82B1D00703D5224A99695E
:10C090001160DA7A910703D5204AD9691160DA7AFA
:10C0A000520702D51E4A1B6A136070BD236A002B1B
:10C0B0002BD0D97A626DE1B172B6D97ACE0706D5A6
:10C0C0001848D9680668314099610160D97A8807B3
:10C0D00006D51548196906683140D9610160D97AD9
:10C0E0004E0705D51148596906683140196201604B
:10C0F00062B61B68D968914207D00D4818600D4997
:10C10000DA6042F0804018611960226C216D13687A
:10C1100023EA01031360A0E700E100E004E100E08E
:10C1200008E100E080E100E084E100E088E100E077
:10C1300001403F0000003F80436A2DE9F041054681
:10C140000E469046002B3ED090F82C100124A140C2
:10C1500083F83B1083F85E4083F85D40406A0368D3
:10C1600000211B6808F1FF379847FFB2B8F1000FB4
:10C1700023D03744A046013E686A16F8011F0368C1
:10C180001B6898470134B742E4B216D0202CF3D193
:10C190000121686AFFF70CFB95F82C206B6A5200AE
:10C1A00083F83B2083F85E8083F85D80686A0368CB
:10C1B00000211B6898470124DEE7686A0121BDE879
:10C1C000F041FFF7F5BAC26BC16C136823EA0103B3
:10C1D00006EB080413604FF00048A6420ED02B6A0D
:10C1E00016F801EB63B11A68C2F82C80C2F834E08B
:10C1F000D36A002BFCDAA642936BF0D1BDE8F08144
:10C20000AB6BD5F834C008208021DCF800206F6CBF
:10C210001EEA010F14BF3A43BA43CCF800201A6853
:10C22000AF6C3A431A601A68AF6C013822EA070211
:10C230004FEA51011A60E8D1CFE700BF70B504465C
:10C24000406A0D46002828D0A16DFFF74FF920461F
:10C250002946FFF7A9FE606A20B1E16DBDE8704094
:10C26000FFF744B9216C226D0868236A02430A6013
:10C2700093B1DA7A82B1D00703D5234A9969116064
:10C28000DA7A910703D5214AD9691160DA7A52071F
:10C2900002D51F4A1B6A136070BD236A002B2BD086
:10C2A000D97A626DE1B172B6D97ACE0706D519484E
:10C2B000D9680668314099610160D97A880706D546
:10C2C0001548196906683140D9610160D97A4E076D
:10C2D00005D512485969066831401962016062B695
:10C2E0001B68D968914207D00D4818600D49DA6083
:10C2F00042F0804018611960226C216D136823EAB6
:10C3000001031360A3E700BF00E100E004E100E0E7
:10C3100008E100E080E100E084E100E088E100E085
:10C3200001403F0000003F802DE9F041044686B007
:10C33000806A9DF830801E460F461546B4F90830D5
:10C34000002800F04281DA1D48BF03F10E02B4F963
:10C350000630D21003FB02F2002105F0FDFDB4F916
:10C360000820202A00F39280B4F90610A34B012084
:10C37000203A733902EBD27201EBD1714FF0200EEB
:10C38000029073208DE8014042F34F0241F34F01C8
:10C39000204600F051FE606A84F82D70002800F0FD
:10C3A0004D81002D40F08A80B4F90830202B14BF55
:10C3B0003D253C2584F82C50B8F1000F40F08580D5
:10C3C00006B394F93300002818DBC0B2012102F053
:10C3D000E7F8012194F8330002F0CEF8012002F0D2
:10C3E00007F9002194F8330002F0C6F80A2002F0A1
:10C3F000FFF8012194F8330002F0BEF8606A0028CB
:10C4000000F08280A16DFFF771F804227C4920467C
:10C41000FFF792FE217A0139C9B22046FFF7C4FD29
:10C42000784904222046FFF787FE94F92D30012B2E
:10C4300014BF142110212046FFF7B6FD04227249D3
:10C440002046FFF779FEB4F90630802B00F0928089
:10C45000602B00F0A680D9212046FFF7A5FD94F9B6
:10C460002D30012B14BFF12122212046FFF79CFD26
:10C47000204606226549FFF75FFE606A50B3E16D12
:10C48000FFF734F8012006B0BDE8F081B4F90610DA
:10C490005F4B0120403A52394FF0400E029002EBC0
:10C4A000D272522001EBD1718DE8014042F34F026C
:10C4B00041F34F01204600F0BFFD6CE76DB284F8F8
:10C4C0002C50B8F1000F3FF47BAFFEF7C5FF002EF4
:10C4D00094D076E7216C226D0868236A02430A60D3
:10C4E00073B1DA7A62B1D00703D54A4A996911600B
:10C4F000DA7A91077CD4520702D5474A1B6A136047
:10C50000012006B0BDE8F081236A002B2BD0D97A38
:10C51000626DE1B172B6D97ACF0706D53F48D968C6
:10C520000568294099610160D97A8E0706D53C4893
:10C53000196905682940D9610160D97A4D0705D587
:10C5400038485969056829401962016062B61B685C
:10C55000D968914207D0344818603449DA6042F013
:10C56000804018611960226C216D136823EA010371
:10C5700013604AE7B4F90830202B00F08680402B86
:10C580007FF469AF2A4920460322FFF7D5FD94F9CD
:10C590002D30012B14BFCF219F212046FFF704FD32
:10C5A00059E7B4F90830102B7FF455AF21492046E4
:10C5B0000322FFF7C1FD94F92D30012B14BFAF21E9
:10C5C00010212046FFF7F0FC45E7DA1D48BF03F1D4
:10C5D0000E02B4F90630D21003FB02F210460592A7
:10C5E00005F08EF9A06200283FF44DAF059AB3E63E
:10C5F000114AD9691160DA7A7DE700BFE448010089
:10C60000C44A0100C84A0100CC4A0100D04A0100D6
:10C61000D84A010000E100E008E100E080E100E02C
:10C6200084E100E088E100E001403F0000003F803D
:10C63000E0480100984D010004E100E0012194F878
:10C640003100244F01F0ACFF94F83200012101F0D9
:10C65000A7FF94F9312094F9323057F83220E26381
:10C6600057F83330206A23640125E56425651A688C
:10C670002A431A6078B1B8F1000F3FF428AFFFF7F2
:10C680005BFB002E3FF4BAAE9BE604221249204623
:10C69000FFF752FDDFE6294694F82F0001F080FFF6
:10C6A000294694F8300001F07BFF94F92F2094F98B
:10C6B000303057F83220626357F833306564A56430
:10C6C0001A68A36322F001021A60002E3FF496AEAE
:10C6D00077E600BF34530100DC480100B0F90820C0
:10C6E000D31D48BF02F10E03B0F90620806ADB10AB
:10C6F00002FB03F2002105F02FBC00BFF0B50029BA
:10C70000BDF814502EDBB0F90660B1422ADA002AD7
:10C7100059DBB0F9087014461C44BC42C4BFBB1AB4
:10C720001BB2002B1EDDD2B2D408D0F828E016FBD5
:10C73000041112F00702DBB20EEB010421D0C2F1AA
:10C740000807FAB2374F9342BF5C0CD2C3EB020C1E
:10C75000FF2646FA0CF6012D07EA06073FD005D35F
:10C76000022D36D0F0BD012D39D030D21EF8016037
:10C7700026EA07070EF801709342F3D3B0F90610CA
:10C780000C449A1AD2B2072A10D9022D36D0002DA5
:10C7900014BFFF26002613462670083BB0F906108A
:10C7A000DBB2072B0C44F7D802F00702002AD9D0DD
:10C7B0001D4B012D9B5C1DD017D3022DD2D12278A9
:10C7C00053402370F0BD13441BB20022A1E7022D99
:10C7D00025D11EF8016077400EF80170CCE71EF8F5
:10C7E000016037430EF80170C6E7227822EA03039E
:10C7F0002370F0BD227813432370F0BD11462378D7
:10C80000DB4323700839B0F90630C9B207291C444C
:10C81000F5D812F00702A5D0034B9B5CCFE7344458
:10C82000AFE700BF7C4801006C48010070B4C47DD4
:10C83000BDF80C50022C18D0032C1FD0012C0BD0AB
:10C84000002A03DBB0F90840944201DC70BC704759
:10C85000039570BCFFF7B0BAC4880395013CA41AD5
:10C860000A4621B270BCFFF749BF0689C488013E61
:10C87000641AB21AE41A12B221B2E1E704890395EC
:10C88000E41A641A114622B270BCFFF737BF00BF2A
:10C8900070B4C57DBDF80C60022D1AD0032D12D0E6
:10C8A000012D03D0039670BCFFF728BFC488E41A9B
:10C8B000A41A0A4621B2002A03DBB0F908409442C8
:10C8C00013DC70BC70470489013C641A114622B223
:10C8D000F1E7C48805890396013CAD1AED1A621A86
:10C8E00011B22AB270BCFFF709BF039670BCFFF704
:10C8F00063BA00BF2DE9F8430446406A002863D0BC
:10C90000A16DFEF7F3FD052274492046FFF714FCE4
:10C91000A1790139C9B22046FFF746FBB4F90820D6
:10C92000E588A66AD31D48BF02F10E03DB10626AD8
:10C9300015FB03F51FFA85F8002A7BD094F82C30FC
:10C940000125AB4082F83B3082F85E5082F85D50A2
:10C95000606A036840211B6808F1FF379847BFB23F
:10C96000B8F1000F23D03744A846013E606A16F89C
:10C97000011F03681B6898470135B742EDB216D016
:10C98000202DF3D10121606AFEF712FF94F82C20CC
:10C99000636A520083F83B2083F85E8083F85D80F1
:10C9A000606A036840211B6898470125DEE7012182
:10C9B000606AFEF7FDFE606A002800F08D80E16D80
:10C9C000BDE8F843FEF792BD236A002B2BD0D97A3D
:10C9D000626DE1B172B6D97ACE0706D54048D96802
:10C9E0000568294099610160D97A8D0706D53D48CF
:10C9F000196905682940D9610160D97A480705D5C8
:10CA000039485969056829401962016062B61B6896
:10CA1000D968914207D0354818603549DA6042F04C
:10CA2000804018611960226C216D136823EA0103AC
:10CA3000136068E7E26BE36C1168276A0B4306EB4F
:10CA4000080913604FF0004E4E450DD016F801CB8B
:10CA50002FB33A68C2F82CE0C2F834C0D36A002B76
:10CA6000FCDA4E45936BF1D1226C236D11680B43B8
:10CA7000136097B1FB7A83B1D90703D51D4BBA690F
:10CA80001A60FB7A9A0703D51B4BFA691A60FB7A86
:10CA90005B0702D5194B3A6A1A60BDE8F883A36BAD
:10CAA000D4F8348008208021D8F80020656C1CEA76
:10CAB000010F14BF2A43AA43C8F800201A68A56CC6
:10CAC0002A431A601A68A56C013822EA05024FEA67
:10CAD00051011A60E8D1B7E7276AC5E77448010039
:10CAE00080E100E084E100E088E100E001403F00F7
:10CAF00000003F8000E100E004E100E008E100E028
:10CB00002DE9F04F85B09946BDF93870BDF83CA0CD
:10CB1000BB1AC1EB090B002BB8BF5B42BBF1000F86
:10CB2000B8BFCBF1000B5B450D461646009380461F
:10CB300048DC4D453A4633464CDC194613460A4616
:10CB4000C5EB09019B1A89B2002B0CB2B8BF5B423E
:10CB500004EBD474BE42ACBF4FF0FF3201224D450E
:10CB6000039102924FEA640429DC9BB201930DE029
:10CB7000D8F80070BF69B847019BE41AA3B21CB291
:10CB80000135002C2DB211DBA94518DB009B5B455C
:10CB90002A46534631464046EADCD8F80020534640
:10CBA0009769294632464046B847E5E7029A164457
:10CBB000039AA94502EB030436B224B2E6DA05B0C3
:10CBC000BDE8F08F4A462B46B94635464D451746D7
:10CBD0001E46B2DD304629463E464D46074689464A
:10CBE000AEE700BF10B404682469A44610BC6047D7
:10CBF00030B40468BDF808500295A46BA44630BC5C
:10CC0000604700BF30B40468BDF808500295E46B7B
:10CC1000A44630BC604700BF70B40468BDF90C6026
:10CC2000BDF8105003960495246CA44670BC604770
:10CC3000704700BF10B582B0B0F90C2001910168B7
:10CC4000009200220C6CB0F90A301146A04702B0E5
:10CC500010BD00BF704700BF01F003010129C1757D
:10CC600006D0032904D0C28803894281838170479A
:10CC70000289C38842818381704700BF2DE9F0415A
:10CC80000568134E6F6986B0B7420446BDF8308020
:10CC900010D1013B13441BB20093CDF804800B4626
:10CCA000AD6A2046A8472368DB6AB3420AD106B0C2
:10CCB000BDE8F081059304920391B84703A9256864
:10CCC0000EC9E6E7204606B0BDE8F041184700BFB0
:10CCD00031CC00002DE9F0410568124E6F6986B035
:10CCE000B7420446BDF830800FD1013BCDF8048037
:10CCF0000B4400921BB2AD6A2046A8472368DB6A4A
:10CD0000B3420AD106B0BDE8F081059304920391C5
:10CD1000B84703A925680EC9E7E7204606B0BDE875
:10CD2000F041184731CC00002DE9F04F0568DFF8DD
:10CD300058B06F6985B05F450646BDF93890BDF8BB
:10CD40003CA00C46904615D11F19BC420CDACDF818
:10CD500000A0214601342D6A4B464246304624B29B
:10CD6000A847BC423568F2DBEB6A5B4507D105B0EA
:10CD7000BDE8F08F0393B8473568039BE4E730467E
:10CD800005B0BDE8F04F184731CC00002DE9F04365
:10CD900087B099420546BDF93840BDF83C6025D0C2
:10CDA000A24212D00768DFF88080D7F81490C145FE
:10CDB00032D18DE850002846BC6AA0472B68DB6A58
:10CDC000434524D107B0BDE8F083994202DD08460F
:10CDD0001946034628680E96C46B01335B1A1BB2D2
:10CDE0002846A44607B0BDE8F0436047A24202DDF2
:10CDF000134622461C4628680E96631C846B9B1AB9
:10CE00001BB22846A44607B0BDE8F0436047284659
:10CE100007B0BDE8F0431847059304920391C84753
:10CE200003A92F680EC9C4E731CC00002DE9F04FEB
:10CE3000D0F800E0DFF89090DEF814B083B0CB4576
:10CE40000446BDF93080BDF834A00D4617461E4695
:10CE500031D1CDF800A0DEF824B0294633463A4659
:10CE60002046D8472368CDF800A008F1FF323A44A5
:10CE7000D3F824B0294612B233462046D847236857
:10CE8000CDF800A02946D3F820B03A4643462046C4
:10CE9000D8472068CDF800A0711E29444346056A92
:10CEA00009B23A462046A8472368DB6A4B4506D1BB
:10CEB00003B0BDE8F08FD847D4F800E0C9E72046BA
:10CEC00003B0BDE8F04F184731CC0000F0B40024A7
:10CED00001264FF6FF75094F07600471C475C481C0
:10CEE00004824476C4618675067685824582C18057
:10CEF000028141818281F0BC704700BFA44D0100D6
:10CF00002DE9F04F85B00668BDF84450BDF9388072
:10CF1000CDF8008004460195D6F848B00392BDF9DB
:10CF20003C60BDF9407089469A46D8472368019510
:10CF3000009742465146D3F8488020463346C047C2
:10CF40002068039B0E930F95856C4B463A463146FD
:10CF50002046AC4605B0BDE8F04F60472DE9F04FE4
:10CF600087B01746BDF9404000912546E91D05935D
:10CF700044BF2B4603F10E010268BDF848605369B7
:10CF80000294C91003912B49BDF9444001968B428C
:10CF9000824645D1002C3CDD029B3C445E1EB6B26D
:10CFA0004FF0000923B2049301364D46029B002B3B
:10CFB00028DD059B002403EB090806E0EDB22B06F3
:10CFC00004F1010411D4A6421CD0A1B211F0070F44
:10CFD00023B24FEA4505F1D1002BB8BF0733DB1070
:10CFE000013418F803502B06EDD5009BD2F818B089
:10CFF00019443A4609B2019B5046D847A642DAF88E
:10D000000020E2D1039B01379944049B3FB2BB420D
:10D01000CCD1D36A074A934206D107B0BDE8F08F5E
:10D020009847DAF80020B5E7504607B0BDE8F04F62
:10D03000184700BF31CC000070B4BDF90C60BDF9D9
:10D040001050BDF8144003960495059470BCFFF78A
:10D0500085BF00BF2DE9F04F93B090460591C1699F
:10D060001090BDF870000790BDF874909DF878A0FE
:10D070000493002900F0CD800A7A0AC989460499F0
:10D080008A1AD2B203EBC203BAF1010FDA780B921B
:10D0900093F905201E8893F802B00F9293F9064089
:10D0A00079D913B2099323B20C93109B1A68A94B38
:10D0B0001193194653698B4240F0A6800B9B002BBD
:10D0C00055D01FFA88F300210D93C8462344DDF89C
:10D0D000409006910E930F460C46BBF1000F3FD0D7
:10D0E000BDF818100C9B03971FFA8AF0CB1813FB9E
:10D0F00000F304900E9801440D98034409B21BB24A
:10D100000A910893002505E00135EBB264009B45C8
:10D11000E4B222D9039B2B44590703D1731C18F89E
:10D1200006409EB22306EFD5099BBDF81000E91812
:10D1300011FB00F10598BAF1010F0FFA8AF30144CF
:10D140001CD0079801900093D26909B2174648464F
:10D15000089AB847D9F80020D6E7039F5F44FFB28A
:10D16000069B0B9901330693DBB29942B5D8D36A7B
:10D17000119A934243D113B0BDE8F08F0F9B191859
:10D1800093690A9A29441F4609B2079B4846B84743
:10D19000D9F80020B8E700230C93099385E70A9A91
:10D1A0000D9B0132013B52B213F0FF030A920D9323
:10D1B0006FD1DDF81890079BDDF83C80DDF820A0EA
:10D1C0004B4517D0BAF1010F00F0C8800B9A109DA3
:10D1D000CDF804900BEB8B014FEACB030A4400938C
:10D1E0001146DEF81C405346424609B22846A04785
:10D1F000D5F800E0DEF82C30119A9342BBD010989D
:10D2000013B0BDE8F04F1847109D284698472A688C
:10D2100054E7109A0598B2F90A308342ABDDB2F9AF
:10D220000C304345A7DD062313FB0A03002BA2DDC8
:10D2300008EBCA03002B9EDD537E2BB9049BAF2B5A
:10D2400002D90133DBB20493109BD3F800E0414BC9
:10D2500011931A46DEF81430934240F08E801FFA84
:10D2600088F30E9308339BB2BDF814200593052371
:10D270000D9300230A93CDF83C800FFA8AF3DDF872
:10D280004080CDF818900B921FFA8AFBCDF820A0B1
:10D2900099460A9ABDF810000B9C0E9D052319466D
:10D2A00011FB00232C481146C75C039702FB0B427D
:10D2B00014FA81F312B21BB209920C932C462E463B
:10D2C0001CE0089B0999012B2AB24B4640462DD001
:10D2D000079F0197CDF80090DEF81CA0D047D8F842
:10D2E00000E0039B5B0801340393059BA4B25D44FB
:10D2F0005E44A342ADB2B6B23FF451AF039BD80730
:10D30000DFD4079B069A9342EBD0089B012B16D0E3
:10D31000069B0193CDF80090DEF81CA009994B46BE
:10D3200032B24046D047D8F800E0DAE7DEF818A07D
:10D33000079B0C9922B2D047D8F800E0D1E7DEF87D
:10D3400018A00C991346404622B2D047D8F800E006
:10D35000C7E700BF31CC0000F44D01000B99109DD0
:10D36000CDF800900531DEF8204009B2424608238E
:10D370002846A047D5F800E03CE7109C2046984797
:10D38000D4F800E06BE700BFF0B5C36985B0044690
:10D390002BB30A2968D00D294AD01A7A914247D373
:10D3A000587A884244D35D688A1A05EBC205AA7888
:10D3B000002A50D0E87800284DD0207E00283AD0AE
:10D3C00095F905E0B4F90E00A67DB4F90A7072442F
:10D3D00006FB0202BA4262DCB4F9102030E00A29EE
:10D3E00056D00D2924D0027E002A4BD0B0F90E0071
:10D3F000A57DB4F90A60062212FB0502B2423EDDA9
:10D40000228AE38102EBC50212B218462282A78A61
:10D41000668A02950B468DE8C00001462046FFF75C
:10D4200019FEA37DE28903EB430302EB4303E3818F
:10D43000012005B0F0BDA67DB4F90E00B4F91020AE
:10D44000B4F814E0678A02960B468DE880400146E6
:10D450002046FFF7FFFD2979E389A27D012001FB2A
:10D460000233E38105B0F0BD0022C2819A7A817D4A
:10D47000038A01FB02330382012005B0F0BDB4F939
:10D480001020C4E7857DB4F91020B0F90E00BEE786
:10D49000028A817DC38102EBC1030382C8E70020B9
:10D4A000E0819B7A228A03FB062212B22282C7E71E
:10D4B000C1810282704700BF002908BF0121817528
:10D4C000704700BF81824182704700BFC07D7047B6
:10D4D000B0F90A00704700BFB0F90C00704700BFF8
:10D4E00010B4EFF3108272B6437F33B9017F012984
:10D4F00007D003290FD00123437702B962B610BCCD
:10D500007047124C2168A1B1114943610B688361D6
:10D5100008605861EFE70F4C216881B10E49436103
:10D520000B688361086058610C4B4FF080511960A3
:10D53000E1E7074B4161816120601860DBE7064B42
:10D540004161816120601860EEE700BFC8A0FF1F45
:10D55000C4A0FF1FB8A0FF1FBCA0FF1F04ED00E088
:10D5600070B5EFF3108272B60C4C206880B10C4E8F
:10D5700000254369236073B19D6102B962B64577A6
:10D5800083689847EFF3108272B620680028F0D1C4
:10D5900002B962B670BD3360EFE700BFB8A0FF1FED
:10D5A000BCA0FF1FFFF7DCBF184A30B41468002C82
:10D5B00027D0036821688B420ED2CB1A00218460E9
:10D5C000C1602360E06010600223037530BC7047C7
:10D5D00011688B42144608D3A2685B1A0360002AC4
:10D5E000F6D18260C460A060EEE7D268C260846059
:10D5F000E060C568CB1A0222A8602360027530BCC7
:10D6000070478460C4601060DEE700BFC0A0FF1FE9
:10D61000F8B5224E34682CB32368002B3AD1204F42
:10D620001D4604E03468ECB12368002B32D1A368B6
:10D6300003B1DD6020693360036825751B68BB4258
:10D6400021D1037F4560022BC46020D0FFF748FF43
:10D650006368002BE6D023602046FFF7A5FF3468FF
:10D66000002CE1D1EFF3108372B60E4A002110684E
:10D67000116003B962B628B18468FFF795FF2046B0
:10D680000028F9D1F8BD224600219847E0E78368D9
:10D690009847DDE7013B2360E4E700BFC0A0FF1F20
:10D6A00021BD0000D0A0FF1F024A136801331360A0
:10D6B000FFF7AEBFDCA0FF1F704700BF0368F0B4E8
:10D6C000FBB1002501249D60DC601B4C1A601C44EA
:10D6D000241104F144056A11032692009E60174F3D
:10D6E0000679174B47F8241002F1604202F56142B7
:10D6F00005F01F05012000FA05F5E6541560F0BCA1
:10D700007047104C236843F40003236000BF0E4BA6
:10D710000E4DA4F58734A4F59E7401261E602346A1
:10D7200004609C68002CD0D01033AB420360F8D169
:10D73000002303601846E2E7008FFCBFCC92FF1F76
:10D7400044E400E03C80044000700340407103402A
:10D750000168A9B10B4BF0B40B441B110A4E0B4FDF
:10D760000B4D46F8237003F1440202F01F0401231D
:10D770005211A340002445F822308C600460F0BCB4
:10D78000704700BF008FFCBFCC92FF1FB9D60000CE
:10D7900080E100E0024A034B012111601B68184739
:10D7A0000C710340CC92FF1F024A034B0121116010
:10D7B0005B6818471C710340CC92FF1F024A034B61
:10D7C000012111609B6818472C710340CC92FF1F08
:10D7D000024A034B01211160DB6818473C7103408A
:10D7E000CC92FF1FF8B50E4671B17AB107461446C8
:10D7F00000253B6816F8011B1B6838469847013C1A
:10D800000544F6D12846F8BD0846F8BD1046F8BDD7
:10D8100000B5064A036812885B6883B001A9ADF8B9
:10D8200004200222984703B05DF804FBF452010083
:10D83000F0B507468BB0002A33D0012A08BF0A2270
:10D8400051B3212400E0F4B2B1FBF2F502FB151153
:10D85000C8B2092900F1300198BFC8B20AA988BF2F
:10D860003730214488BFC0B201F8240C661E294617
:10D87000002DE8D133B1013CE4B20AAB23442D22A0
:10D8800003F8242C3B6801AA11195B683846C4F1DF
:10D89000220298470BB0F0BD30228DF825202124BC
:10D8A000E8E70368C9B21B6898470BB0F0BD00BF3A
:10D8B0000029BABF49422D2300230A22FFF7B8BF2F
:10D8C000374A384913681B06FCD40B6813F08003F1
:10D8D000F8D172B634490A78002A5FD0334A344806
:10D8E000F0B4344C176806682568D4680C303E44A0
:10D8F000143200681268304F35442C4420440244EE
:10D90000C2F34E022D4E2E482E4D2F4C42F40042B3
:10D910003A60376806682D682C4A24680C303E440B
:10D92000006812682A4F35442C4420440244C2F354
:10D930004E02284E2848294D294C42F400423A60B4
:10D94000376806682D68274A24680C303E44006812
:10D950001268254F35442C4420440244C2F34E0241
:10D96000224E2348234D244C42F400423A6037684B
:10D9700006682D68214A24680C303E44006812680D
:10D9800035442C4420440244C2F34E021C4842F465
:10D99000004202600B7062B6F0BC704762B670471E
:10D9A00024B0034024B00B40D5A0FF1F38B0034083
:10D9B0003CB0034040B003402CB0034058B003409B
:10D9C0005CB0034060B0034064B003406CB00340FF
:10D9D00030B0034038B00B403CB00B4040B00B407F
:10D9E00044B00B404CB00B402CB00B4058B00B4037
:10D9F0005CB00B4060B00B4064B00B406CB00B40AF
:10DA000030B00B4030B42948294A2A4B2A4D6024B3
:10DA1000E121047011701B78284C082B30D00A2BA0
:10DA20002748284937D00C2B0CBF35223D22122322
:10DA30002A60236002600B60234B24491B78244A30
:10DA4000BBB101230B601360224B23491B78234A8F
:10DA5000012B26D9042B0FD9082B1ED9102B94BFCC
:10DA6000862387230B6013601D4B01221A7030BC84
:10DA700070470B601360E7E784230B601360F3E7E4
:10DA800000F58E200F490830012213232A602360FD
:10DA900002600B60D0E73922F7E785230B60136043
:10DAA000E2E780230B601360DEE700BF0040074021
:10DAB00001400740DC92FF1F08B003400CB0034058
:10DAC00008B00B400CB00B40D8A0FF1F20B00340A3
:10DAD00020B00B40DD92FF1F24B0034024B00B4068
:10DAE000D5A0FF1F0C2830B417D91023984228BFA7
:10DAF00018461C46104A114D1178181A8C4228708D
:10DB000018D00F4913700B7823B10E490E4A002329
:10DB10000B60136030BCFFF775BF0A2802D90C23D5
:10DB20001C46E7E7082802D90A231C46E2E7082337
:10DB30001C46DFE730BC7047DC92FF1FD4A0FF1FFC
:10DB4000D5A0FF1F24B0034024B00B4028282FD8B5
:10DB5000334B2DE9F0411E5CFF2E2BD0314B1B784F
:10DB6000002B2AD132062CD472B62F4D2F4C2F46C3
:10DB7000012326602B7062B672B623681B060CD494
:10DB80003B781BB9F4E72B78002BF1D062B602F09A
:10DB900073FB72B623681806F5D5254B1B68002267
:10DBA0002A7062B6234A107843FA00F0BDE8F0818B
:10DBB000002070470020BDE8F081FFF781FE3206AB
:10DBC000D2D572B61C4DDFF87C801C4C06F04007A5
:10DBD000FFB206F03F06D8F80030DFB123F01003A3
:10DBE000C8F8003001232660134A2B7062B672B663
:10DBF000236819060CD413781BB9ECE72B78002B9B
:10DC0000E9D062B602F038FB72B623681B06F5D580
:10DC10000B4BC3E743F01003C8F80030E2E700BF46
:10DC2000F8520100D5A0FF1FD7A0FF1F00B003408E
:10DC300010B00340D4A0FF1FD6A0FF1F00B00B40C0
:10DC400010B00B400CB00B400A4A0B49136843F468
:10DC5000805313600B7843B9084BC0221A70084BED
:10DC600080F30C0000B218807047044B80221A70B9
:10DC7000F5E700BF2C800440D8A0FF1F21C00C4056
:10DC800000C00C40F0B51B4B1B4E596818689A68D1
:10DC9000DB6885B06C460FC4337899071DD5174AE9
:10DCA000174C1378174913F0700318BF1370164AF6
:10DCB000164B8027177000263320032226706D46EE
:10DCC00008701A7072B6043C45F001052046A8475A
:10DCD00062B6237813F0700309D10D4B064901E0B9
:10DCE000013B02D00A78D207FAD505B0F0BD237007
:10DCF00005B0F0BD245301000100024000000240C5
:10DD0000040002400B000240070002400A000240EB
:10DD1000410D0300B0F5006F0AD210B5094B1B7816
:10DD2000DB07044606D504F1A0500078C0B210BD50
:10DD300000207047FFF7A6FF04F1A0500078C0B2A2
:10DD400010BD00BF01000240B0F5006F17D238B51A
:10DD50000F4B1B78DA070D46044611D504F1A0508D
:10DD60000378AB420AD00B4A137813F0700318BF44
:10DD70001370074A05701378DB07FCD538BD704770
:10DD8000FFF780FF04F1A0500378AB42EBD1F5E739
:10DD9000010002400000024008B5F3F7F3FFF4F77A
:10DDA00039FF02F069FAFAE7844641EA000313F00A
:10DDB00003036DD1403A41D351F8043B40F8043B92
:10DDC00051F8043B40F8043B51F8043B40F8043B55
:10DDD00051F8043B40F8043B51F8043B40F8043B45
:10DDE00051F8043B40F8043B51F8043B40F8043B35
:10DDF00051F8043B40F8043B51F8043B40F8043B25
:10DE000051F8043B40F8043B51F8043B40F8043B14
:10DE100051F8043B40F8043B51F8043B40F8043B04
:10DE200051F8043B40F8043B51F8043B40F8043BF4
:10DE300051F8043B40F8043B403ABDD2303211D394
:10DE400051F8043B40F8043B51F8043B40F8043BD4
:10DE500051F8043B40F8043B51F8043B40F8043BC4
:10DE6000103AEDD20C3205D351F8043B40F8043B94
:10DE7000043AF9D2043208D0D2071CBF11F8013B92
:10DE800000F8013B01D30B8803806046704700BF58
:10DE9000082A13D38B078DD010F003038AD0C3F167
:10DEA0000403D21ADB071CBF11F8013B00F8013B49
:10DEB00080D331F8023B20F8023B7BE7043AD9D308
:10DEC000013A11F8013B00F8013BF9D20B780370DD
:10DED0004B7843708B7883706046704708B5104C60
:10DEE00008E0236859050DD423681A050FD4236868
:10DEF000DB0411D423685803F3D501F065F82368D7
:10DF00005905F1D502F01CFA23681A05EFD500F087
:10DF10007FFD2368DB04EDD500F0C8FEEAE700BF13
:10DF20003480044008B5FFF7D9FF00BF014B102231
:10DF30001A80704700200540704700BF094908B5A6
:10DF40000B6830B16A461844A2F58052904202D262
:10DF50000860184608BD03F0A5FC0C2303604FF0D1
:10DF6000FF3008BDE092FF1FFEE700BFEFF3138014
:10DF700070B9EFF310836BB9EFF305825AB94FF420
:10DF80008070EFF311832BB1984228BF1846704779
:10DF90004FF0FF3070470F2A01D81846F1E7014BC8
:10DFA000D05CEEE7F0E300E0F0B44D1E2E46002416
:10DFB00000E00134B0FBF2F302FB1300092800F18A
:10DFC00030078ABF3730F8B2C0B206F8010F1846E2
:10DFD000002BEED10A1953704CB1107815F8016F6F
:10DFE00028700133E01A834202F80169F5DB084624
:10DFF000F0BC7047704700BF10B40F4B53F830208F
:10E0000092F880422CB1012369B182F8803010BCB3
:10E01000704703EBC0035B681A6841B922F0020243
:10E020001A6010BC704782F8003110BC704742F093
:10E0300003021A6010BC7047345301001C4A02EB03
:10E04000C00301295B6811D004291BD052F83000AD
:10E05000002280F8802229B1022920D0032922D071
:10E060001A6070474FF480721A60704752F830009F
:10E070004FF4A27280F880121A601A6822F020020F
:10E080001A60704752F830104FF4A272012081F8E4
:10E0900080021A601A6842F020021A60704740F24B
:10E0A00003121A6070474FF481721A60704700BF04
:10E0B00034530100212848D8F8B5042A44D8DFE8B1
:10E0C00002F0484B4E0345004FF410262B4B03EB58
:10E0D000C0030D465C68216811F4E06148D0284B0C
:10E0E000284A2949C3F89C2104F140422748C3F833
:10E0F000A411A2F59221264FC3F8A0017C2925483E
:10E10000C3F8A871C3F8AC012CD9A2F594237C2BD9
:10E110002AD9A2F596237C2B28D9A2F598237C2B0B
:10E1200029D9A2F59A227C2A27D81B4872B62368DF
:10E1300023F4702343F08072C4F3840116432360F8
:10E1400040F82150266062B6F8BD70474FF4302683
:10E15000BCE74FF40026B9E74FF44026B6E74FF48A
:10E160002026B3E70D48E1E70D48DFE70D48DDE77E
:10E17000FFF764FFB3E70C48D8E7F8BD345301005C
:10E180000082FF1FF188FF1F9988FF1FC588FF1FAE
:10E190006D88FF1F4188FF1FBC93FF1FE492FF1F84
:10E1A0001C93FF1F6C93FF1F9C93FF1F1A4B03EBE5
:10E1B000C00010B4426802F14043A3F592217C29CB
:10E1C00023D9A3F594217C290DD9A3F596217C2987
:10E1D0001FD9A3F598217C2919D9A3F59A237C2B63
:10E1E00011D80E4C00E00E4C72B613680D4823F0A7
:10E1F0008773C2F3840123F4803343F08073136088
:10E2000044F8210062B610BC7047074CECE7074C9D
:10E21000EAE7074CE8E700BF34530100BC93FF1F57
:10E220001C93FF1FF5DF0000E492FF1F9C93FF1F6C
:10E230006C93FF1F30B4054B054D064C0022102196
:10E240001A602A602060196030BC704714D0034007
:10E2500004D0034000D00340282838B52ED0002930
:10E2600004464FDD5F4B1B78012505FA03F28A4215
:10E2700002D8212837D938BD0338C2B2012A3AD989
:10E28000202C4AD0192C48D0574A126802FB0112A0
:10E2900022FA03F31D2800F29B80DFE800F0928B46
:10E2A000847D9999766F999999999999999999688D
:10E2B000615A53994C99999999999945494B1B7869
:10E2C0000B2B08D90C2B1CBF0C3B19410846BDE891
:10E2D0003840FFF7B9BCC3F10C0399400846BDE8CC
:10E2E0003840FFF7B1BC2946FFF786FE2946BDE856
:10E2F0003840FFF7A3BE3D4A126802FB011222FA22
:10E3000003F3C7E72128B6D80021FFF775FE2046A2
:10E310000121BDE83840FFF791BE354A126802FB83
:10E32000011222FA03F3B5E73249334A0B604FF486
:10E330005173136038BD3149314A0B604FF451734A
:10E34000136038BD2F49304A0B6040F244431360DC
:10E3500038BD2E492E4A0B6040F24443136038BD4D
:10E360002C492D4A0B6040F24443136038BD2B49C1
:10E370002B4A0B6040F24443136038BD29492A4AB6
:10E380000B6040F24443136038BD2849284A0B60B3
:10E3900040F24443136038BD2649274A0B6040F2DF
:10E3A0004443136038BD2549254A0B6040F244437D
:10E3B000136038BD2349244A0B604FF45173136036
:10E3C00038BD2249224A0B604FF45173136038BDA7
:10E3D000212C3FF650AF7F29D4BF002101212046D8
:10E3E00093E700BFC493FF1F0880034008900340D9
:10E3F00008800B4010800B4048A0044018800B4060
:10E400004CA004401880034008B004401080034032
:10E4100004B004404080034018C0044038800340EA
:10E4200014C004402880034010B004402080034002
:10E430000CB004403080034010C0044048800340CA
:10E440001CC00440189003403490044010900340D6
:10E450003090044038B1102828BF1020044AC3B2BD
:10E46000107813707047024A0123107813707047B8
:10E47000C493FF1F2DE9F8430E4680463249334DC1
:10E48000304603F095F947F6122300281ABF1D46BF
:10E490004FF002094FF00109002425FA04F002F0C0
:10E4A00091FF4FF05E51074602F0E4FF014630460F
:10E4B00003F092F930B90134072CEED1E80902F0EB
:10E4C00081FF07463146384603F088F84FF07C510B
:10E4D00002F0C6FE03F0BAF94FF6FF729042A8F1BF
:10E4E000030328BF1046012B29D9B8F1170F17D8FD
:10E4F000174B23FA08F303F0010383F0010223B959
:10E50000B8F1190F0FD0BDE8F883124B124D134923
:10E510001A6044EAC9042A6008601C60BDE8F883F8
:10E52000B8F1200FECD10E4B0E4D0F49002244EAFA
:10E53000C9041A602A6008601C60BDE8F8830B4BB0
:10E540000B4D0C49F2E700BF001BB740006CDC022A
:10E550006006F00000800340048003400880034010
:10E5600000800B4004800B4008800B40009003406B
:10E570000490034008900340212801D8FFF73CBDD8
:10E58000704700BF212806D8044B53F8303093F869
:10E590000002C0B270470020704700BF3453010032
:10E5A000212801D8FFF74ABD704700BF72B60C4959
:10E5B0000C4B0D4A1B680868126862B6520102D5FE
:10E5C000322B88BF01300949C3F5BB334FF47A724F
:10E5D000FF33A1FB031302FB00F000EB9310704725
:10E5E000DCA0FF1F18E000E004ED00E0ABAAAAAA3F
:10E5F0002DE9F843054672B6204F214B214A1B688E
:10E600003C68126862B6520102D5322B88BF0134D1
:10E6100095B3C3F5BB331C4EDFF86490DFF864801C
:10E62000FF334FF47A72A6FB031302FB04F404EBEE
:10E63000931472B6D9F800103A68D8F800E062B6C0
:10E64000C1F5BB33FF33A6FB03031EF0806FC4EBA1
:10E6500093134FF47A7002D0322988BF013200FB45
:10E660000233B3F57A7F04D3013D05D004F57A7403
:10E67000DFE701F001FEDCE7BDE8F883DCA0FF1F67
:10E6800018E000E004ED00E0ABAAAAAAF8B52D4B13
:10E690002D49DFF8D0E0DFF8D0C02C4E2C4D2D4CAA
:10E6A0002D4A2E4F4FF4000018604FF08070186014
:10E6B0004FF0007018604FF0806018604FF00060FD
:10E6C00018600020086028234BF6FF71CCF800107A
:10E6D000CEF80030336013602B6023603B60B36280
:10E6E0009362092245F8242CC4F8D80F05F57F65FC
:10E6F000C7F8D41F07F5FF2707F5FA67C6F8F83FF4
:10E700002B6006F5FF26C4F8D42F05F5FD2504F58A
:10E71000FF24386006F2F4761148316005F5FF6594
:10E7200004F5FD642B6023600260FFF76BF919208C
:10E73000FFF75EFF01F08EF940F21310BDE8F840DC
:10E74000FFF756BF08E100E0048003401480034057
:10E75000248003402C8003401C800340348003400D
:10E7600000800B400C800340088003402B4A2C495A
:10E770001368F0B543F4006313600A78294F2A4EFA
:10E780002A4D2B4C2B490023092A3B7033702B70E8
:10E7900023700B703DD01A2A21D0274B1B780A2BEF
:10E7A00025D01F2B30D01F2827D800200246012556
:10E7B000224B234C1A7023495D7004224FF0020E45
:10E7C00088273C26402598729A704FF4004083F8C1
:10E7D00013E05A751F74DE7025700860F0BD1A4B87
:10E7E00040F213321A60144B1B780A2BD9D1174B05
:10E7F0004FF451721F281A60D7D9C0F34432C0F3C6
:10E80000471500F01F00D3E7114B4FF451721A6007
:10E81000C9E7104B40F213321A60BEE7348004405F
:10E82000C593FF1F50A1FF1FE5A0FF1F58A1FF1FA9
:10E8300051A1FF1FE4A0FF1FC693FF1F00B00640B9
:10E840002FE400E004E100E004D0044010B00440F4
:10E8500000D004400CB0044009B140F08000174AD9
:10E860001378984216D010B4154C246824050FD59F
:10E8700003F07F030A2B1CD01F2B11D0002900F0BE
:10E880007F0114BF602344230A290DD01F2902D021
:10E89000107010BC70470B4943F440730B60F7E7EE
:10E8A000084B00241C60E9E7074943F440730B6000
:10E8B000EEE7054B00241C60E0E700BFC693FF1F96
:10E8C0003480044000D0044010B00440124B1A7849
:10E8D00082420CD011490968090507D5092A16D0CA
:10E8E0001A2A0AD009280DD01A2801D018707047AA
:10E8F0000B4A40F213311160F8E7094A0021092858
:10E900001160F1D1074A40F213311160EEE7054A78
:10E9100000211160E6E700BFC593FF1F348004406B
:10E9200004D004400CB004402DE9F84F234B1B6881
:10E930001A053BD5224B1B680BB101221A70DFF878
:10E940009090204D99F80040DFF888801E4E0134E9
:10E95000272C8ABF4FF0000A5FFA84FA5446074614
:10E96000AB462B789C4216D1FFF700FB40281FDCFA
:10E9700033791B06F5D59BF800300133272B86BF72
:10E9800000221346DAB218F80330DBB2F3712A70B2
:10E990002B789C42E8D00D490B4BFFB20120BC22E2
:10E9A00008F80470087089F800A0DA70BDE8F88FE4
:10E9B000FF28D6DD01F060FCD3E700BF34800440BF
:10E9C00054A1FF1F51A1FF1F00B00640E4A0FF1F8C
:10E9D00058A1FF1FE8A0FF1F10B5044C237823B1F6
:10E9E00001F04AFC2378002BFAD110BDE4A0FF1FF0
:10E9F000054A064B10781B78C0B2DBB2984238BF8C
:10EA00004030C01A704700BF50A1FF1FE5A0FF1F94
:10EA1000F0B4384B1A7912F0300F2CD072B6997DC1
:10EA200001F0FF0200293DD062B6334F33493878F8
:10EA30000D78334E1C46C0B2EDB2431C402BE17939
:10EA400028BF0023AB4202F1FF32C9B21CBFF15410
:10EA5000184612F0FF02F0D12A4B1B68C2B23A707E
:10EA60004BB1A84236BFC5F14005401B40192728CD
:10EA7000C4BF01221A701F49CA78D2B2150616D433
:10EA800052060DD51B4B1B795B0609D51E4B1F4942
:10EA90001B6800220A7003B11A70164B3C22DA7010
:10EAA000F0BC70474022D9795A7462B6E3E70B791B
:10EAB0001C06E5D5164B174E1C783378E4B2DBB252
:10EAC0009C420ED0144D01E0A3420AD00133282B02
:10EAD00028BF00230879E85CC0B2C871087D072808
:10EAE000F2D9DBB2034933700B79180644BF7C239B
:10EAF000CB70C5E700B0064050A1FF1FE5A0FF1F87
:10EB000010A1FF1FE0A0FF1F54A1FF1FE4A0FF1FE3
:10EB100058A1FF1F51A1FF1FE8A0FF1F2DE9F84FCB
:10EB2000214B1B6807460BB101221A70DFF8889051
:10EB30001E4D99F80040DFF884801D4E0134272CCB
:10EB40008ABF4FF0000A5FFA84FA5446AB462B782E
:10EB5000A34216D1FFF70AFA40281FDC33791B06BF
:10EB6000F5D59BF800300133272B86BF00221346D2
:10EB7000DAB218F80330DBB2F3712A702B78A342B3
:10EB8000E8D00C490A4BFFB208F804700120AC220F
:10EB9000087089F800A0DA70BDE8F88FFF28D6DD8C
:10EBA00001F06AFBD3E700BFD0A1FF1FCDA1FF1F7B
:10EBB00000C00640CCA1FF1FD4A1FF1F64A1FF1F0E
:10EBC0001C4BDFF894C01A681B49F0B542F4805220
:10EBD0001A4D1A60DFF884E0194F1A4E1A4C0023C0
:10EBE0008CF800304FF451722B701F2840F213350F
:10EBF0008EF800303B70337025600A6012D81946D9
:10EC00000124124A124D11701248547000212C2711
:10EC1000402693724FF4003491701174D7702E70A7
:10EC20000460F0BDC0F34431C0F3471400F01F038B
:10EC3000E7E700BF348004400CC0044061A1FF1F1F
:10EC4000CDA1FF1FCCA1FF1F08C0044000C006409B
:10EC500031E400E004E100E060A1FF1FD4A1FF1F48
:10EC6000034B1B68DB0401D5FFF758BF704700BF9B
:10EC70003480044010B5044C237823B101F0FCFA31
:10EC80002378002BFAD110BDCCA1FF1F054A064BFB
:10EC900010781B78C0B2DBB2984238BF4030C01A3F
:10ECA000704700BF60A1FF1F61A1FF1F30B42B4B55
:10ECB0001A7994061FD52A48DA790378294901334D
:10ECC0003F2B0978C8BF00238B42D2B203D0264C19
:10ECD000D9B2E2540170254A116861B1244A127810
:10ECE000D2B2934236BFC2F140029B1A9B18272B27
:10ECF000C4BF01230B70194AD378DBB2180611D4B4
:10ED00005A060DD5154B1B795B0609D5194B1A49C7
:10ED10001B6800220A7003B11A70104B2C22DA70A3
:10ED200030BC704711790906EAD5144910480C78AF
:10ED30000178C9B28C420DD04A1C272A84BF002119
:10ED40000A460F4D054C98BFD1B2AA5CD2B2E2710F
:10ED50000170D5E76C21D170D2E700BF00C006403A
:10ED600060A1FF1F61A1FF1F8CA1FF1F5CA1FF1FFE
:10ED7000CDA1FF1FD0A1FF1FCCA1FF1FD4A1FF1F5A
:10ED800064A1FF1F21282FD8184B195CFF292BD015
:10ED9000174B184ADFF870C003EBC000F0B54368AA
:10EDA000DFF868E0144F154D154E00241C60DEF8A6
:10EDB0000030012043F020038840CEF8003014607A
:10EDC0004FF4A07338602E60C2F800C0013BFDD143
:10EDD00013689B05FCD42023013BFDD1094B09B2EC
:10EDE00033F8110080B2F0BD002070474454010098
:10EDF00034530100005004400850044004500440C3
:10EE0000000002030051044080014A0038800440A1
:10EE1000431E032B14D872B60A4951F8230068B177
:10EE200070B4094C058834F81320466841F8236013
:10EE3000521B24F8132062B670BC704762B670474C
:10EE40000020704730A2FF1FF8A3FF1F01380328DE
:10EE50000BD872B6074B53F8203043B100205B68E3
:10EE60000130002BFBD162B6704700207047184676
:10EE7000F9E700BF84A2FF1F30B472B62B4A1378A3
:10EE80001D0706D52A4B196A002936D0996A002930
:10EE900041D053781C0706D5254B196C00293ED06C
:10EEA000996C002939D09378190705D5204B196E34
:10EEB000002936D0996E89B1D3781B0707D51C4B32
:10EEC000D3F880207AB3D3F8882011213AB162B602
:10EED000184B00221A7030BC00F04ABE0D21154CB0
:10EEE000154D227843F8315003EBC1030830013A45
:10EEF0005860227062B630BC704704220D4C0F4D32
:10EF0000217843F8325003EBC20308304A1E5860A0
:10EF1000227062B6EFE70521E1E70921DFE7082269
:10EF2000ECE70C22EAE71022E8E700BF6854010092
:10EF30000080FF1FADA2FF1FC800400088004000F6
:10EF4000431E032B1DD81B4A400140F0100030B473
:10EF5000104472B6184CE25C032A1BD8DFE802F0BA
:10EF60000212151703220D88E25410F0080F14BF87
:10EF7000C823882343EA054308310360416062B631
:10EF800030BC704708300222EDE70522EBE708307D
:10EF90000422E8E7094A52F8230038B1084A52F837
:10EFA0002300416042F8231062B6E9E742F82310DB
:10EFB000034AF7E70080FF1FBCA2FF1F84A2FF1FC8
:10EFC00094A2FF1F00BE70472DE9F04FDFF818B381
:10EFD000DFF818A387B044E0AD4F4FEA930807EB82
:10EFE000C809013ED9F8042003F00803F6B2A2F1E3
:10EFF000080003F0FF04002B40F0018157F838307F
:10F000001B0C99B222F8081C002B00F0EF80A14BDA
:10F0100022F8064C42F8044C53F82620002A00F04F
:10F02000CF819D4D55F8263058609C4C45F8260000
:10F0300034F81630194424F8161000F079FD002831
:10F0400000F0C281964A974B19F0080F00F10800B2
:10F0500018BF1346C9F8040047F8383008238BF866
:10F0600000309BF80040E4B265071CD58E4B1B783E
:10F07000B3B18E490A7802F0FF0322B1013BDBB243
:10F080000B7003B900BE8A490A7802F0FF032AB167
:10F09000013BDBB20B70002B00F0688100F066FED4
:10F0A00004238BF8003004F0080303F0FF02002B68
:10F0B00000F0C9809AF80030DBB21E098CD19A08A2
:10F0C000DFF8CC9159F8321009EBC200C1F383018B
:10F0D000013940680C2900F28580DFE801F07A7A76
:10F0E0008383838383834683838307000168714D11
:10F0F0004068714F714E6860296088B240F281614A
:10F100000024674B49F832304FF0010E88423C60D2
:10F11000C9F81040C9F8184086F800E05C4A00F2CF
:10F12000E780B0F5D06F80F01B82B0F5817F00F0F2
:10F13000D98100F26981802800F02A82822840F07B
:10F14000D781A98801F07F01042900F2D1815C48B0
:10F150005C4A890008441470547001788C0740F1AF
:10F16000608382F800E0022173E1534F3A682AB3CA
:10F17000554B524E554819883478057840298E46AB
:10F1800045F0020828BF4FF0400E002C84F0010427
:10F190003470CEEB01010CBF8824C82409EBC806EB
:10F1A00089B285F0010544EA0E447260198049F87D
:10F1B000384072440570002965D03A603D4B1A888A
:10F1C000B2F5A06F0ED100219A785970404B1A7099
:10F1D00008E038493F4C0D68A54200F0988030495E
:10F1E00049F832103C4A0123137037E72C4A2D4B63
:10F1F00019F0080F18BF134647F838302EE700F013
:10F20000B7FC364A364952F82630002B00F0E3802E
:10F2100058688C5D42F8260003F10802C9F8042002
:10F22000032C05D8DFE804F02C02292602228A5597
:10F230001A8819F0080F0CBF8823C82343EA024339
:10F2400047F838300AE7E00700F19380210600F123
:10F25000D180A20706D5234A234913780220DBB2C6
:10F2600013700870E30602D51F4B10221A7007B006
:10F27000BDE8F08F04228A55DAE705228A55D7E7E0
:10F2800003228A55D4E7BEF1400F18BF002294E74D
:10F290000080FF1F30A2FF1FDCA1FF1FF8A3FF1F8C
:10F2A000C800400088004000B8A2FF1F41A2FF1F15
:10F2B0002CA3FF1FA4A2FF1FD8A1FF1F40A2FF1F66
:10F2C000C0200740B0A2FF1FECA1FF1FACA2FF1F90
:10F2D00098200740210900039420074084A2FF1FC3
:10F2E000BCA2FF1F882007408020074090200740D5
:10F2F000B0F5106F00F07C8140F2A38040F621123F
:10F30000904240F07B82A54A012313706AE74C6863
:10F31000A3498C427FF463AF0178A9297FF45FAFE2
:10F32000417845297FF45BAF8178C2297FF457AFDC
:10F33000C1786B297FF453AF9A489B4E017834789B
:10F3400081F00105002C41F0020105700CBF8820FE
:10F35000C82084F0010449F8310009EBC101934849
:10F360003470002505244D60047038E700F064FF18
:10F3700094E68F4B89488B491A614FF0020E80F852
:10F3800000E08C4F0A708C49196099608B4E8C4D4F
:10F390008C4C9A610D213970FF213170DFF84CE2FD
:10F3A00029702270884D894A8EF800109F27012409
:10F3B00006F8047C5D600470DA6007B0BDE8F08F89
:10F3C00043F82600824D30E6824A47F83800137829
:10F3D0000133137042E68B5D032B00F2BA8001A269
:10F3E00052F823F05DF000005DF000003DF40000F5
:10F3F00037F400006F49724B80220D2008701A709C
:10F40000A2077FF52FAF26E740F20232904240F08C
:10F41000ED81AA8802F07F02042A69D86D88002D48
:10F4200066D16449CDF804E0920011440A7842F0B4
:10F4300002020A70C1E101238B550FE600238B55B0
:10F440000CE6B0F5086F53D16349644A097811702E
:10F450007146ED888D4280F0E88252480478402D54
:10F46000AE4644F0020C28BF4FF0400E02EB0E03F4
:10F4700009EBCC01029301234A604FEA0E48CEEB20
:10F48000050101930025C82242EA080384F0010225
:10F4900049F83C3035700270DFF814C1424BDFF898
:10F4A000048149BBBEF1400F7FF42DAF42F0020C46
:10F4B00009EBCC03029ADFF8F8E05A608DBB0D042B
:10F4C00045F088059DF804304EF83C500A443370EE
:10F4D0000470134640297FF416AF0021404A3B6078
:10F4E000118010E7AA8802F07F02042A40F28B8183
:10F4F000304A0F23137006E74029D7D942F00202A1
:10F500000CEBC200029E4660BDB19DF80450354828
:10F510001D703346403988F8004040334CF83200C3
:10F52000DCE79DF8043033700D04029B047045F055
:10F53000C8050B444EF83C50CCE79DF804501D70B4
:10F54000029B1D4888F80040403940334CF8320097
:10F55000C4E719F0080F0CBF022303238B557DE588
:10F5600021494A68002AC3D06C88B5F804E003E05A
:10F570000C314A68002ABBD00B88A342F8D14B88D3
:10F580007345F5D1240A032C0CBF1178098960E773
:10F59000124A0221147054705BE700BF94200740A8
:10F5A00001000400ACA2FF1F40A2FF1F41A2FF1FE9
:10F5B0000080FF1FC02007408800400088200740CF
:10F5C0008020074098200740F0A1FF1F44A2FF1FA2
:10F5D000DCA1FF1FADA2FF1FB8A2FF1FB0A2FF1F3B
:10F5E000ECA1FF1FC80040006C5401008C200740B4
:10F5F000B248116AAC7804700C0600F19881D9F811
:10F600002820AF49100600F1DB81D9F83020AC4941
:10F61000120600F1D081D9F83820A949130600F16B
:10F62000C581D9F84020A649150600F1BA81D9F85C
:10F630004820A349140600F1AF81D9F85020A04911
:10F64000100600F1A481D9F858209D49120600F156
:10F650009981D9F860209A49130600F18E81D9F872
:10F6600068209749150600F18381D9F870209449E4
:10F67000140600F17881D9F878209149100600F13C
:10F680006D81D9F880208E49120600F16181D9F888
:10F6900088208B49130600F15581D9F890208849BC
:10F6A000150600F14981D9F898208549140600F122
:10F6B000FF808448844A854901908548854D864C61
:10F6C000049700230596029580460F4616461D4670
:10F6D0000394306828B1446800F04AFA2046002CB0
:10F6E000F9D100233360029B38681A46002342F8A0
:10F6F000253028B1446800F03BFA2046002CF9D1AF
:10F7000000223A60019A98F800301146002241F830
:10F71000042B039A0191023B4FF0000122F81510CF
:10F72000032B07D8DFE803F05D025D024FF0010311
:10F7300088F800300135042D06F1040607F10407AE
:10F7400008F10108C5D1654C654D2278654B049FD1
:10F75000059E0021100729701A7000F192806249FD
:10F7600062780A700021C9F83010C9F83810110702
:10F77000DFF84C816ED4A2785C49DFF844810A70CE
:10F7800000211207C9F85010C9F858104BD4E2787C
:10F7900057494B4C0A7013074FF00001C9F870101D
:10F7A000C9F8781000F1AE8033780193002283F01D
:10F7B0000105C9F89020C9F89820002102918846D7
:10F7C0008E460A464B48047844F0020C09EBCC0301
:10F7D0000393019B002B039B5A600CBF8822C82215
:10F7E00052E64FF0000388F80030A3E7B0F5A06FB1
:10F7F0007FF47EAE012300250193DEE740F621224F
:10F800009042F7D074E66D88002D7FF471AE3A49CE
:10F81000CDF804E0920011440A7822F002020A7046
:10F82000CBE7022115E600F083F9002800F0EB8019
:10F830000830324AC8F86400C8F8602000F078F94F
:10F84000002800F0DA8008302D4AC9F86C00C9F8A9
:10F8500068209CE700F06CF9002800F0E080083098
:10F86000264AC8F84400C8F8402000F061F9002892
:10F8700000F0CF800830224AC9F84C00C9F848206F
:10F8800079E700F055F9002800F0A58008301B4A00
:10F89000C9F82400C9F8202000F04AF9002800F037
:10F8A00094800830164AC9F82C00C9F8282056E779
:10F8B000D1F89C00083800F05BF9FAE6B8A2FF1F07
:10F8C0000080FF1F94A2FF1F30A2FF1F84A2FF1F12
:10F8D000BCA2FF1FDCA1FF1FF8A3FF1F685401009B
:10F8E000ADA2FF1FC4200740C8200740CC2007401E
:10F8F000D0200740ACA2FF1FC02007408800400076
:10F90000C800400000F014F9002870D008304F4AB9
:10F91000C4F88400C4F8802000F00AF9002860D000
:10F9200008304B4AC9F88C00C9F888203CE7506A77
:10F93000083800F01DF962E6D1F89400083800F0AC
:10F9400017F9B0E6D1F88C00083800F011F9A4E6F8
:10F95000D1F88400083800F00BF998E6C86F083831
:10F9600000F006F98DE6486F083800F001F982E6EC
:10F97000C86E083800F0FCF877E6486E083800F0EA
:10F98000F7F86CE6C86D083800F0F2F861E6486DEB
:10F99000083800F0EDF856E6C86C083800F0E8F8D2
:10F9A0004BE6486C083800F0E3F840E6C86B0838CE
:10F9B00000F0DEF835E6486B083800F0D9F82AE6A2
:10F9C000C86A083800F0D4F81FE62A78C9F8280079
:10F9D00001322A70C3E62A78C9F8200001322A7061
:10F9E0005AE72A78C9F8880001322A70DCE62A78BA
:10F9F000C4F8800001322A708EE72A78C9F86800BE
:10FA000001322A70C3E62A78C8F8600001322A70F1
:10FA100014E72A78C9F8480001322A70ABE62A7840
:10FA2000C8F8400001322A701FE740298E4628BFDF
:10FA30004FF0400E02EB0E0302930123CEEB0101C7
:10FA40004FEA0E4800250193BCE600BF8800400045
:10FA5000C8004000F8B500F0F9FC294B29482A4CB1
:10FA60002A4F2B4DDFF8BCC0DFF8BCE0294E002246
:10FA70001A605A609A60DA601A615A619A61DA61B2
:10FA80001A625A629A62DA621A635A639A63DA6392
:10FA90001A645A649A64DA641A655A659A65DA6572
:10FAA0001A665A669A66DA661A675A679A67DA6752
:10FAB000C3F880200168C3F8842041F480210160EC
:10FAC000C3F307212170C3F30740134938701B0E9D
:10FAD0002B70FF238CF80030104D8EF8003010484A
:10FAE0000B700123337084F8642070264FF4007487
:10FAF000102207F82C3C2E70046081F8F820F8BD25
:10FB00000080FF1F348004409C200740B020074045
:10FB1000B4200740942007401020074049E400E04B
:10FB200008E100E08020074088200740704700BFC0
:10FB300072B60D480268B2FA82F30F2B10DC4FF058
:10FB40000041D94022EA0102026062B6074803EB95
:10FB5000C303DB00C2180021C1501046516070473A
:10FB600062B60020704700BFC893FF1FBC83FF1F11
:10FB70000D4B0E4AC31AA2FB03231B090F2B0CD8F3
:10FB80000B4A127852B972B60A484FF00041026827
:10FB900021FA03F31A43026062B67047064A1278EC
:10FBA000002AF0D0FFF768B9BC83FF1F398EE33815
:10FBB000ADA2FF1FC893FF1FB8A2FF1F38B50E4BA1
:10FBC0000E4C1B68218805468BB1B1F5917F05D29B
:10FBD0000B4A4B1C55549BB2238038BD0022084869
:10FBE00098470021064A55540123238038BDB1F5BA
:10FBF000917FEDD338BD00BFE4A2FF1F02A4FF1F19
:10FC000008A4FF1F2DE9F843214E224F316801233C
:10FC100080463B70B1B1204D4B8801EB830201332C
:10FC200000240F2BC2F808802C7004D84B800023CE
:10FC30003B70BDE8F88340230B800320FFF780F979
:10FC40003460F4E7DFF8549099F80030002BF0D0DE
:10FC5000114D45F6215408E0013C12D02B7883B9B0
:10FC600000F00AFB99F800307BB10320FFF7EEF8B3
:10FC70000528F1D8FFF75CFF014630600028EBD083
:10FC8000CAE701232B70BDE8F883BDE8F88300BF05
:10FC900000A3FF1FD4A2FF1F04A3FF1FB8A2FF1FD2
:10FCA0001201F8B5D5B2A1B3012943D04378044677
:10FCB00000781B0643EA004040F4704045F004061B
:10FCC0008F1E3043FFF79EFF022F04F1020314D969
:10FCD000053414F8023C14F8032C14F8010C1B042E
:10FCE00043EA0223334343EA0060033FFFF78AFFFE
:10FCF000022F234604F10304EBD8022F23D0012F57
:10FD00000DD045F4774040F00500BDE8F840FFF71E
:10FD100079BF14482843BDE8F840FFF773BF18784F
:10FD200045F4770545F0060545EA0020BDE8F840B2
:10FD3000FFF768BF03780C4845EA03452843BDE850
:10FD4000F840FFF75FBF1A78587845F0774545F0DF
:10FD5000070545EA022545EA0040BDE8F840FFF7FF
:10FD600051BF00BF06F0F70007F000F738B5084BA9
:10FD70001C7824B9074D296809B14B8803B938BDEF
:10FD80009B000B800320FFF7DBF82C6038BD00BF21
:10FD9000D4A2FF1F00A3FF1F2DE9F041AD4E336831
:10FDA0000746002B00F092801D885A88910803EBCB
:10FDB00081010432AA428C6842D25A8004F00F06B4
:10FDC0004FEA1428A449A6F1080208F00F00C4F372
:10FDD0000313062A00F101050B701AD9B31E012B7B
:10FDE0005FFA88F04ED9052E48D0042E00F0A48189
:10FDF000731F022B7FD90F2E0ED1F72842D8F0287F
:10FE000002D0964B1B883BB1FFF7D8FE0020BDE81F
:10FE1000F08127B1BD4202D00020BDE8F081082E5C
:10FE2000C4F3033300F08780092E11D00A2E40F06E
:10FE300094800A2BF0D18A4B8A4A1B68A02181E06A
:10FE40001846FFF795FE0420FEF7E2FF3060B5E7A5
:10FE5000092BE1D1270E00F07B81834B814A1B687F
:10FE60009021C4F307461170EDB2FCB2002B00F0F4
:10FE70009D80224631462846984797E0F02843D98E
:10FE8000F72841D0F1380E28C6D801A353F820F046
:10FE9000470001002B0001001900010019FE0000BD
:10FEA00019FE00000B00010019FE0000EB0001002C
:10FEB00019FE0000B5000100CF000100F3FF0000B3
:10FEC00019FE0000DBFF0000BFFF0000674B1B783E
:10FED000002BA1D00420FEF79BFF034630600028D2
:10FEE0009AD00588002D7FF460AFFFF741FE3560A2
:10FEF0002846BDE8F081FFF761FEC4F30740FFF735
:10FF00005DFE072E02D1200EFFF758FE534B584AD4
:10FF1000198858481468584D524A017000270E0A33
:10FF2000F0201F802E7010700CB301225348A047A0
:10FF30000120BDE8F081082B7FF46EAF504B494A99
:10FF40001B688021C4F307461170EDB2240E6BB319
:10FF5000284622463146984728E00B2E11D10B2B1C
:10FF60007FF45AAF474B3F4A1B68B021EAE7464B44
:10FF70001B68002B00F0FB80404898470120BDE83B
:10FF8000F0810C2E40F000810C2B7FF445AF3F4BED
:10FF9000344A1B68C0211170EDB2C4F30746002B30
:10FFA00000F0C88028463146240E98473849314A27
:10FFB000314B0D7016701C700120BDE8F081354B7F
:10FFC0001B68002B00F0D6809847C4F30746254BEA
:10FFD000EDB2240E83F80080E8E72F4B1B68002B5E
:10FFE000F2D12E4B1B68A3B1FE209847C4F30746FD
:10FFF000EDE72B4B1B68002BE6D1284B1B6843B168
:020000021000EC
:10000000FC209847C4F30746E1E7264B1B68002B0A
:10001000DAD1C4F30746DAE7234B1B68C4F307467B
:10002000002BD4D030469847D1E7204B1A68002ADD
:10003000EFD0260C630C06F07F0003F47E531843C8
:10004000F6B29047C3E71A4B1B68C4F30746002B70
:10005000E8D1BCE70CA3FF1F06A4FF1F02A4FF1FEB
:10006000E8A2FF1F00A4FF1F1CA3FF1FB8A2FF1FD1
:10007000E4A2FF1F04A4FF1F05A4FF1F08A4FF1F85
:1000800014A3FF1F18A3FF1FFCA2FF1FD8A2FF1F6E
:1000900007A4FF1FC4A2FF1FC8A2FF1FCCA2FF1FFF
:1000A00008A3FF1FF8A2FF1F10A3FF1FE0A2FF1F5E
:1000B000F4A2FF1F3F4B1B68002B85D13E4B1B68F2
:1000C000002BA6D0FA209847C4F307467FE73B4BA6
:1000D0001B68002B7FF478AF374B1B68002B98D040
:1000E000FB209847C4F3074671E7354B1B68002B8C
:1000F0007FF46AAF304B1B68002B8AD0F8209847FA
:10010000C4F3074663E70E2B7FF486AE2D4A2E4BD1
:100110001268E0211970002A47D0260C610C06F005
:100120007F0301F47E511943EDB2A1F50051284639
:100130009047F6B2240E39E7FFF740FDC4F30740BD
:10014000FFF73CFD200EFFF739FD0020BDE8F081F0
:100150001E4B1D4A1B6880211170EDB2C4F3074687
:1001600083B1314628463A4698473C461EE701206F
:10017000BDE8F081104B1B68002B3FF44AAFFF2015
:10018000984746E71C4611E70D2EBCD10D2B7FF496
:1001900043AE0F4B0C4A1B68D0211170EDB2C4F373
:1001A0000746002B7FF4FEAEC4E7C4F30746EDB26A
:1001B000240EFBE6F0A2FF1FCCA2FF1FD0A2FF1F60
:1001C000C0A2FF1FDCA2FF1F00A4FF1F14A3FF1F7C
:1001D000ECA2FF1F38B5164D2868E0B101884488AD
:1001E000A14213DD03191B7A83B104F10803C2187D
:1001F0000C1B002302E012F8011F21B10133A342BE
:10020000F9D1204638BD1C46204638BDFFF7B0FC6A
:100210000020286038BD074B1B780BB9002038BD83
:100220000220FEF7F5FD28600028D7D1F6E700BFD1
:1002300028A3FF1FB8A2FF1F0D4B1B78BBB910B539
:100240000C4C216803F0FF024B883F2B07DC07337F
:100250000B4401F1470003F8012F8342FBD14023F7
:100260000B800120FEF76CFE0023236010BD704759
:1002700020A3FF1F24A3FF1F38B5224C237803B10E
:1002800038BD01232370FFF7A5FF70BB00F048F8CD
:1002900040BBFEF7ADFB10BBFEF7F8FCE0B9002356
:1002A0002370EFF30583002BEAD1EFF3108172B6D0
:1002B000154B1868E0B1154C2278CAB945691D6024
:1002C00001232370C5B1AA6101B962B60025457743
:1002D000836898472570D3E700F020F8DFE700F047
:1002E0001BF8D9E700F016F8D3E7FFF71FFCCDE7BE
:1002F0000029C5D162B638BD054B1D600029E5D186
:10030000E3E700BF2DA3FF1FC8A0FF1FCCA0FF1F66
:10031000C4A0FF1F704700BF704700BF704700BFF9
:10032000054A064B10781B78C0B2DBB2984238BF42
:100330004030C01A704700BF34A3FF1F35A3FF1F12
:10034000F0B4384B1A7912F0300F2CD072B6997D78
:1003500001F0FF0200293DD062B6334F33493878AF
:100360000D78334E1C46C0B2EDB2431C402BE179F0
:1003700028BF0023AB4202F1FF32C9B21CBFF154C7
:10038000184612F0FF02F0D12A4B1B68C2B23A7035
:100390004BB1A84236BFC5F14005401B4019272884
:1003A000C4BF01221A701F49CA78D2B2150616D4EA
:1003B00052060DD51B4B1B795B0609D51E4B1F49F9
:1003C0001B6800220A7003B11A70164B3C22DA70C7
:1003D000F0BC70474022D9795A7462B6E3E70B79D2
:1003E0001C06E5D5164B174E1C783378E4B2DBB209
:1003F0009C420ED0144D01E0A3420AD00133402BA1
:1004000028BF00230879E85CC0B2C871087D0728BE
:10041000F2D9DBB2034933700B79180644BF7C2351
:10042000CB70C5E700A0064034A3FF1F35A3FF1F14
:1004300078A3FF1F30A3FF1FBCA3FF1FB8A3FF1F9C
:10044000C0A3FF1FB9A3FF1F38A3FF1F70B584B05F
:1004500072B6194B194D1A48702241260F2480217B
:100460001A702E701A460470197013781B06FCD58A
:10047000144B186862B6144B144C984298BF00EBAA
:10048000800001A998BF40000A22FDF78DFD01A957
:100490002046002311F8012B01333AB10A2B20F832
:1004A000022FF7D11623237004B070BD5B00DBB2BE
:1004B000237004B070BD00BF00000240070002407E
:1004C00006000240080002407F9698009494FF1FA7
:1004D0002DE9F043DFF8EC808BB006460F4600F0C4
:1004E00073F898F90030013304460D4637D0304692
:1004F000394600F0DFF9002831D02BA3D3E90023DF
:100500003046394600F026FE814668BB28A3D3E971
:1005100000233046394600F0FFFD00B398F9003063
:10052000254ACDF82090042400200021022BCDE99B
:100530000467CDE9026700940192CDE906012CD051
:10054000684600F0BDF940B3089B1BB101F0AAF961
:10055000089B0360DDE906010BB0BDE8F08320468F
:1005600029460BB0BDE8F083134A98F90030019298
:1005700003210022CDE90467CDE9026700910892CA
:100580002BB90E4B4FF06042CDE90623D8E70C495A
:100590000020022BCDE90601D2D101F083F92223FC
:1005A0000360D1E7AFF30080EF39FAFE422E8640B8
:1005B00051302DD5104987C0D8540100FFFFEF47B7
:1005C0000000F07FAA94FF1F2DE9F04FB04F21F0FB
:1005D0000042BA4283B00C464FEAD17605460DD9A7
:1005E000AC4FBA4225D9C1F31303034340F0EF8067
:1005F0000EB10020014603B0BDE8F08FA64B9A4231
:1006000000F2CC80A54B9A4200F2DE808AA3D3E9A7
:10061000002300F05DF90022A14B00F09BFD0028B3
:1006200000F005812846214600229D4B00F050F93C
:10063000E1E783A3D3E9002300F08CFD002840F01C
:10064000CB802846214680A3D3E9002300F064FD37
:100650000028CED1934B284603EBC60821467CA345
:10066000D3E9002300F0E6FAD8E9002300F030F9DE
:1006700000F07AFD804600F077FA77A3D3E90023F3
:1006800006460F4600F0D6FA02460B46284621469B
:1006900000F01CF972A3D3E90023CDE90001304634
:1006A000394600F0C7FA82468B4652465B46DDE982
:1006B000000100F00BF905460C462A462346284661
:1006C000214600F0B7FA68A3D3E9002306460F4697
:1006D00000F0B0FA66A3D3E9002300F0F7F8324641
:1006E0003B4600F0A7FA64A3D3E9002300F0F0F83A
:1006F00032463B4600F09EFA61A3D3E9002300F0A6
:10070000E5F832463B4600F095FA5FA3D3E90023B3
:1007100000F0DEF832463B4600F08CFA02460B460B
:100720002846214600F0D2F806460F4628462146C4
:1007300032463B46B8F1000F56D000F07BFA324605
:1007400004460D463B4600204FF0804100F0BEF8C5
:1007500002460B462046294600F096FB02460B4611
:100760005046594600F0B2F8DDE9002300F0AEF83B
:100770000B4602464A49002000F0A8F86FF47F7348
:1007800098454FDA08F57A7801EB085100224FF0CE
:10079000B87300F04FFA03B0BDE8F08F424B9A42B5
:1007A0003FF658AF414BF4002344D3E9002300F057
:1007B0008DF83F4BC6F101081C44CDE90001D4E996
:1007C00000ABC6EB080870E74FF0000875E702467B
:1007D0000B4600F07DF80EE717A3D3E9002310467F
:1007E000194600F027FA06E700F024FA00228046B6
:1007F00089464FF080433046394600F067F802469C
:100800000B464046494600F03FFB2A46234600F08F
:100810005DF802460B460020214900F057F803B06E
:10082000BDE8F08F01EB085103B0BDE8F08F8046C2
:1008300043E700BFAFF300809C7500883CE4377E3F
:10084000EF39FAFE422E864051302DD5104987C02F
:10085000FE822B654715F73F0000E0FE422EE63F83
:10086000763C7935EF39EA3DD0A4BE726937663EF1
:10087000F16BD2C541BDBB3E2CDE25AF6A56113FA0
:1008800093BDBE166CC1663F3E5555555555C53F87
:10089000412E8640FFFFEF7F422ED63FFFFF2F3EC7
:1008A0000000F03FE0540100B1A2F03F005501000C
:1008B000F054010041F0004101F58010C00F704775
:1008C0000020704781F0004102E000BF83F0004348
:1008D00030B54FEA41044FEA430594EA050F08BFDB
:1008E00090EA020F1FBF54EA000C55EA020C7FEA9F
:1008F000645C7FEA655C00F0E2804FEA5454D4EB1C
:100900005555B8BF6D420CDD2C4480EA020281EAE5
:10091000030382EA000083EA010180EA020281EA1D
:100920000303362D88BF30BD11F0004F4FEA01316F
:100930004FF4801C4CEA113102D0404261EB41017E
:1009400013F0004F4FEA03334CEA133302D0524204
:1009500063EB430394EA050F00F0A780A4F10104C0
:10096000D5F1200E0DDB02FA0EFC22FA05F28018FA
:1009700041F1000103FA0EF2801843FA05F35941E0
:100980000EE0A5F120050EF1200E012A03FA0EFC5F
:1009900028BF4CF0020C43FA05F3C01851EBE37189
:1009A00001F0004507D54FF0000EDCF1000C7EEBA6
:1009B00000006EEB0101B1F5801F1BD3B1F5001FE4
:1009C0000CD349085FEA30004FEA3C0C04F1010403
:1009D0004FEA445212F5800F80F09A80BCF1004F2C
:1009E00008BF5FEA500C50F1000041EB045141EAAE
:1009F000050130BD5FEA4C0C404141EB010111F4AF
:100A0000801FA4F10104E9D191F0000F04BF014659
:100A10000020B1FA81F308BF2033A3F10B03B3F137
:100A200020020CDA0C3208DD02F1140CC2F10C02C7
:100A300001FA0CF021FA02F10CE002F11402D8BF25
:100A4000C2F1200C01FA02F120FA0CFCDCBF41EAF1
:100A50000C019040E41AA2BF01EB0451294330BDC0
:100A60006FEA04041F3C1CDA0C340EDC04F114049D
:100A7000C4F1200220FA04F001FA02F340EA030074
:100A800021FA04F345EA030130BDC4F10C04C4F1BA
:100A9000200220FA02F001FA04F340EA030029469A
:100AA00030BD21FA04F0294630BD94F0000F83F4E4
:100AB000801306BF81F480110134013D4EE77FEAC7
:100AC000645C18BF7FEA655C29D094EA050F08BF13
:100AD00090EA020F05D054EA000C04BF19461046F4
:100AE00030BD91EA030F1EBF0021002030BD5FEA38
:100AF000545C05D14000494128BF41F0004130BD60
:100B000014F580043CBF01F5801130BD01F00045B3
:100B100045F0FE4141F470014FF0000030BD7FEA26
:100B2000645C1ABF194610467FEA655C1CBF0B4621
:100B3000024650EA013406BF52EA033591EA030F38
:100B400041F4002130BD00BF90F0000F04BF002130
:100B5000704730B54FF4806404F132044FF0000563
:100B60004FF0000150E700BF90F0000F04BF0021DC
:100B7000704730B54FF4806404F1320410F0004542
:100B800048BF40424FF000013EE700BF42004FEA3D
:100B9000E2014FEA31014FEA02701FBF12F07F43BA
:100BA00093F07F4F81F06051704792F0000F14BFB7
:100BB00093F07F4F704730B54FF4607401F00045FB
:100BC00021F0004120E700BF50EA010208BF704752
:100BD00030B54FF000050AE050EA010208BF704747
:100BE00030B511F0004502D5404261EB41014FF4B0
:100BF000806404F132045FEA915C3FF4DCAE4FF0B4
:100C000003025FEADC0C18BF03325FEADC0C18BF9A
:100C1000033202EBDC02C2F1200300FA03FC20FAEB
:100C200002F001FA03FE40EA0E0021FA02F1144438
:100C3000C1E600BF70B54FF0FF0C4CF4E06C1CEA4D
:100C400011541DBF1CEA135594EA0C0F95EA0C0FC2
:100C500000F0DEF82C4481EA030621EA4C5123EA35
:100C60004C5350EA013518BF52EA033541F4801164
:100C700043F4801338D0A0FB02CE4FF00005E1FB17
:100C800002E506F00042E0FB03E54FF00006E1FB61
:100C900003569CF0000F18BF4EF0010EA4F1FF04A4
:100CA000B6F5007F64F5407404D25FEA4E0E6D41E4
:100CB00046EB060642EAC62141EA55514FEAC520F5
:100CC00040EA5E504FEACE2EB4F1FD0C88BFBCF571
:100CD000E06F1ED8BEF1004F08BF5FEA500E50F122
:100CE000000041EB045170BD06F0004646EA0101E8
:100CF00040EA020081EA0301B4EB5C04C2BFD4EB1A
:100D00000C0541EA045170BD41F480114FF0000E12
:100D1000013C00F3AB8014F1360FDEBF002001F080
:100D2000004170BDC4F10004203C35DA0C341BDCFA
:100D300004F11404C4F1200500FA05F320FA04F0CC
:100D400001FA05F240EA020001F0004221F0004100
:100D500010EBD37021FA04F642EB06015EEA430E73
:100D600008BF20EAD37070BDC4F10C04C4F12005A3
:100D700000FA04F320FA05F001FA04F240EA020056
:100D800001F0004110EBD37041F100015EEA430E27
:100D900008BF20EAD37070BDC4F1200500FA05F247
:100DA0004EEA020E20FA04F301FA05F243EA0203C6
:100DB00021FA04F001F0004121FA04F220EA0200D5
:100DC00000EBD3705EEA430E08BF20EAD37070BD1B
:100DD00094F0000F0FD101F00046400041EB0101FB
:100DE00011F4801F08BF013CF7D041EA060195F0DD
:100DF000000F18BF704703F00046520043EB030397
:100E000013F4801F08BF013DF7D043EA0603704783
:100E100094EA0C0F0CEA135518BF95EA0C0F0CD08E
:100E200050EA410618BF52EA4306D1D181EA0301D4
:100E300001F000414FF0000070BD50EA410606BFCE
:100E40001046194652EA430619D094EA0C0F02D113
:100E500050EA013613D195EA0C0F05D152EA033658
:100E60001CBF104619460AD181EA030101F0004176
:100E700041F0FE4141F470014FF0000070BD41F0BF
:100E8000FE4141F4780170BD70B54FF0FF0C4CF499
:100E9000E06C1CEA11541DBF1CEA135594EA0C0FB8
:100EA00095EA0C0F00F0A7F8A4EB050481EA030E05
:100EB00052EA03354FEA013100F088804FEA0333EC
:100EC0004FF0805545EA131343EA12634FEA0222BA
:100ED00045EA111545EA10654FEA00260EF000417B
:100EE0009D4208BF964244F1FD0404F5407402D2CD
:100EF0005B084FEA3202B61A65EB03055B084FEA5E
:100F000032024FF480104FF4002CB6EB020E75EB5A
:100F1000030E22BFB61A754640EA0C005B084FEA82
:100F20003202B6EB020E75EB030E22BFB61A7546FF
:100F300040EA5C005B084FEA3202B6EB020E75EB4A
:100F4000030E22BFB61A754640EA9C005B084FEAC2
:100F50003202B6EB020E75EB030E22BFB61A7546CF
:100F600040EADC0055EA060E18D04FEA051545EABE
:100F700016754FEA06164FEAC30343EA52734FEA67
:100F8000C2025FEA1C1CC0D111F4801F0BD141EAE0
:100F900000014FF000004FF0004CB6E711F4801F45
:100FA00004BF01430020B4F1FD0C88BFBCF5E06F25
:100FB0003FF6AFAEB5EB030C04BFB6EB020C5FEA35
:100FC000500C50F1000041EB045170BD0EF0004E8A
:100FD0004EEA113114EB5C04C2BFD4EB0C0541EABC
:100FE000045170BD41F480114FF0000E013C90E6B9
:100FF00045EA060E8DE60CEA135594EA0C0F08BF7D
:1010000095EA0C0F3FF43BAF94EA0C0F0AD150EA7B
:1010100001347FF434AF95EA0C0F7FF425AF10460E
:1010200019462CE795EA0C0F06D152EA03353FF436
:10103000FDAE1046194622E750EA410618BF52EAB3
:1010400043067FF4C5AE50EA41047FF40DAF52EA87
:1010500043057FF4EBAE12E74FF0FF3C06E000BF24
:101060004FF0010C02E000BF4FF0010C4DF804CD31
:101070004FEA410C7FEA6C5C4FEA430C18BF7FEAF1
:101080006C5C1BD001B050EA410C0CBF52EA430C1F
:1010900091EA030F02BF90EA020F0020704710F19F
:1010A000000F91EA030F58BF994208BF90422CBF2E
:1010B000D8176FEAE37040F0010070474FEA410C27
:1010C0007FEA6C5C02D150EA013C07D14FEA430C45
:1010D0007FEA6C5CD6D152EA033CD3D05DF8040BB6
:1010E000704700BF8446104662468C4619466346E8
:1010F00000E000BF01B5FFF7B7FF002848BF10F1BF
:10110000000F01BD4DF808EDFFF7F4FF0CBF012003
:1011100000205DF808FB00BF4DF808EDFFF7EAFF7F
:1011200034BF012000205DF808FB00BF4DF808ED3A
:10113000FFF7E0FF94BF012000205DF808FB00BF2F
:101140004DF808EDFFF7CEFF94BF012000205DF8B9
:1011500008FB00BF4DF808EDFFF7C4FF34BF0120C6
:1011600000205DF808FB00BF4FEA410212F50012B3
:1011700015D211D56FF47873B3EB625212D94FEADE
:10118000C12343F0004343EA505311F0004F23FAC8
:1011900002F018BF404270474FF00000704750EA1D
:1011A000013005D111F0004008BF6FF000407047DA
:1011B0004FF00000704700BF4FEA4102B2F1E04338
:1011C00024BFB3F5001CDCF1FE5C0DD901F0004C2E
:1011D0004FEAC0024CEA5070B2F1004F40EB83007E
:1011E00008BF20F00100704711F0804F21D113F1AA
:1011F0003872BCBF01F00040704741F480114FEAE3
:101200005252C2F11802C2F1200C10FA0CF320FA6B
:1012100002F018BF40F001004FEAC1234FEAD32388
:1012200003FA0CFC40EA0C0023FA02F34FEA4303F2
:10123000CCE77FEA625307D150EA01331EBF4FF07B
:10124000FE4040F44000704701F0004040F0FE4096
:1012500040F40000704700BF80F0004002E000BF93
:1012600081F0004142001FBF5FEA410392EA030F91
:101270007FEA226C7FEA236C6AD04FEA1262D2EBDB
:101280001363C1BFD218414048404140B8BF5B42E0
:10129000192B88BF704710F0004F40F4000020F079
:1012A0007F4018BF404211F0004F41F4000121F08F
:1012B0007F4118BF494292EA030F3FD0A2F10102D9
:1012C00041FA03FC10EB0C00C3F1200301FA03F117
:1012D00000F0004302D5494260EB4000B0F5000F3A
:1012E00013D3B0F1807F06D340084FEA310102F1F9
:1012F0000102FE2A51D2B1F1004F40EBC25008BFAB
:1013000020F0010040EA03007047490040EB000074
:1013100010F4000FA2F10102EDD1B0FA80FCACF1A3
:10132000080CB2EB0C0200FA0CF0AABF00EBC250A2
:1013300052421843BCBFD0401843704792F0000F90
:1013400081F4000106BF80F400000132013BB5E7E3
:101350004FEA41037FEA226C18BF7FEA236C21D059
:1013600092EA030F04D092F0000F08BF08467047BE
:1013700090EA010F1CBF0020704712F07F4F04D18C
:10138000400028BF40F00040704712F100723CBF9F
:1013900000F50000704700F0004343F0FE4040F4C9
:1013A000000070477FEA226216BF08467FEA236387
:1013B0000146420206BF5FEA412390EA010F40F472
:1013C000800070474FF0000304E000BF10F00043BE
:1013D00048BF40425FEA000C08BF704743F09643A5
:1013E00001464FF000001CE050EA010208BF7047C0
:1013F0004FF000030AE000BF50EA010208BF704747
:1014000011F0004302D5404261EB41015FEA010C5B
:1014100002BF84460146002043F0B64308BFA3F153
:101420008053A3F50003BCFA8CF2083AA3EBC25335
:1014300010DB01FA02FC634400FA02FCC2F1200254
:10144000BCF1004F20FA02F243EB020008BF20F08B
:101450000100704702F1200201FA02FCC2F12002F1
:1014600050EA4C0021FA02F243EB020008BF20EAE6
:10147000DC7070474FF0FF0C1CEAD0521EBF1CEA14
:10148000D15392EA0C0F93EA0C0F6FD01A4480EA02
:10149000010C400218BF5FEA41211ED04FF00063EB
:1014A00043EA501043EA5111A0FB01310CF0004017
:1014B000B1F5000F3EBF490041EAD3715B0040EA3D
:1014C000010062F17F02FD2A1DD8B3F1004F40EB0D
:1014D000C25008BF20F00100704790F0000F0CF0E0
:1014E000004C08BF49024CEA502040EA51207F3AA4
:1014F000C2BFD2F1FF0340EAC250704740F400007F
:101500004FF00003013A5DDC12F1190FDCBF00F06F
:1015100000407047C2F10002410021FA02F1C2F11D
:10152000200200FA02FC5FEA310040F1000053EAB9
:101530004C0308BF20EADC70704792F0000F00F007
:10154000004C02BF400010F4000F013AF9D040EA0D
:101550000C0093F0000F01F0004C02BF490011F4A1
:10156000000F013BF9D041EA0C018FE70CEAD1539F
:1015700092EA0C0F18BF93EA0C0F0AD030F0004C1F
:1015800018BF31F0004CD8D180EA010000F00040D3
:10159000704790F0000F17BF90F0004F084691F091
:1015A000000F91F0004F14D092EA0C0F01D14202CB
:1015B0000FD193EA0C0F03D14B0218BF084608D194
:1015C00080EA010000F0004040F0FE4040F40000DE
:1015D000704740F0FE4040F4400070474FF0FF0C71
:1015E0001CEAD0521EBF1CEAD15392EA0C0F93EAB8
:1015F0000C0F69D0A2EB030280EA010C49024FEA0A
:10160000402037D04FF0805343EA111143EA1013C2
:101610000CF000408B4238BF5B0042F17D024FF47A
:10162000000C8B4224BF5B1A40EA0C00B3EB510F55
:1016300024BFA3EB510340EA5C00B3EB910F24BF3E
:10164000A3EB910340EA9C00B3EBD10F24BFA3EBC3
:10165000D10340EADC001B0118BF5FEA1C1CE0D18B
:10166000FD2A3FF650AF8B4240EBC25008BF20F03E
:10167000010070470CF0004C4CEA50207F32C2BF92
:10168000D2F1FF0340EAC250704740F400004FF02F
:101690000003013A37E792F0000F00F0004C02BF60
:1016A000400010F4000F013AF9D040EA0C0093F02A
:1016B000000F01F0004C02BF490011F4000F013B84
:1016C000F9D041EA0C0195E70CEAD15392EA0C0FEC
:1016D00008D142027FF47DAF93EA0C0F7FF470AF24
:1016E000084676E793EA0C0F04D14B023FF44CAF67
:1016F00008466EE730F0004C18BF31F0004CCAD1FC
:1017000030F000427FF45CAF31F000437FF43CAF37
:101710005FE700BF4FF0FF3C06E000BF4FF0010C59
:1017200002E000BF4FF0010C4DF804CD4FEA40023B
:101730004FEA41037FEA226C18BF7FEA236C11D085
:1017400001B052EA530C18BF90EA010F58BFB2EB38
:10175000030088BFC81738BF6FEAE17018BF40F0B8
:10176000010070477FEA226C02D15FEA402C05D16C
:101770007FEA236CE4D15FEA412CE1D05DF8040BF1
:10178000704700BF844608466146FFE70FB5FFF784
:10179000C9FF002848BF10F1000F0FBD4DF808ED3C
:1017A000FFF7F4FF0CBF012000205DF808FB00BF2D
:1017B0004DF808EDFFF7EAFF34BF012000205DF887
:1017C00008FB00BF4DF808EDFFF7E0FF94BF0120D4
:1017D00000205DF808FB00BF4DF808EDFFF7D2FFD1
:1017E00094BF012000205DF808FB00BF4DF808ED14
:1017F000FFF7C8FF34BF012000205DF808FB00BFE1
:101800004FEA4002B2F1FE4F0FD34FF09E03B3EB0D
:1018100012620DD94FEA002343F0004310F0004F4D
:1018200023FA02F018BF404270474FF000007047A3
:1018300012F1610F01D1420205D110F0004008BF42
:101840006FF0004070474FF00000704742000ED22A
:10185000B2F1FE4F0BD34FF09E03B3EB126209D4EB
:101860004FEA002343F0004323FA02F070474FF0A1
:101870000000704712F1610F01D1420202D14FF016
:10188000FF3070474FF00000704700BF0B46014625
:10189000184600F001B800BF13460A460146022070
:1018A00000F0C0BE014B1868704700BFD898FF1FFA
:1018B00070B50F4E0F4D761BB61018BF002405D023
:1018C000013455F8043B9847A642F9D10A4E0B4D16
:1018D000761B03F01FFEB61018BF002406D001349B
:1018E00055F8043B9847A642F9D170BD70BD00BFC2
:1018F00020550100205501003455010020550100FC
:10190000024B0146186800F00BB800BFD898FF1FC3
:10191000024B0146186800F049BF00BFD898FF1F6E
:101920002DE9F04F01F10B05162D83B0064640F26C
:101930009F8035F0070500F1BF80A94200F2BC800E
:1019400000F058FBB5F5FC7FC0F09C826B0A00F0FC
:10195000BA80042B00F28381A80900F1390E4FEA06
:101960004E033830C44F07EB8303A3F108015C68D2
:10197000A14207D1ACE0002A80F2AC80E468A14229
:1019800000F0A680636823F003035A1B0F2AF2DDE0
:10199000B9493C6901F1080E744500F0B3816368F0
:1019A00023F003035A1B0F2A00F39981002AC1F880
:1019B00014E0C1F810E080F29E80B3F5007F80F063
:1019C0006781DB0803F1010C01229B1002FA03F38B
:1019D0004A6851F83C80C4F8088001EBCC091A43EE
:1019E000A9F10803E3604A6041F83C40C8F80C40A4
:1019F000831001249C40944200F28A80144206D154
:101A000020F003006400144200F10400FAD007EB58
:101A1000C009CC468046DCF80C108C4507D173E138
:101A2000002A80F28181C9688C4500F06D814B6885
:101A300023F003035A1B0F2AF2DD0C46D1F80CC029
:101A400054F8088F4B1945F001054D6042F0010133
:101A5000C8F80CC03046CCF808807B613B61C3F805
:101A60000CE0C3F808E059609A5000F0C5FA1FE096
:101A7000102921D800F0BEFA1025062302207E4F3F
:101A800007EB8303A3F108025C68944200F04581F0
:101A90006368E168A56823F00303234430465A686D
:101AA000E96042F001028D605A6000F0A5FA083446
:101AB000204603B0BDE8F08F00240C23204633609D
:101AC00003B0BDE8F08F80234FF0400E3F2049E780
:101AD00070465DE72344E1685A68A56842F0010258
:101AE000E96030468D605A6000F086FA083420467E
:101AF00003B0BDE8F08F234430465A6842F001023B
:101B00005A6000F079FA0834204603B0BDE8F08F3F
:101B1000BC68636823F00308A84504D3C5EB080339
:101B20000F2B00F38C80554BDFF860911A68D9F8C1
:101B3000003001332A4404EB080A00F0608102F50A
:101B400080520F3222F47F6222F00F02114630469B
:101B5000019200F04BFCB0F1FF3F8346019A00F088
:101B60005881824500F2FC80454B1968DA451144E2
:101B7000196000F05381D9F80000DFF810E101305E
:101B80001BBFCAEB0B0A5144CEF800B019601BF022
:101B9000070100F01781C1F10800C1F580518344AD
:101BA00008315A44C2F30B02C2EB010949463046E0
:101BB000019300F01BFC431C019B00F03F81CBEB29
:101BC00000024A4442F001021968C7F808B04944CB
:101BD000BC42CBF804201960DFF8A49016D0B8F10D
:101BE0000F0F40F2FD806268A8F10C0323F0070399
:101BF000E01802F001024FF0050E1A430F2B62604D
:101C0000C0F804E0C0F808E000F21C811D4BBC687D
